:100000000C94C91A0D94E7250D94BC250D949125E7
:100010000D9466250D943B250D9410250D94E52433
:100020000D94BA240C94FA1A0C94FA1A0C94FA1A35
:100030000C94FA1A0C94FA1A0C94FA1A0D94414082
:100040000C94FA1A0C94FA1A0C94FA1A0C94FA1AE0
:100050000C94FA1A0C94FA1A0C94FA1A0D9425239B
:100060000C94FA1A0D944D290D9423290C94FA1A24
:100070000C94FA1A0C94FA1A0C94FA1A0C94FA1AB0
:100080000C94FA1A0C94FA1A0C94FA1A0C94FA1AA0
:100090000D94BD2E0D94332E0D94752E0D94D941D3
:1000A0000C94FA1A0C94FA1A0C94FA1A0C94FA1A80
:1000B0000C94FA1A0C94FA1A0C94FA1A0C94FA1A70
:1000C0000C94FA1A0C94FA1A0C94FA1A0D94F92852
:1000D0000D94CF280C94FA1A0D94A5280D947B2822
:1000E0000C94FA1A07634236B79BD8A71A39685698
:1000F00018AEBAAB558C1D3CB7CC5763BD6DEDFD4A
:10010000753EF6177231BF000000803F0800000006
:10011000BE922449123EABAAAA2ABECDCCCC4C3EFC
:1001200000000080BEABAAAAAA3E00000000BF00EB
:100130000000803F0000000000084178D3BB4387E7
:10014000D1133D190E3CC3BD4282AD2B3E68EC82FB
:1001500076BED98FE1A93E4C80EFFFBE01C4FF7F80
:100160003F00000000000C945E660C9472FE0C943C
:10017000B1A90C941A3D0C948D540C94AF9E0C9420
:100180002FA50C94DC310D9416230D94B9200C94FA
:100190008D280C94B9480C94166A0C94CEF70D94E3
:1001A00036020C94B02E0C94352D0C9442F80C941D
:1001B0005DFE0C94A87A0D9425030C94ABB00C94BE
:1001C0006AC50C9435710C9408AA0C94EEA70C9493
:1001D00083A90C94FF1A0C9458CD0C94577D0C9461
:1001E00079FE0C94735E0D9474200C9477F20D9448
:1001F000F2020C94CE7A0C94C77A0C941B7C0C946B
:10020000066E0C94B7BA0C94E8AE0C9420F90C94DA
:10021000682C0C94A9CA0C94CCE10D942C020C947B
:1002200032DE0C94D41C0C940CF80C9431C50C9454
:10023000FFA80D9480380C9450240C9484B00C9436
:100240007FE20C94F3420C94E4A70C9447AD0C9419
:10025000F0310C94814B0C946C860C94B3E10C94AB
:10026000929E0D94A8470C9402700C949BCB0C9416
:100270001A8E0C94C2BA0C9454700D945C030D94B5
:100280001D030C947BCB0C94DCA50C940A7A0D9482
:1002900014020C943FE00C9461DE0D9468370C94CA
:1002A000C6AD0D9409200D94D3200C94A1540C9448
:1002B0008CB00D940D020C9408B80C9460A40C94AE
:1002C000761C0C942FDE0C942DDD0C949AAD0C94BE
:1002D0002DA70C944BAD0D946E1E0C9495D20C94DE
:1002E00085BA0D944A380C9417330C942E6F0C94E5
:1002F000061B0C94C2690C94ADAC0C944CB50C94D8
:100300005A290C9400310C949AA80C94B11B0C94AB
:1003100044BA0D941A220C94F5740C94A6B80C945B
:100320004FF20C94461C0C9438F80C94B1A60C9423
:100330006DDD0D9420210C94D21C0D941A020C94A6
:100340003EDE0C946BFE0D94FD200C9498A80C944A
:10035000CCA20C9493790C9480AC0D94DD1F0C947A
:1003600016F80D9440020C94AE3C0C94EB220D94C4
:10037000E1340D9498340C948A7A0D941E210C94D7
:10038000ADF20C94737D0C94217B0C9457BA0C94B1
:10039000F3BA0D946B1E0D94EA020C9465CA0C948A
:1003A00073E00C94A7E20C9431270D94E51E0C9495
:1003B00041700C944FDE0C9460BA0C942A490D9451
:1003C0006D1E0C94D8790C9466280C949EEB0D94B9
:1003D000FC360C940A4E0C94416F0C940E320C9423
:1003E000FAF90C949A790C94B03C0D942A200C9450
:1003F000B3AD0D94FA210C9443AD0C94C1F90C9457
:10040000EC1B0C941B3D0D94F7020C94576D0C944F
:10041000999E0C94ADBA0D9470030C948FD20C94E9
:100420003BAD0C944FFE0D94D2270D943F020C94DB
:10043000A8CB0D94D9370D9414210C94C6220C949A
:10044000064C0C94FAF70C94CF2F0C94CA3F0C94E2
:1004500072BA0D94B1090D9444020C949DE00C9471
:10046000D81C0C94167B0C9429F90C943F5E0C94C8
:10047000B9DD0C9498CB0C94723D0C94801C0C94B8
:10048000BD570C94997A0C94266F0C945D4C0C9487
:10049000CB690D9432020C94334C0D948F3F0C9425
:1004A00000B80C9408670C94B3A90C9452A40C9453
:1004B00014670C943E310C94F69E0C94511C0C94D1
:1004C000CC2C0C9437AD0C940D7A0C9456F20C9401
:1004D000A17A0D94A2090C94307B0C9441470C94A2
:1004E000E9E00C948A490C9433A90C949EAD0D94C8
:1004F0002F030D9474210D9415030D9466030C9431
:10050000B3540C94B2A70C94F9250C94E8A90C945C
:10051000EAAE0C94F75C0C94BF2C0C940C1C0C945D
:10052000F2310D94B7340D94CB210C941E310C9400
:10053000524B0C94A31B0C94C4BA0C9424DE0C9460
:10054000AA5D0C9424F80C9433AD0C9414A90D946A
:100550007A030C943B1C0C9408330D9424020C94E5
:1005600048A60C9447B10D94E8260D9428020C94EB
:100570007EA90C945FAC0C9497A70C943CE10C946E
:10058000A6DD0C94CF320C9457A90C948BA80C9434
:10059000771F0D94EC1F0C9491B60C9488CD0C949D
:1005A0001C250C949AAC0C94F73D0C94EC310D94F2
:1005B00022340C944CF80D94A3090C94C56B0C9444
:1005C000CCA70D9432220C94E0AD0C9496F20C94CE
:1005D0006FA80D9493470C94ECF70D94C31E0C94E4
:1005E000635D0C94C3420C940B7B0D9427380C94E0
:1005F000ADE20D94673B0D94F5200C947A1C0C949D
:100600005EA60D9438200C9404500C9449660C940A
:10061000D47A0C94FB480C94D9C50C94ED700C94CE
:10062000CB1B0D94F2310D94AA200C94EC7A0C940F
:10063000712C0C94707C0C94ED7C0D94E3200D9443
:10064000FE200C945D220C94DD7C0C94BAA80C94D2
:100650006A630C940E2C0C947C1C0C94FDB70C94C7
:100660001DB40C948F220D94EA200C9439280C941C
:100670007DAD0C94DA1C0C945ACD0C942A6F0C941A
:10068000AF3C0C9441DE0C943C7D0C947B690C9443
:10069000165E0D941E020C94DD320C9459A80D9434
:1006A000DA3B0C941CA50C945DAD0C94D8490C94C9
:1006B00091A90C940FF90C94BB530C9472A90C944F
:1006C0004CDE0C949AB60C94CFA70C94843F0C94F7
:1006D000C5320C94A0AD0D9411020C94FC1A0C942C
:1006E000694B0D947E1F0C940DB70C949CA60C9432
:1006F000EBCA0C9479E20C94006A0C9448AD0C940B
:10070000F25D0C9406B70C9428CA0C94D61C0C9479
:10071000E8420C94C6490C94CD260C9492DD0C94BE
:1007200040F90D9473210D94F2370C9485230D94A8
:1007300075210C94DEF70C9493E10D94311F0C9409
:1007400003B80C943CB40C943A9D0C94EDAD0D940C
:1007500009020C94C81B0D9405020C9448FE0C94DD
:1007600013A60C942FAD0C94381C0C94E7960C94A3
:10077000B8300D9452030C9485E20C943BA60C9473
:10078000CF5D0C94817A0D9484210C9467790D943B
:10079000DF330D9401030C94097C0C94ECA80D94A8
:1007A000CF200C94E4A50C9455540C9459CB0C9484
:1007B0007E1C0D940B030D94B4090C941C3D0D94F8
:1007C000FF010C9473540C94781C0C945C310C94C1
:1007D000377B0C94855D0D94C7330C94275E0C9485
:1007E0001CE10C9494B60C94F8A50C940FB20C94E4
:1007F000AC310C9456FE0C94DD7A0C9499BA0C949E
:100800003DA90C9403670C9468F20C94EBB30C9420
:10081000941B0D9439030D9484030C942DCB0C94EC
:10082000221D0D941B3F0D94D71E0C94EC750C9457
:100830009EB30C94FAB70C94DC1C0C943FAD0D9451
:100840003A020D947B200C9464A90D9497210C948A
:10085000B13C0C9455E10C94F17B0D9462200D9405
:10086000B41E0C9487AD0C944ACB0C944DBA0C94E6
:100870009B310C94C5860C940FC60C9442C60C9404
:10088000F4310D9400370C94AFF90D949E210D9422
:10089000B2380D94DF3E0C9486D20D9443030D9430
:1008A0006C1E0C94CD7B0C942EF80C94DCAD0C9447
:1008B000CAA80C947D3C0C94F7B70C94D9690C949D
:1008C000F94A0C94E1B90C9425A60C94C0764E41DB
:1008D0004E494E495459494E46CDCCCC3D0AD723BA
:1008E0003C17B7D13877CC2B329595E6241FB14F02
:1008F0000A000020410000C84200401C4620BCBE47
:100900004CCA1B0E5AAEC59D746364696E6F7073DA
:100910007578585B0041433A2053657269616C20D9
:1009200075736564206279204143202D20646973CA
:1009300061626C696E672073657269616C206C6FAF
:100940006767696E6720616E6420636D6400414370
:100950003A204F7574206F66206D656D6F72790057
:1009600041433A20496E69743A200041433A204499
:10097000652D496E69743A20004552520041433A50
:1009800020426164204352430041433A204F4B00D0
:10099000203E3E200041433A0041433A20506F6CD4
:1009A0006C696E670041433A20556E6D7574650041
:1009B000000000000000000000004F4E000000009A
:1009C000000000004F4646000000000000005245B5
:1009D0005354000000000000544F47474C450000AE
:1009E000000048414C54000000000000584F4E00E9
:1009F000000000000000584F4646000000000000C4
:100A0000494E4352454153450000444543524541F8
:100A100053450000454E41424C450000000044490A
:100A20005341424C45000000554E465245455A45FB
:100A30000000465245455A45000000004155544FBC
:100A400000000000000046414E5F4F4E4C59000030
:100A5000484947480000000000004D454449554DB5
:100A6000000000004C4F5700000000000000484507
:100A700041545F434F4F4C00484541540000000033
:100A80000000434F4F4C000000000000445259004A
:100A9000000000000000524742000000000000007B
:100AA0004853560000000000000072617700717525
:100AB000656974007377696E67006C6F636B0055CE
:100AC0006E6B6E6F776E2073756666697820005561
:100AD0006E6B6E6F776E20636D642000436F756E72
:100AE0007465723A2000444D582D4F757420496E3C
:100AF00069743A2000444D582D4F75742073746FFB
:100B0000703A200041737369676E65643A00444D22
:100B100058206374726C3A200069313600016933E1
:100B200032000275313600037533320004693868CB
:100B3000000569386C0006753868000775386C0068
:100B4000087831300009313030000A44656661753B
:100B50006C742073657269616C206D6F6465204EE2
:100B60003831207573656400384531002600384EF1
:100B700031000600384532002E00384E32000E009B
:100B8000384F31003600384F32003E0037453100D3
:100B90002400374532002C00374F31003400374FE6
:100BA00032003C00374E31000400374E32000C005A
:100BB000206164646564206279206E756D20004D4B
:100BC0004255533A2000416464696E67207265673C
:100BD00073207769746820616374696F6E733A007B
:100BE000416464696E67207265666572726564202F
:100BF000726567733A00416464696E67207072655C
:100C0000666574636820726567733A004D42555398
:100C10003A204D6F646275732074656D706C6174F9
:100C200065206E6F7420666F756E643A20004D42C9
:100C300055533A20496E76616C69642074656D7015
:100C40006C6174652E002C002C002C002C004D4291
:100C500055533A20636F6E666967206661696C65FB
:100C6000643A004D4255533A20636F6E66696720BF
:100C70006572726F72004D4255533A20636F6E6613
:100C80006967206C6F6164656420004D4255533A7A
:100C9000204F7574206F66206D656D6F7279004D01
:100CA0004255533A20506F6C6C696E6720657272C2
:100CB0006F7220004D4255533A204E6F7420737569
:100CC00070706F72746564207265672074797065E6
:100CD0000A004D425553443A2049676E6F7265646D
:100CE000202D20657175616C2077697468207365AB
:100CF000747465642076616C004D425553443A200B
:100D00004D61707065643A004D425553443A204E2F
:100D100065737465644D61707065643A004C61730D
:100D2000744B6E6F776E2076616C75653A20005358
:100D30006561726368696E67207265673A2000209A
:100D40006F7574206F662072616E676520627566CC
:100D50006665722C206665746368696E67006465F9
:100D600066207265672320004D425553443A205354
:100D70006561726368696E672072656723003A0077
:100D80002066726F6D207479706520004D42555356
:100D9000443A2020676F7420002076616C3A00206E
:100DA000004D425553207265733A20002076616CE5
:100DB000206E6F74206368616E6765642E20436FD8
:100DC0006E74696E7565004D4255533A003A206560
:100DD0007175616C20746172676572742E003D00DC
:100DE0004D4255533A002076616C206368616E670E
:100DF00065642E004D4255533A00204E6F773A00FD
:100E0000204C6173743A002023002070726566657F
:100E10007463682000205265672F636F696C206DD2
:100E200075737420626520696E740020696E746544
:100E3000726E616C2073656E64206572726F7220D1
:100E40002D206E6F207265672F636F696C002069BB
:100E50006E7465726E616C2073656E64206572726B
:100E60006F72202D206E6F2074656D706C617465DB
:100E70000020696E7465726E616C2073656E64200B
:100E80006572726F72202D206E6F2073746F7265A1
:100E9000004D425553443A20656E64506F6C6C208F
:100EA000004D425553443A20506F6C6C2000206E28
:100EB0006F7420666F756E64004D4255533A202062
:100EC000706172616D20002073656E64696E6720C9
:100ED00063616E63656C6C6564004D4255533A20E6
:100EE00020706172616D20004D4255533A20200000
:100EF0002073656E64206572726F722E20004D4201
:100F000055533A2020004164642040563A20002086
:100F100056616C3A20004D425553443A2073756631
:100F20006669783A00206F7220737566666978206A
:100F3000004D4255533A204E6F2074656D706C61C0
:100F4000746520666F7220004D6F746F723A207462
:100F5000696D656F757400556E6B6E6F776E20638B
:100F60006D64004D6F746F723A20466F72636564F2
:100F700020657865637574696F6E0056454E543A06
:100F800020636F6E666967206661696C65640056F0
:100F9000454E543A20696E69740056454E543A20C5
:100FA00050494420503D0056454E543A2044652D4A
:100FB000496E69740056454E543A204368616E206C
:100FC00062616C616E63653D0020736574205245FB
:100FD0005645525345206D6F64650056454E543A50
:100FE000205049443A2000207365742044495245FA
:100FF0004354206D6F64650056454E543A20504965
:10100000443A20002073657420524556455253459A
:10101000206D6F64650056454E543A20504153533D
:10102000205049443A2000207365742044495245B9
:101030004354206D6F64650056454E543A2050412C
:101040005353205049443A2000206F75743A0020D1
:101050007365743A0020696E3A0056454E543A2042
:1010600000204F75743A00205265713A0056454E83
:10107000543A2000206D33002066726F6D200020EE
:101080004D6178207265713A002066616E253A00E4
:101090002061637469766520563A0056454E543A8D
:1010A00020546F74616C20563A0056454E543A20D5
:1010B00076616C7565200041432061697220726F12
:1010C0006F6D74656D703A200056454E543A00417C
:1010D00043206D6F64653A200056454E543A0041F6
:1010E00043206169722074656D703A200056454E48
:1010F000543A005049443A20616C72656164792029
:10110000696E697469616C697A6564005049443A32
:1011100020496E76616C696420706172616D206136
:10112000727261792E002C002C002C002C0050498A
:10113000443A20636F6E666967206661696C656416
:101140003A005049443A20636F6E666967206572C1
:10115000726F72005049443A20636F6E666967206F
:101160006C6F6164656420005049443A204F757487
:10117000206F66206D656D6F7279005049443A208A
:1011800044652D496E69742000203C414C4D3E0061
:1011900020443A0020493A0020503A0020696E3A33
:1011A00000207365743A005049443A200050494485
:1011B0003A20496E76616C696420706172616D20BD
:1011C00061727261792E00536574206F757420749A
:1011D0006F20002050494420616C61726D2E200008
:1011E0002050494420616C61726D3A20636C6F73CA
:1011F0006564005049443A20556E6B6E6F776E20DF
:1012000073756666697820005049443A20556E6BC4
:101210006E6F776E20636D64200020536574706F6D
:10122000696E743A005049443A200020496E707546
:10123000742076616C75653A005049443A2000206C
:10124000696E697400200050574D2D4F757420232E
:10125000002073746F7000200050574D2D4F75742F
:101260002023003D0050696E3A0020696E697400C9
:1012700070696E230072656C61794374723A200064
:101280002073746F700052656C61792D4F757420F6
:10129000230072656C61794374723A200069646C52
:1012A00065006F66660068656174696E67006661F7
:1012B0006E00647279696E6700636F6F6C696E6748
:1012C00000616374696F6E0020697320004F75744C
:1012D000200072656C61794374723A2000556E6B20
:1012E0006E6F776E20737566666978200072656C24
:1012F00061794374723A2000556E6B6E6F776E2081
:10130000636D64200072656C61794374723A2000E9
:10131000616374696F6E0072656C61794374723ACF
:10132000200053686F770020636D643D002D005BE3
:10133000305D3A2000202D202D202D20EFBBBF0056
:101340003E003E31202D20005B305D3A2000202DF4
:10135000202D202D20EFBBBF003E003E31202D2050
:10136000005379736C6F6720726573756D656400E7
:101370005379736C6F6720726573756D6564005384
:1013800079736C6F672073757370656E6465640044
:101390000000000000636D64000073657400007657
:1013A000616C000064656C000048535600005247B1
:1013B00042000066616E00006D6F646500637472C8
:1013C0006C006875650000736174000074656D7071
:1013D00000726177000020002E00696E00735F6F5D
:1013E0007574006D79686F6D65004354524C2F65BC
:1013F0007865633A204F75744F664D656D6F7279ED
:101400003A2000202D3E20004D5154543A20002017
:101410002D3E2000456D69743A203C00202D3E2071
:10142000004974656D436D643A2000202D3E200014
:101430004974656D3A20004D423A204E6F74207316
:101440007570706F7274656420726567207479704E
:10145000650A002056616C3A30780020543A00202A
:101460005265673A3078004D423A20416464723ADE
:1014700000444D58000000000000444D58524742BF
:10148000570000444D5852474200000050574D004D
:1014900000000000004D42555344494D000054489F
:1014A00045524D4F00000052454C4159000000008C
:1014B00047524F555000000000564354454D5000D0
:1014C00000004D42555356430000004143484149F6
:1014D000455200005350494C45440000004D4F54C4
:1014E0004F52000000005049440000000000004D31
:1014F00042555300000000005541525442524447A7
:101500000052454C415950574D00444D58524742A6
:1015100057570056454E545300000000454C455661
:1015200041544F5200434F554E54455200004855C8
:101530004D0000000000004D455243555259000037
:1015400020002D3E00436F6E76657274696E6720D1
:10155000002D3E0057726F6E672041737369676E8E
:101560006D656E742000524742783A200020764C18
:101570006576656C3A0020436F6E76563A002043DC
:101580006F6E76533A0020486F743A00436F6C6474
:101590003A0020436F6E76657274656420563A0097
:1015A000436F6E76657274656420533A002D3E0079
:1015B00057726F6E672041737369676E6D656E74E5
:1015C00020002D3E0057726F6E672041737369676C
:1015D0006E6D656E7420004D41503A2076616C202E
:1015E0006D617070656420746F2020004D41503A29
:1015F0002076616C75652061626F7665207269671F
:10160000687420626F756E642000206973206265C3
:101610006C6F77206C65667420626F756E64200055
:101620004D41503A2076616C756520004D41503A2D
:1016300020636D64206D617070656420746F20009C
:10164000000000000000000000004F4E00000000FD
:10165000000000004F464600000000000000524518
:101660005354000000000000544F47474C45000011
:10167000000048414C54000000000000584F4E004C
:10168000000000000000584F464600000000000027
:10169000494E43524541534500004445435245415C
:1016A00053450000454E41424C450000000044496E
:1016B0005341424C45000000554E465245455A455F
:1016C0000000465245455A45000000004155544F20
:1016D00000000000000046414E5F4F4E4C59000094
:1016E000484947480000000000004D454449554D19
:1016F000000000004C4F570000000000000048456B
:1017000041545F434F4F4C00484541540000000096
:101710000000434F4F4C00000000000044525900AD
:1017200000000000000052474200000000000000DE
:101730004853560000000000000020537566663ACA
:10174000002041543A0053746F7070696E672049ED
:101750006E7075747300206973200044656C657445
:10176000696E6720636F6E662E2052414D2077614F
:10177000733A0053746F70706564006E6F746869BB
:101780006E6720746F2073746F700053746F707085
:10179000696E67206368616E6E656C73202E2E2EF5
:1017A0000043616E206E6F7420636C65616E202D46
:1017B000206C6F636B6564004D5154543A20436F45
:1017C0006D706C6574652E2052656D6F7665207442
:1017D0006F706963200024636F6D6D616E64004DEE
:1017E0005154543A20436C65616E55702072657493
:1017F00061696E656420746F706963200022002245
:10180000004F75744F664D656D6F727921005D20D4
:10181000003A5B004D5154543A005D00456D7074C0
:10182000793A205B000A003A004D41433A005544A2
:1018300050205379736C6F6720696E697469616CAD
:10184000697A65642E0A005379736C6F6720706142
:1018500072616D733A002E6C6F63616C0053657238
:1018600076696365207265636F72643A20006D4427
:101870004E5320726573706F6E646572207374616D
:10188000727465642E004572726F72207365747491
:10189000696E67207570204D444E532072657370D9
:1018A0006F6E6465722100476F7420495020616437
:1018B00064726573733A00276970205B69705B2CF2
:1018C000646E735B2C67775B2C7375626E65745DF9
:1018D0005D5D5D27202D20736574207374617469CC
:1018E000632049500A004661696C656420746F206A
:1018F000636F6E6669677572652045746865726EA0
:101900006574207573696E6720444843502E2059D2
:101910006F752063616E20736574206970206D613E
:101920006E75616C6C792100204D41534B3A00205B
:1019300047573A0020444E533A004C6F6164656447
:101940002066726F6D20666C6173682049503A00A2
:101950000A7573657320444843500A0053746172DA
:1019600074696E67206C616E004D5154543A207456
:10197000727969796E67206E656E78742062726F15
:101980006B6572004D5154543A20546F6F206D6155
:101990006E7920636F6E6E656374696F6E20657219
:1019A000726F72732E2052657374617274204C4191
:1019B0004E002074727920616761696E20696E2023
:1019C00035207365636F6E6473004D5154543A2033
:1019D0006661696C65642C2072633D004D515454FE
:1019E0003A204177616974696E6720666F72207270
:1019F000657461696E656420746F706963730063F8
:101A00006F6E6E65637465642061732000202E2EF6
:101A10002E0020757365723A003A000A4D515454F5
:101A20003A20417474656D7074696E6720636F6EDF
:101A30006E656374696F6E20746F200064697363F0
:101A40006F6E6E6563746564005573696E67204DD3
:101A50005154542070617373776F72642066726F93
:101A60006D20636F6E666967002E6C6F63616C003A
:101A70006D444E53206E616D6520757064617465B0
:101A8000643A2000446576696365204E616D653A6D
:101A9000004D5154543A204174206C656173742098
:101AA000646576696365206E616D6520616E642092
:101AB00062726F6B6572204950206D75737420627D
:101AC0006520636F6E6669677572656400246E6F6A
:101AD000646573004F4E2C4F46462C48414C542CA5
:101AE000524553542C584F4E2C584F46462C544F69
:101AF00047474C450024666F726D617400656E75D2
:101B00006D00246461746174797065006873760097
:101B1000636F6C6F7200302D32353500696E7465FD
:101B200067657200666C6F617400332E302E310071
:101B300024686F6D696500757074696D652C6672D7
:101B400065656865617000343063316663615F327A
:101B50003032362D30312D3130004C696768744891
:101B600075622000246E616D6500526562696E6465
:101B700020737563636573732E204950206164641C
:101B8000726573733A004572726F723A20726562C1
:101B9000696E64206661696C0052656E6577656484
:101BA00020737563636573732E20495020616464EC
:101BB000726573733A004572726F723A2072656E85
:101BC00065776564206661696C000A4E6F206C69F8
:101BD0006E6B00436F6E74696E756520776974680B
:101BE0002070726576696F75736C79206C6F6164B3
:101BF000656420636F6E6669670033307320454506
:101C000050524F4D206973206E6F742072656C6F57
:101C1000616465642E205265626F6F74004D51548B
:101C2000543A20416363657074696E6720636F6D19
:101C30006D616E64732E2E2E0A004E6F204D51542E
:101C40005420636F6E66696775726564004C6F61DE
:101C500064696E6720636F6E6669672066726F6D78
:101C600020706F7274616C2064697361626C65646A
:101C70002E2075736520676574204F4E20746F2089
:101C8000656E61626C6500436F6E6669672069739B
:101C90002076616C696400436F6E74696E756520AF
:101CA000776974682070726576696F75736C7920D6
:101CB0006C6F6164656420636F6E6669670053656D
:101CC000747570204F5441004D5154543A2073653F
:101CD000742066697273742062726F6B6572004360
:101CE000757272656E74204C414E20636F6E66692A
:101CF000672869702C646E732C67772C7375626E1D
:101D00006574293A000A5573652074686573652007
:101D1000636F6D6D616E64733A202768656C702720
:101D2000202D207468697320746578740A276D61AA
:101D3000632064653A61643A62653A65663A66654D
:101D40003A3030272073657420616E642073746F9D
:101D50007265204D41432D6164647265737320691F
:101D60006E20454550524F4D0A276970205B6970BF
:101D70005B2C646E735B2C67775B2C7375626E658E
:101D8000745D5D5D5D27202D207365742073746123
:101D90007469632049500A277361766527202D20D6
:101DA000736176652063757272656E7420636F6E01
:101DB00066696720696E204E5652414D3B204F4E5A
:101DC0007C4F4646202D20656E61626C652F6469EC
:101DD0007361626C65206175746F736176650A2743
:101DE00067657427205B636F6E6669672061646452
:101DF000725D27202D2067657420636F6E666967AA
:101E00002066726F6D207072652D636F6E666967F4
:101E1000757265642055524C20616E642073746F36
:101E2000726520616464722C204F4E7C4F464620C0
:101E30002D20656E61626C652F64697361626C65EB
:101E400020646F776E6C6F6164206F6E20737461B5
:101E5000727475700A276C6F616427202D206C6F77
:101E6000616420636F6E6669672066726F6D204ED5
:101E70005652414D0A2770776427202D20646566ED
:101E8000696E6520616E642073746F7265204D51B8
:101E900054542070617373776F72640A276F746192
:101EA00070776427202D20646566696E6520616EF9
:101EB000642073746F726520485454502041504917
:101EC0002070617373776F72640A276C6F67205B91
:101ED00073657269616C5F6C6F676C6576656C5D6C
:101EE000205B7564705F6C6F676C6576656C5D27F1
:101EF000202D20646566696E65206C6F67206C65B7
:101F000076656C2028302E2E37290A276B696C6C79
:101F100027202D2074657374207761746368646F63
:101F2000670A27636C65617227202D20636C6561E9
:101F30007220454550524F4D0A27736561726368A0
:101F400027202D2073656172636820312D776972B7
:101F500065206465760A277265626F6F7427202D8D
:101F6000207265626F6F7420636F6E74726F6C6C39
:101F7000657200536F6674207265626F6F74696E6C
:101F8000672E2E2E00206E657700206973200031A9
:101F900057543A003157543A205365617263686967
:101FA0006E67206465760052414D3D000A53797397
:101FB0006C6F6720000A312D7769726520000A6D09
:101FC00071747420000A6D6F64627573207632003C
:101FD0000A6D6F6462757320763120282B29000A00
:101FE000696E7075747320000A6974656D732000E2
:101FF0000A436F6E666967757265643A002F00491F
:102000006E3A2000496E697469616C697A696E671D
:1020100020496E70757473003157543A207365749B
:102020007570207265736F6C7574696F6E20003106
:1020300057543A204453323438322D313030206EE8
:102040006F742070726573656E74003157543A2056
:102050004453323438322D313030204932432072EB
:102060006573746F726564003157543A204275731A
:10207000207265736574206572726F7200315754F7
:102080003A2042757320526573657420646F6E65E3
:10209000003157543A204453323438322D313030E5
:1020A0002070726573656E742C20726573657400A0
:1020B0004572726F7220312D7720696E697400311C
:1020C00057543A204453323438325F3130305F490C
:1020D00032435F544F5F31575F4252494447452076
:1020E000696E697400444D584F75742E20467265B0
:1020F000653A00444D58696E2042756666657220E7
:10210000616C6C6F632065727200496E697420693E
:102110006E2063683A003B003D0050696E3A003B18
:10212000003D4C4F5700546865726D6F3A004F6E1A
:102130006520776972652052656164790A0046728C
:1021400065653A00444D58206F7574207374617250
:102150007465642E204368616E6E656C733A20006E
:10216000444D5820696E20737461727465642E202A
:102170004368616E6E656C733A0042726F6B657294
:102180007320636F6E666967757265643A004170AB
:10219000706C79696E6720636F6E666967004C6F5B
:1021A0006164656420455441473A004E6F20737462
:1021B0006F72656420636F6E666967004C6F61645F
:1021C00065642066726F6D20454550524F4D006C1E
:1021D0006F6164206661696C6564004A534F4E20EC
:1021E0006465746563746564004C6F6164696E67EF
:1021F00020436F6E6669672066726F6D204545509B
:10220000524F4D00436F6E666967206175746F733E
:102210006176653A000A5379736C6F672064656272
:102220007567206C6576656C3A0053657269616C00
:10223000206465627567206C6576656C3A00536151
:102240007665640A005365742064796E616D696314
:102250002049500A004F54412050617373776F72C8
:102260006420757064617465640A004E6F20495083
:102270002061647265737300205361766564004C5D
:102280006F6164696E67204854545020636F6E66B6
:102290006967206F6E20737461727475703A000004
:1022A0000000000000000000004F4E000000000091
:1022B0000000004F46460000000000000052455359
:1022C00054000000000000544F47474C45000000F8
:1022D0000048414C54000000000000584F4E0000E0
:1022E0000000000000584F46460000000000004972
:1022F0004E435245415345000044454352454153E6
:10230000450000454E41424C450000000044495301
:1023100041424C45000000554E465245455A450045
:1023200000465245455A45000000004155544F00B3
:10233000000000000046414E5F4F4E4C59000048DF
:102340004947480000000000004D454449554D00F4
:102350000000004C4F5700000000000000484541BD
:10236000545F434F4F4C004845415400000000006B
:1023700000434F4F4C000000000000445259000041
:10238000000000000052474200000000000000482A
:10239000535600000000000000636F756C64206EEF
:1023A0006F742070617273653A20005570646174B7
:1023B00065640A00454550524F4D20636C6561725B
:1023C00065640A004D5154542050617373776F72E5
:1023D0006420757064617465640A002B002D0045EB
:1023E0005461673A200047657420455441473A20BC
:1023F00000485454502F312E310025733A20257354
:102400000D0A0020485454502F312E310D0A486FC8
:1024100073743A2025730D0A4163636570743A2022
:102420002A2F2A0D0A436F6E6E656374696F6E3AC8
:1024300020636C6F73650D0A0025730020000D0A80
:1024400000474554006661696C656420746F2063C1
:102450006F6E6E6563740A004552524F523A2053B4
:1024600065727665722072657475726E656420009F
:10247000436F6E666967206E6F74206368616E6774
:1024800065640A00446F6E652E0A00436F6E6669CC
:10249000672070617273696E67206661696C65643C
:1024A0000A004765742061626F7274656400676F2B
:1024B0007420436F6E6669670A00687474702072D6
:1024C0006574636F64652000667265652000436F04
:1024D0006E666967205552493A20687474703A2FC5
:1024E0002F002044656661756C7420636F6E6669A9
:1024F000672073657276657220757365643A200093
:102500006C617A79686F6D652E7275000A282D29C5
:102510004352595054000A282D2950554C534520F8
:102520006F6E2050494E3132000A282D2943414E0A
:10253000000A282D294D455243555259000A282B8F
:10254000294D554C544956454E54000A282B2950C4
:10255000574D5F52454C4159000A282B294D444E96
:1025600053000A282D2955415254425249444745A7
:10257000000A282B295359534C4F47000A282B296E
:10258000504944000A282D294D4350323330313709
:10259000000A282D294152544E4554000A282D295D
:1025A0004F5441000A282B29535049204C454400E0
:1025B0000A282B294D4F544F5220435452000A28C9
:1025C0002B294143204841494552206F6E205365D5
:1025D0007269616C33000A282B2943435338313127
:1025E00020262048444331303830000A282B295215
:1025F0004553544152545F4C414E5F4F4E5F4D51D5
:1026000054545F4552524F5253000A282D294841D5
:10261000524452455345542C207573696E6720739C
:102620006F6674000A282B29434F554E54455200BB
:102630000A282B29444854000A282B2944533234B1
:1026400038322D313030000A282B294F5749524556
:10265000000A282D2949504D4F44425553000A285D
:102660002B294D4F44425553203078303620617429
:102670002053657269616C322073706565643A3904
:10268000363030000A282B294144414652554954DE
:10269000204C4544000A282B29444D58000A282B79
:1026A0002957697A6E657435313030000A282B2934
:1026B0004672656552616D207072696E74696E67ED
:1026C000000A282B295741544348444F47006C6166
:1026D0007A79686F6D652E7275000A436F6E666950
:1026E00067207365727665723A003230313130336B
:1026F0004C0020432B2B2076657273696F6E3A0075
:10270000343063316663615F323032362D30312DC3
:102710003130000A4C617A79686F6D652E727520D0
:102720004C6967687448756220636F6E74726F6C71
:102730006C65722000204F464600204F4E0020421C
:10274000595041535300536176656420746F20459E
:102750004550524F4D00536176696E6720636F6E2E
:1027600066696720746F20454550524F4D2E2E00EC
:102770004343533831313A20416C726561647920AA
:10278000696E697469616C697A65640043435338A2
:1027900031313A20496E6974206572726F7220007F
:1027A0004343533831313A20496E697400484443F9
:1027B000313038303A20416C726561647920696E3D
:1027C000697469616C697A656400446576696365FA
:1027D0002053657269616C204E756D6265723D00B3
:1027E000204465766963652049443D3078004D6139
:1027F0006E7566616374757265722049443D307808
:1028000000484443313038303A20496E69742E20F4
:1028100000432C2052483D00484443313038303A80
:10282000205374617475733D00484443313038302F
:102830003A204E6F7420696E697469616C697A65BB
:1028400064004D7367496E76616C6964005265611E
:1028500064526567496E76616C6964004D656173A9
:102860004D6F6465496E76616C6964004D617852A4
:102870006573697374616E63650048656174657240
:102880004661756C7400486561746572537570704B
:102890006C79004343533831313A204572726F727C
:1028A00020004343533831313A204661696C6564F6
:1028B00020746F20676574204552524F525F49441F
:1028C0002072656769737465722E005D20626173A2
:1028D000656C696E655B005D2074564F435B00203C
:1028E000434F325B006363733831313A2064617463
:1028F00061206E6F7420617661696C61626C650045
:10290000636373383131206E6F7420696E69746946
:10291000616C697A656400203C3C200041433A00C8
:10292000556E6B6E6F776E207375666669782000E2
:10293000556E6B6E6F776E20636D642000636C72F2
:102940004374723A2000444D58494E3A00454F4670
:10295000003D00494E3A002500C2B04320483D00EA
:1029600020444854323220747970652E20543D0042
:10297000494E3A00204E6F20656D69742064617481
:1029800061210020436F756E7465722074797065E3
:102990002E2076616C3D00494E3A0020436F756EE3
:1029A00074657220747970652E20494E434F5252DF
:1029B00045435420496E74657272757074206E754B
:1029C0006D626572212121004952513A00416374C0
:1029D000697661746520696E20004163746976616F
:1029E000746520696E20002D3E00200023002D3EDE
:1029F00000200050656E6465643A2023002D3E007F
:102A0000456D69743A002D3E00456D69743A002D9C
:102A10003E00456D69743A002D3E00456D69743A7B
:102A2000003D004C454741435920494E3A0020663D
:102A30006F7220286D73293A004354524C3A205348
:102A400063686564756C6520636D642000206D7338
:102A50000020666F7220004354524C3A2041726D40
:102A6000656420002044697361726D65640043549D
:102A7000524C3A20002074696D653A004354524C20
:102A80003A205265733A004354524C3A206D6F6DB0
:102A9000656E74617279206576656E74002054539A
:102AA0003A0020543A00544845524D3A00436C6570
:102AB000616E696E6720616C61726D20003D00502F
:102AC000696E3A004354524C3A20436F6D6D616E0B
:102AD0006420626C6F636B65642062792064726944
:102AE000766572004354524C3A204F4E3A416C7214
:102AF00065616479204163746976650A00435452C4
:102B00004C3A2048414C543A416C726561647920DA
:102B1000496E6163746976650A004354524C3A20E9
:102B2000584F4E3A2044697361626C65640A0043F1
:102B300054524C3A20584F4E3A416C726561647958
:102B4000204163746976650A004354524C3A205818
:102B50004F464620736B69707065642E2050726515
:102B60007620636D643A004354524C3A2054757297
:102B70006E6564206F66662066726F6D3A0043541E
:102B8000524C3A20526573746F7265642066726F9E
:102B90006D3A004354524C3A2049676E6F72656437
:102BA0002C206368616E6E656C20636D643D00204F
:102BB000457865633A004354524C3A204163746946
:102BC00076653A004354524C3A2048414C543A41BD
:102BD0006C726561647920496E6163746976650A17
:102BE000004354524C3A20584F4E3A204469736186
:102BF000626C65640A004354524C3A20584F4E3A76
:102C0000416C7265616479204163746976650A007C
:102C10004354524C3A20584F464620736B697070AB
:102C200065642E205072657620636D643A004354CB
:102C3000524C3A205475726E6564206F6666206649
:102C4000726F6D3A004354524C3A20526573746F60
:102C50007265642066726F6D3A0044697361726DCB
:102C6000696E67206E6F7420617574686F72697A1F
:102C70006564004354524C3A20636F6D6D616E641D
:102C8000206A75737420666F7220004354524C3A68
:102C9000204E6F7420656E6F756768206D656D6F6F
:102CA000727920666F722067726F7570206F706521
:102CB000726174696F6E00496E76616C696420613F
:102CC000726700496E76616C6964206172670049C1
:102CD0006E76616C696420617267004354524C3AAD
:102CE00020556E6B6E6F776E20737566666978001F
:102CF000536B697070696E67207363686564756C87
:102D000065642067726F7570206578656300435451
:102D1000524C3A206368616E6E656C2066726F7A01
:102D2000656E004354524C3A206368616E6E656C68
:102D30002066726F7A656E00536B697070656420EF
:102D4000686F6D6965207374756666002000205396
:102D500075623D00204974656D3D004354524C3A04
:102D60002052414D3D004354524C3A204F75744F10
:102D7000664D656D6F72793A2000282D2920002854
:102D80002B2920002076616C756520697320002056
:102D9000756E6B6E6F776E0A005D3D005B0020699B
:102DA0006E76616C69640020004143544956453A8F
:102DB00000206F6B003A00206661696C6564003A20
:102DC000005265747279696E6720564354454D50C0
:102DD00020434D440A005265747279696E6720562B
:102DE0004320434D440A005265747279696E67202E
:102DF0006D6F6462757320434D440A0052657472AE
:102E000079696E6720434D440A00206572726F72C3
:102E10003D004D423A20706F6C6C696E6720002057
:102E200056616C3A20004D423A20004D423A204E05
:102E30006F7420737570706F72746564207265674B
:102E400020747970650A004D423A20706F6C6C698D
:102E50006E672064696D6D657220004D423A2049AD
:102E60006C6C6567616C20617267756D656E7473FB
:102E70000A00206572726F723D004D423A20706FF9
:102E80006C6C696E6720504920002D004D423A203D
:102E900050492056616C203A004D423A20706F6CC8
:102EA0006C696E6720504920004D423A20706F6C6B
:102EB0006C696E6720464D206661756C7420002039
:102EC0006572726F723D004D423A20706F6C6C6992
:102ED0006E6720002D004D423A20464D2056616C11
:102EE000203A004D423A20706F6C6C696E67204644
:102EF0004D20004354524C2F706F6C6C3A204F752C
:102F0000744F664D656D6F72793A2000207365636A
:102F10002072656D61696E696E67005374617475C6
:102F2000732064656666657265640A002D3E005014
:102F300075623A20002D3E005075623A20002D3E09
:102F4000005075623A20000000000000636D6400CC
:102F500000736574000076616C000064656C0000AD
:102F60004853560000524742000066616E00006DF3
:102F70006F6465006374726C00687565000073614E
:102F800074000074656D700072617700002D3E0062
:102F90005075623A20002D3E005075623A20005371
:102FA000454E445354415455533A20556E6B6E6F01
:102FB000776E20636D64200A0000000000000000AE
:102FC0000000004F4E00000000000000004F464689
:102FD00000000000000000524553540000000000B3
:102FE00000544F47474C450000000048414C5400F6
:102FF0000000000000584F4E000000000000005884
:103000004F4646000000000000494E4352454153E0
:1030100045000044454352454153450000454E415B
:10302000424C450000000044495341424C450000D9
:1030300000554E465245455A450000465245455AB0
:1030400045000000004155544F00000000000046BC
:10305000414E5F4F4E4C5900004849474800000020
:103060000000004D454449554D000000004C4F57AD
:1030700000000000000000484541545F434F4F4CA2
:103080000048454154000000000000434F4F4C00F1
:1030900000000000004452590000000000000052EF
:1030A00047420000000000000048535600000000A6
:1030B000000000206661696C65643A004D6F6462CF
:1030C0007573206F7020004D423A206F6B003D00F9
:1030D0004D423A205643230020636D643D003D007D
:1030E0004D423A2056435F68656174230000002218
:1030F00000250028002B002E0031003400020100C2
:1031000000050108010B0100000A0B02090C0D0E5D
:103110000807030401000000000000000000000098
:10312000000000000000000000000000000000009F
:10313000000000121110000000000000000000005C
:10314000000000000000000000000000004D42559B
:10315000533A204164642040533A2000000021008B
:10316000240027002A002D00300033000101000058
:10317000040107010A010102102020080810204064
:10318000102040800201020108040201010204082B
:1031900010204080804020100804020180040201B9
:1031A0008040201008040201080402010102040802
:1031B000102040800102040810204080050505050C
:1031C000070508080808020202020A0A080804049F
:1031D00004040101010101010101030303030303CD
:1031E0000303040707070C0C0C0C0C0C0C0C02025C
:1031F000020206060606060606060B0B0B0B0B0B59
:103200000B0B556E73706563696669656420657242
:10321000726F722E0047454E455249435F455252E8
:103220004F5200494E5445524E414C5F4552524F09
:1032300052004932435F4552524F520049445F4564
:1032400052524F5200535543434553530043435347
:103250003831313A200057726F6E67207061796C97
:103260006164004D5154543A204354524C2F7478A9
:10327000743A204F75744F664D656D6F72793A20C0
:1032800000202D3E2041543A004368616E2074793D
:1032900070653A004E6F2073746F726564207661BA
:1032A0006C756573202D2064656661756C743A20B9
:1032B00000536176656420455441473A0053657474
:1032C00020455441473A20003157543A2042757303
:1032D000207265736574206572726F720031575485
:1032E0003A2042757320526573657420646F6E6571
:1032F000003157543A2044533234383220707265CA
:1033000073656E742C2072657365740049324320B6
:10331000526573657400005EBCE2613FDD83C29C50
:103320007E20A3FD1F419DC3217FFCA2401E5F01A3
:10333000E3BD3E6082DC237D9FC1421CFEA0E1BF55
:103340005D0380DE3C62BEE0025CDF81633D7C2287
:10335000C09E1D43A1FF4618FAA427799BC584DAB5
:103360003866E5BB5907DB856739BAE40658194763
:10337000A5FB7826C49A653BD987045AB8E6A7F915
:103380001B45C6987A24F8A6441A99C7257B3A6447
:1033900086D85B05E7B98CD2306EEDB3510F4E1075
:1033A000F2AC2F7193CD114FADF3702ECC92D38D23
:1033B0006F31B2EC0E50AFF1134DCE90722C6D33D5
:1033C000D18F0C52B0EE326C8ED0530DEFB1F0AE07
:1033D0004C1291CF2D73CA947628ABF51749085635
:1033E000B4EA6937D58B5709EBB536688AD495CBE3
:1033F0002977F4AA4816E9B7550B88D6346A2B7595
:1034000097C94A14F6A8742AC896154BA9F7B6E8C6
:103410000A54D7896B35436F6E6E65637465642E8D
:1034200000436F6E6E2E2061626F72746564003EA1
:103430003E2000496E76616C696420636F6D6D613A
:103440006E6400000020002300260029002C002FBD
:10345000003200000100000301060109013E3E3E6A
:10346000004E6F204D414320636F6E666967757231
:1034700065643A20736574206669726D7761726560
:103480002773204D41430A00454550524F4D20734C
:1034900069676E6174757265206F6B00496E69743F
:1034A00069616C697A696E6720454550524F4D2EAF
:1034B000002072656164206572726F7220666F729F
:1034C00020003E2000203C003157543A0031575430
:1034D0003A206E6F7420696E6974003157543A2037
:1034E000425553592074696D656F75740031575496
:1034F0003A204453323438325F4552524F525F4380
:103500004F4E464947003157543A20312D77697262
:10351000652073686F727465640072656164790018
:1035200024737461746500757074696D65006672EA
:10353000656568656170002473746174730020456B
:103540007870697265640A00202D74617267657411
:10355000207A6F6E652D0020416C61726D20457878
:1035600070697265640A0020636D643A00204375D7
:10357000723A00205365743A002054696D65723ABE
:1035800000204C6F636B733A0052414D3D00310196
:10359000E90211241FBECFEFD1E2DEBFCDBF00E0B4
:1035A0000CBF1AE0A0E0B2E0E6E5FAEC02E00BBFE7
:1035B00002C007900D92AC36B107D9F722E1ACE614
:1035C000BAE001C01D92AE3AB207E1F71AE1C8ECC9
:1035D000DAE100E006C021970109802FFE010F9477
:1035E000EF5CC73CD10780E00807A9F70F94D64BE2
:1035F0000D9419650C94000090E080E00895DC01C2
:10360000ED91FC910284F385E02D1994DF92EF9205
:10361000FF920F931F93CF93DF93EC010C891D89C9
:103620000115110559F01D8A1C8AC801DF91CF913F
:103630001F910F91FF90EF90DF900895EC85FD852D
:103640008E859F85DF01A80FB91F2C91243209F0C8
:1036500055C011962C912B3709F050C00296E80FF7
:10366000F91FF12CE12CDF01D190DD2009F446C0D7
:103670008DE7D816E9F08FEFE81AF80AF4CF198A27
:10368000188A2C853D852115310579F08E859F8519
:10369000280F391FF9012081222321F001969F87ED
:1036A0008E873EC01D861C86C0CF0FEF1FEFBDCF9B
:1036B000E114F10419F11C928E859F8502966C85A8
:1036C0007D85680F791FE881F9810684F785E02DF3
:1036D000CE011995998B888B1B8A1A8AEC85FD85FA
:1036E0008E859F85E80FF91FEE0DFF1DD2828E8516
:1036F0009F850396E80EF91EFF86EE862889398994
:103700002115310509F4BDCF8A899B89280F391FFE
:10371000F9012081222309F4B2CF01969B8B8A8B79
:10372000022F220F110B81CFDC011C96ED91FC9131
:103730001D971E968D919C91E80FF91F8081082E90
:10374000000C990B0895DC0115968D919C910097C2
:1037500039F0DC01ED91FC910680F781E02D1994A0
:103760000895FC01838594859C0144E03595279557
:103770004A95E1F756E0959587955A95E1F7281710
:10378000390719F081E090E0089582E090E0089513
:1037900083E090E00895DC011296ED91FC9113977F
:1037A0003097B9F016968D919C918430910541F037
:1037B0008530910541F0039749F482E090E0089547
:1037C00081E090E0089581E190E00895828590E0A5
:1037D000089590E080E0089585E090E008951F93BB
:1037E000CF93DF930097A1F0FC011085212F2F705C
:1037F000223071F4EC0161857285838594850F9484
:10380000355B69877A878B879C87107F1360188761
:10381000DF91CF911F9108958EE090E00895CF93AE
:10382000DF93FC01C681D78180858F70853079F068
:103830008630E1F42097D1F0E881F981309719F0D2
:1038400080818F7B79F40A80DB81C02DF3CF2097B4
:1038500069F0CE010E940F1C811105C00A80DB8136
:10386000C02DF5CF81E0DF91CF91089580E0FBCFAF
:1038700084E190E00895DC01ED91FC910484F585EC
:10388000E02D60E0199581E090E00895DC01149648
:10389000ED91FC9180E0309711F085A1817090E06E
:1038A0000895CF93DF93EC0165EF7AE088E290E131
:1038B0000F942A28EA81FB810280F381E02D608148
:1038C000718188E290E10F94142888E290E10F94CE
:1038D000BE26E881F9810484F585E02D60E0CE0103
:1038E000199581E090E0DF91CF9108950D949C535C
:1038F0000D949C530D949C530D949C530D949C5388
:10390000EF92FF920F931F93CF93DF938C0167EA9F
:103910007FE088E290E10F942A2888E290E10F94FA
:10392000BE26D8011496ED91FC91309749F1C681DD
:10393000D781209729F1E881F9813097E9F08081DA
:103940008823D1F065E675E0CE010E9470F17C011C
:10395000009791F0FC0181859285A385B48500973D
:10396000A105B10549F00F949C53D70119961D92FA
:103970001D921D921C921C970A80DB81C02DD9CF0D
:10398000D801ED91FC910484F585E02D60E0C8013B
:10399000199581E090E0DF91CF911F910F91FF90F9
:1039A000EF9008950D949C530D949C530D949C534B
:1039B0000D949C530D949C53EF92FF920F931F9381
:1039C000CF93DF93EC018B018091740A9091750A7B
:1039D0000097A9F0FC0120852F70263081F40E9409
:1039E00070F1FC0190859F70943049F48185928537
:1039F000DF91CF911F910F91FF90EF900895EE8886
:103A0000FF88C70101970D97D0F469E675E0C801FA
:103A10000F945C61892B99F48FE2888F85E08E9DED
:103A2000B0018F9D700D112460577C4E46E050E030
:103A3000CE0149960F947055CE014896D9CF90E0AB
:103A400080E0D6CF3F924F925F926F927F928F929B
:103A50009F92AF92BF92CF92DF92EF92FF920F931D
:103A60001F93CF93DF9300D000D0CDB7DEB77C019A
:103A7000362E8091710A882309F40CC1D70114965F
:103A80009C9180914402891708F404C18091D50A61
:103A90009091D60ABAE06B1316C28058954FFC017C
:103AA0001082D70118968D919C91892B09F4EEC054
:103AB00080917C0A90917D0AA0917E0AB0917F0A44
:103AC000892B8A2B8B2B09F0CDC00F94AD062B01CF
:103AD0003C01F70100851185D80119966D917C9103
:103AE0006115710599F4F80185809680A780B084EE
:103AF0008091680D9091690DA0916A0DB0916B0D48
:103B000088169906AA06BB0609F486C0D8011B963A
:103B10004D915C911C974115510509F47DC0F70149
:103B2000248153968C91539790E0322F377002C0C6
:103B3000959587953A95E2F780FF6EC0C22ED12CFD
:103B4000C601887F9370892B39F451968D919C9191
:103B5000887F9370C82AD92AD8018D919C91DC0165
:103B6000ED91FC916115710509F4C3C00688F789D0
:103B7000E02D1995019709F04FC06CE3F8018081A1
:103B800091810F947C274AE050E0B601D8018D91D5
:103B90009C910F94DB26F80122818081918162E45F
:103BA00073E1222311F060E473E10F942A28D80115
:103BB0001D966D917C911E978D919C910F94142868
:103BC00060E2F801808191810F947C27D8011F96D3
:103BD0006D917C9150978D919C910F941428F801D0
:103BE00022818081918165E373E1222311F06FE2EC
:103BF00073E10F942A2860E87AE0D8018D919C91B6
:103C00000F941428F80180819181DC01ED91FC91E1
:103C1000008CF18DE02D19950F94AD06AB01BC0120
:103C20004419550966097709F7018581968145365A
:103C300051056105710508F472C0009721F06FE726
:103C400073E10F944E284FEF5FEFBA0180E00F94BD
:103C5000674760937C0A70937D0A80937E0A9093F5
:103C60007F0A14C00F94AD0600917C0A10917D0A62
:103C700020917E0A30917F0A601B710B820B930B9F
:103C8000603375478105910508F01FCF1092D60A61
:103C90001092D50AD70115968D919C911697009791
:103CA00071F014963C9120914502231740F0DC01FD
:103CB000ED91FC910190F081E02D632D199581E04B
:103CC00090E026960FB6F894DEBF0FBECDBFDF9111
:103CD000CF911F910F91FF90EF90DF90CF90BF9009
:103CE000AF909F908F907F906F905F904F903F909C
:103CF00008950488F589E02D20E435E03A8329838E
:103D0000D80115968D909D90AD90BC9018978B82A0
:103D10009C82AD82BE82BE016F5F7F4F2ACF4091F1
:103D20007C0A50917D0A60917E0A70917F0A452B32
:103D3000462B472B09F4AACF009721F060E773E1E7
:103D40000F944E2810927C0A10927D0A10927E0ADF
:103D500010927F0AD70118960D911C91F801618588
:103D600072856115710591F4458056806780708475
:103D70008091680D9091690DA0916A0DB0916B0DC5
:103D8000481659066A067B0609F480CFD8011B96AF
:103D90004D915C911C974115510509F477CFF701BE
:103DA000248153968C91539790E0322F377002C044
:103DB000959587953A95E2F780FF68CFC22ED12C72
:103DC000C601887F9370892B39F451968D919C910F
:103DD000887F9370C82AD92AD8018D919C91DC01E3
:103DE000ED91FC916115710509F457C00688F789BA
:103DF000E02D1995019709F049CF6CE3F801808116
:103E000091810F947C274AE050E0B601D8018D9152
:103E10009C910F94DB26F8012281808191816BE5D2
:103E200073E1222311F069E573E10F942A28D80188
:103E30001D966D917C911E978D919C910F941428E5
:103E400060E2F801808191810F947C27D8011F9650
:103E50006D917C9150978D919C910F941428F8014D
:103E60002281808191816EE473E1222311F068E464
:103E700073E10F942A2861E673E1D8018D919C913A
:103E80000F942A28F80180819181DC01ED91FC9149
:103E9000008CF18DE02D1995F9CE0488F589E02D7F
:103EA00020E435E03A832983D80115964D905D9042
:103EB0006D907C9018974B825C826D827E82BE01F1
:103EC0006F5F7F4F96CF843591050CF0E3CEBDE058
:103ED0006B1709F4DFCE9C012F5F3F4F3093D60A5A
:103EE0002093D50A8058954FFC016083D3CE2F9242
:103EF0003F924F925F926F927F928F929F92AF927A
:103F0000BF92CF92DF92EF92FF920F931F93CF93C6
:103F1000DF93CDB7DEB7AA970FB6F894DEBF0FBE1A
:103F2000CDBF5C010E8F1F8F28A339A34AA35BA3CB
:103F30006CA37DA31C8A1B8ADC0118968D919C9131
:103F400001979E8B8D8BE114F104D1F0CE01459643
:103F50009F938F9302979F938F938DE695E09F9306
:103F60008F93FF92EF920F9411620FB6F894DEBF19
:103F70000FBECDBF019721F48B899C899E8B8D8BC1
:103F80006B897C894AE050E088E290E10F94CB276E
:103F90006DE273E188E290E10F942A286D897E89B1
:103FA0004AE050E088E290E10F94CB2767E273E1AA
:103FB00088E290E10F942A28FE8DFAA74AE050E0AB
:103FC0006F2F88E290E10F94E12688E290E10F9450
:103FD000BE2619861A861B861C861D861E861F868F
:103FE000188A8A85807F84608A87D50118968D918A
:103FF0009C912D893E89281739071CF001979E8BCB
:104000008D8B8B899C8997FF02C01C8A1B8A8B88A9
:104010009C885401312C212C8D899E898A159B0501
:104020000CF46AC1BAA5B13091F1B23009F453C1B0
:10403000EE24EA94FE2C0E8D1F8D28A139A14AA1F1
:104040005BA16CA17DA1CE0109960E943EA72983A8
:104050003A834B835C836D837E838F8398878091C3
:104060007A0A90917B0AFC0122813381A216B30661
:1040700008F088C06F852E8530E050E040E0542F76
:10408000432F322F2227462B6D85262B33C1E090FC
:104090007A0AF0907B0AF70182819381A816B9060B
:1040A00008F070C096855385018512854084A92F3C
:1040B000B0E06484712C658570E09401220D331D9D
:1040C000951372C0A901440F551F240F351F200FEF
:1040D000311FA20FB31F9C91F301E20FF31F108158
:1040E000260F371FD9010C91442009F452C0512CDE
:1040F000712C612C692F70E0762F6627072E000C3B
:10410000880B990BA30192010F94785CC901772762
:1041100066276EA37FA388A799A7612F70E0762FEB
:104120006627072E000C880B990BA30192010F94B0
:10413000785C542F432F322F22278EA19FA1A8A550
:10414000B9A5822B932BA42BB52B8EA39FA3A8A735
:10415000B9A7602F70E0762F6627072E000C880B1A
:10416000990BA30192010F94785C6EA17FA188A5A1
:1041700099A5262B372B482B592B232B242B252B6A
:1041800009F4A0C0FFEFAF1ABF0A2FEF221A320ABC
:1041900043CF212F30E050E040E0542F432F322F07
:1041A0002227492B202BE9CFC901880F991F880F9F
:1041B000991F800F911FA80FB91F3C91DC01A50F1B
:1041C000B11D0C91F301E80FF91FD080860F971FE6
:1041D000DC011C91442009F463C0512C712C612C2A
:1041E000632F70E0762F6627072E000C880B990B43
:1041F000A30192010F94785C922F88277727662776
:104200006EA37FA388A799A7602F70E0762F6627FB
:10421000072E000C880B990BA30192010F94785C78
:10422000A901332722278EA19FA1A8A5B9A5822B7A
:10423000932BA42BB52B8EA39FA3A8A7B9A7612F5F
:1042400070E0762F6627072E000C880B990BA301D0
:1042500092010F94785C6EA17FA188A599A5622B2D
:10426000732B842B952B6EA37FA388A799A76D2D05
:1042700070E0762F6627072E000C880B990BA301A0
:1042800092010F94785C542F432F322F22278EA156
:104290009FA1A8A5B9A5282B392B4A2B5B2B6DCF45
:1042A000802F90E0B0E0A0E0DC0199278827B32BB5
:1042B000AC01412B8A019D011D29012B022B032BEF
:1042C00009F060CF2FEF3FEF4FEF50E0B501C7018E
:1042D0000F941D2D57CF80917A0A90917B0ADC01B3
:1042E00012962D913C91A216B30608F04BCF20E018
:1042F00030E0A901B501ECCFCC2009F488C00091D1
:104300007A0A10917B0AD80119968D919C91892B7C
:1043100009F473C00F94A603F801C784D088E1881C
:10432000F2886C157D058E059F0520F46787708BDC
:10433000818B928BF801C784D088E188F2886C1950
:104340007D098E099F096C3271408105910510F33A
:10435000F894D80114968D919C9115979A8B898B1E
:104360001996ED91FC917F01BFEFEB1AFB0A80815A
:104370008D8FF80190810388F489E02DD80155963E
:104380008C91992309F45EC09081982B9C8F908129
:10439000809589238B8F8B8D888F88E08F8B5C8DA8
:1043A0006B8D4D8D3F89288D89899A89D7015083DE
:1043B00047FD252F3A952083262F39F0441F00C052
:1043C00000006083000000C0F2CF38E04D916083B0
:1043D0000000019761F7D8015496FC93EE93539730
:1043E0004D8F3F8B288F9A8B898B78940F94A603DF
:1043F000F8016787708B818B928B62E273E188E2B0
:1044000090E10F942A2888E290E10F94BE2681E083
:1044100090E0AA960FB6F894DEBF0FBECDBFDF9135
:10442000CF911F910F91FF90EF90DF90CF90BF90B1
:10443000AF909F908F907F906F905F904F903F9044
:104440002F9008959081982B9C8F9081809589233F
:104450008B8F8B8D8A8F88E0898F5C8D6B8D4D8DD6
:10446000398D2A8D89899A89D701508347FD252F57
:1044700000C000C0208300C000C000C000C000C059
:1044800060830000262F3A9541F0441F000000C0D1
:1044900000C000C000C000C0E8CF38E04D9100C0AF
:1044A000608300C0019709F7D8015496FC93EE93FE
:1044B00053974D8F398F2A8F96CFCF93DF93EC018F
:1044C00062E972E188E290E10F942A2866E872E1DD
:1044D00088E290E10F942A286C817D814AE050E0C7
:1044E00088E290E10F94CB2760E872E188E290E1E6
:1044F0000F942A2888E290E10F94BE2660E08C8118
:104500000F947602E881F9810484F585E02D60E05E
:10451000CE01199581E090E0DF91CF9108950F933E
:104520001F93CF93DF938C0163E775E088E290E1FE
:104530000F94C226C0917A0AD0917B0A4C815D818A
:1045400070E060E089859A850F94895A209771F010
:1045500089859A850F949C538E819F8197FD03C016
:1045600060E00F947602CE010F949C53D801ED9138
:10457000FC910484F585E02D60E0C801199581E087
:1045800090E0DF91CF911F910F910895CF93DF932A
:10459000EC0163E875E088E290E10F94C22640E008
:1045A00050E0BA018A819B810E94A6B2E881F9811C
:1045B0000484F585E02D60E0CE0119956D858C8130
:1045C0000F9448026D858D810F94480281E090E040
:1045D000DF91CF910895CF92EF92FF920F931F93A7
:1045E000CF93DF9300D000D01F921F92CDB7DEB7DC
:1045F0007C0109831A832B833C834D835E836F8305
:1046000078876CED7AE088E290E10F942A28CE0159
:1046100001960E947C7D898181112DC00B81013022
:1046200091F130F010E0023009F040C0CC2001F1EF
:1046300060E0CE0101960E944779F7010281138163
:10464000892B81F0C8010E94E7B2672B682B692B88
:1046500079F44FEF5FEFBA0180E00F946747AB0149
:10466000BC0103C040E050E0BA01C8010E94A6B2FC
:1046700081E090E02EC08031D0F58E30D8F58130C9
:10468000C9F18230D9F16FEC7AE088E290E10F94C1
:104690002A284AE050E0698188E290E10F94E126FF
:1046A00088E290E10F94BE2601E010E06FEB7AE023
:1046B00088E290E10F942A284AE050E0B80188E2AD
:1046C00090E10F94CB2788E290E10F94BE2690E012
:1046D00080E028960FB6F894DEBF0FBECDBFDF9105
:1046E000CF911F910F91FF90EF90CF90089583513C
:1046F000843048F6F70102811381A4CF40E050E0F6
:10470000BA01F70182819381B1CFFC01828193814B
:104710000E94E6BA21E030E0823011F430E020E07F
:10472000C90108950F931F93CF93DF938C01D0E0BD
:10473000C0E001151105B1F0BE01675E744FC801FC
:104740000F943955892B51F4FE01E35EF44F8491A7
:1047500090E0DF91CF911F910F9108952596C2337C
:10476000D10539F781E090E0F4CFFF920F931F93CA
:10477000CF93DF93CDB7DEB764970FB6F894DEBF63
:104780000FBECDBF8C01F62EDC0116966C91FF207A
:1047900011F081E06827F80184810F944802F80144
:1047A00087819085A185B285883E9340A105B1059A
:1047B00008F463C062ED72E188E290E10F942A2868
:1047C0006DEC72E188E290E10F942A28D8011496EA
:1047D0006D917C914AE050E088E290E10F94CB2704
:1047E00068EC72E188E290E10F942A286F2D70E066
:1047F0004AE050E088E290E10F94CB2788E290E114
:104800000F94BE268FE290E09C878B87FE013D9639
:1048100088E0DF011D928A95E9F761EC72E1CE0133
:104820000B960F942E55F801828193810E94E6BA6F
:10483000FF2079F169EB72E1853151F062EB72E1B1
:10484000863131F066EA72E18F3011F46EEA72E17E
:10485000CE0101960F944255D8011296ED91FC912C
:104860000280F381E02DAE01455F5F4FBE016F5FB7
:104870007F4F808191810F94680764960FB6F894FA
:10488000DEBF0FBECDBFDF91CF911F910F91FF9083
:10489000089562EA72E18230D9F26DE972E1D8CF0F
:1048A000AF92BF92CF92EF92FF920F931F93CF934D
:1048B000DF9300D000D01F921F92CDB7DEB75C010E
:1048C00009831A832B833C834D835E836F837887B0
:1048D00067E173E188E290E10F942A28CE01019606
:1048E0000E947C7DE114F10439F060E173E1C701BD
:1048F0000F943955009759F1F50102811381011583
:10490000110519F18981811165C08B81813009F40C
:1049100069C078F1823059F1082F10E06DEE72E134
:1049200088E290E10F942A286DED72E188E290E12F
:104930000F942A284AE050E0B80188E290E10F94F1
:10494000CB2788E290E10F94BE2690E080E0289685
:104950000FB6F894DEBF0FBECDBFDF91CF911F9190
:104960000F91FF90EF90CF90BF90AF900895CC2023
:10497000D9F060E0CE0101960E944779892B09F4B5
:1049800050C0C8010E94E7B2672B682B692BF9F46D
:104990004FEF5FEFBA0180E00F946747AB01BC01B6
:1049A000C8010E94A6B213C0C8010E94E6BA8E30A8
:1049B00019F050F4813059F460E0CE0101960E9464
:1049C0004779892B21F0DDCF83518430A8F381E032
:1049D00090E0BDCF803100F58E3098F6813089F2BD
:1049E0008230F9F065E073E188E290E10F942A28C3
:1049F00068EF72E188E290E10F942A284AE050E0E3
:104A0000698188E290E10F94E12688E290E10F94B9
:104A1000BE2601E010E082CF8351843008F4B1CF8C
:104A2000E1CF40E050E0BA01C8010E94A6B260E0C8
:104A3000C5010E94B523CBCF4F925F926F927F92B8
:104A40008F929F92AF92BF92CF92DF92FF920F937D
:104A50001F93CF93DF9300D000D01F921F92CDB74A
:104A6000DEB76130710509F482C0FC016281738197
:104A70006115710509F47BC08C0119821A821B82B1
:104A80001C821D821E821F8218868A81807F8A83F3
:104A900040E050E2CE0101960E94847860E0CE01B1
:104AA00001960E9447796C01F801828193810E94EE
:104AB000E7B22B013C01F801278130854185528501
:104AC000D6010F94C45C2FEF30E040E050E00F942B
:104AD000785C49015A010F94AD06FF24F3948114C8
:104AE0009104A104B10461F064197509860997095C
:104AF000FF24F394681579058A059B0508F4F12CC9
:104B0000411451046104710491F1F801878090848B
:104B1000A184B2840F94AD06F80181149104A1041C
:104B2000B10451F06419750986099709681579056A
:104B30008A059B0508F449C0A280B3804FEF5FEF60
:104B4000BA0180E00F946747AB01BC01C5010E9428
:104B5000A6B2CD2861F0F80184810F945047F80186
:104B60009681891304C061E0C8010E94B52390E0DA
:104B700080E028960FB6F894DEBF0FBECDBFDF9160
:104B8000CF911F910F91FF90DF90CF90BF90AF908A
:104B90009F908F907F906F905F904F900895FF202F
:104BA000D9F060E0C8010E94B523F80182819381A9
:104BB0000E94F3D1892BD9F640E050E0BA01F80108
:104BC000828193810E94A6B2D2CF84810F945047F4
:104BD000F80196818913E3CFCD2849F2F801848149
:104BE0000F945047F80196818913C1CFF110BFCFC0
:104BF000BACFAF92BF92CF92DF92EF92FF920F9314
:104C00001F93CF93DF93CDB7DEB768970FB6F894B5
:104C1000DEBF0FBECDBFFC01098B1A8B2B8B3C8BEB
:104C20004D8B5E8B6F8B788F82819381009709F417
:104C3000A1C024813581232B09F49CC0CC2009F428
:104C400099C06F0170E060E00E9473B3192FD60124
:104C5000ED91FC91008CF18DE02DC60119955C0160
:104C60008230910509F47AC0039709F445C095E0B4
:104C7000F1E0AF16B10409F091E019861A861B869F
:104C80001C861D861E861F86188A8A85807F892B32
:104C90008A87EE24EA94FE2C09891A892B893C899B
:104CA0004D895E896F89788DCE0109960E943EA755
:104CB000F1E0AF16B10409F453C082E0A816B104C4
:104CC00009F049C06F8570E0D60114968C910F945D
:104CD000B20261E070E0C6010E9409EB6E8570E0EF
:104CE0000F94B20262E070E0C6010E9409EB6D858C
:104CF00070E00F94B2022FC0612F661F6627661FF7
:104D0000CE0141960E9447795C01BC01D601149600
:104D10008C910F94B20265E672E188E290E10F9403
:104D20002A28F601648175814AE050E088E290E12A
:104D30000F94CB2763E672E188E290E10F942A2872
:104D40004AE050E0B50188E290E10F94CB2788E279
:104D500090E10F94BE2681E090E00EC094E08DCFEC
:104D600063E070E0C6010E9409EB688970E00F946F
:104D7000B202A8CF90E080E068960FB6F894DEBF4C
:104D80000FBECDBFDF91CF911F910F91FF90EF909C
:104D9000DF90CF90BF90AF900895CF93DF93EC0159
:104DA00069E572E188E290E10F942A286C817D81A7
:104DB0004AE050E088E290E10F94CB2767E572E18A
:104DC00088E290E10F942A28EA81FB810280F38136
:104DD000E02D6081718188E290E10F94142861E5F3
:104DE00072E188E290E10F942A2888E290E10F9422
:104DF000BE26E881F981008CF18DE02DCE01199558
:104E00008130910529F0029759F060E08C811AC039
:104E100063E070E0CE010E9409EB60E00F9476023F
:104E200060E08C810F94760261E070E0CE010E9418
:104E300009EB60E00F94760262E070E0CE010E9420
:104E400009EB60E00F947602E881F9810484F5852E
:104E5000E02D60E0CE01199581E090E0DF91CF91E7
:104E60000895CF92DF92FF920F931F93CF93DF931A
:104E700000D000D01F921F92CDB7DEB76C01F02E8C
:104E80001A83022F10E0FF2029F00115110511F4FB
:104E900001E010E040E050E061E070E0F601828166
:104EA00093810E947BB401301105A9F102301105F4
:104EB00041F0012BB1F563E67FE088E290E10F94C9
:104EC0002A288A818F70B9F1F60102811381C80105
:104ED0000E94E7B2672B682B692B89F401E010E090
:104EE000C80128960FB6F894DEBF0FBECDBFDF9184
:104EF000CF911F910F91FF90DF90CF9008954FEFCA
:104F00005FEFBA0180E00F946747AB01BC01C801B5
:104F10000E94A6B2E3CFF1E0FF1681F082E0F8161E
:104F200069F067E57FE088E290E10F942A2888E243
:104F300090E10F94BE2610E000E0D2CFF601C280CF
:104F4000D380C6010E94E7B2672B682B692B31F230
:104F50004FEF5FEFBA0180E00F946747AB01BC01F0
:104F6000C6010E94A6B2BCCFCF92DF92EF92FF9211
:104F70000F931F93CF93DC011296ED91FC9160E0AB
:104F8000848195810E9422F28C01009729F0FC0116
:104F900080858F708530D1F06DEA71E181E89FE006
:104FA0000F942A2881E89FE00F94BE26C12CD12CB3
:104FB00090E8E92E9FEBF92EC701B601CF911F9122
:104FC0000F91FF90EF90DF90CF900895C8010E945D
:104FD000B3F2813040F18630A8F1893020F565E0E8
:104FE000C8010E9422F2FC0190859F709330F9F471
:104FF000C184D284E384F484C1E060E0C8010E94EB
:1050000022F2FC0190859F70933009F561857285CD
:105010008385948520E030E0A9010F942E5B87FF03
:105020001FC0C111C9CFC12CD12C7601C5CF923080
:1050300049F461857285838594850F94355B6B0196
:105040007C01DACFC0E0C12CD12C7601D6CF9230D2
:1050500039F461857285838594850F94355BDACF49
:10506000C111AACFC12CD12C8FE7E82E83E4F82EF2
:10507000A3CFCF93DF93EC016BE771E188E290E17E
:105080000F942A28EA81FB810280F381E02D608160
:10509000718188E290E10F94C226EC81FD81309706
:1050A00021F0808191810F949C538C819D810F947C
:1050B0009C5370E060E08A819B810E9463B21D82F4
:1050C0001C8281E090E0DF91CF910895CF93DF9330
:1050D000EC0162E975E088E290E10F941428EA811E
:1050E000FB810280F381E02D6081718188E290E193
:1050F0000F94C2268C819D81009711F00F949C53D0
:1051000070E060E08A819B810E9463B21D821C82F4
:1051100081E090E0DF91CF910895CF93DF93FC0180
:1051200022813381232B59F1EC016BE679E088E28F
:1051300090E10F942A284AE050E06E8188E290E1E5
:105140000F94E12688E290E10F94BE268C819D8128
:105150000F949C5370E060E08A819B810E9463B24F
:105160001D821C82E881F9810484F585E02D60E0D0
:10517000CE01199581E090E0DF91CF91089590E004
:1051800080E0FACFCF92DF92EF92FF92CF93DF933E
:1051900069017A010F944F46EC01892BC9F088858B
:1051A000982F9F70923039F0933071F0911110C0A8
:1051B000807F82608887C701B6010F94005E69878F
:1051C0007A878B879C8704C0C986DA86EB86FC8643
:1051D000CE01DF91CF91FF90EF90DF90CF900895B7
:1051E000CF92DF92EF92FF920F931F93CF93DF93B3
:1051F000009701F1DC011896EC91EF70E630D1F4E4
:1052000069017A018B01EC010E9470F10097A1F411
:10521000A7019601B801CE010E9465FFB801CE0139
:10522000DF91CF911F910F91FF90EF90DF90CF9082
:105230000C9470F190E080E0DF91CF911F910F917D
:10524000FF90EF90DF90CF900895CF92DF92EF9292
:10525000FF920F931F93CF93DF93009701F1DC012F
:105260001896EC91EF70E630D1F469017A018B0168
:10527000EC010E9470F10097A1F4A7019601B8011A
:10528000CE010E9441FFB801CE01DF91CF911F9165
:105290000F91FF90EF90DF90CF900C9470F190E021
:1052A00080E0DF91CF911F910F91FF90EF90DF9001
:1052B000CF9008952F923F924F925F926F927F927C
:1052C0008F929F92AF92BF92EF92FF920F931F9394
:1052D000CF93DF93CDB7DEB72C970FB6F894DEBF30
:1052E0000FBECDBF6130710509F463C18C01FC01B3
:1052F000E280F38040E050E061E070E0C7010E948E
:10530000A4B4672B682B692B09F453C140E050E02B
:1053100062E070E0C7010E94A4B4672B682B692B80
:1053200089F480912702882309F443C140E050E0CA
:1053300062E070E0C7010E947BB480912702815037
:1053400080932702F801E280F380C7010E94E7B250
:105350004B015C0119821A821B821C821D821E82F3
:105360001F8218868A81807F8A8340E050E2B701DD
:10537000CE0101960E94847860E0CE0101960E94E1
:1053800047797C01F801828193810E94E6BA8230DC
:1053900011F0853011F4F12CE12CF80186819AECA2
:1053A000980F903108F0B7C121853285A90170E0CE
:1053B00060E049875A876B877C8743845484712CCB
:1053C000612C0F9489039C01990F440B550B2419F0
:1053D000350946095709AFEFB0E00F94B95C29854C
:1053E0003A854B855C8524193509460957090F9480
:1053F0009A5C390137FDB9C15FEF6516710411F090
:105400000CF0B6C181149104A104B10409F08BC160
:10541000E618F70856EFE5165FEFF5060CF0F6C054
:10542000F801658585810F944802F801A280B38058
:10543000C5010E94E7B2672B682B692B59F44FEF27
:105440005FEFBA0180E00F946747AB01BC01C50173
:105450000E94A6B2F801B48065858EEF8B0D8C306A
:1054600028F084ED8B0D833008F070C0AA27BB278D
:10547000AE19BF09662309F45CC09D01A1E0BFEF2E
:105480000F94FE5C29E130E040E050E00F949A5C1C
:10549000BA01A90141505F4F6F4F7F4F942F852F65
:1054A000692F782F6F3F710519F014F06FEF70E0DE
:1054B0006634710514F466E470E08B2D78C068E4FE
:1054C0007FE088E290E10F942A2888E290E10F942F
:1054D000BE2661EA75E088E290E10F94C226F801E9
:1054E000658584810F944802F801658585810F9454
:1054F000480240E050E0BA01F801828193810E94A5
:10550000A6B240E050E061E070E0F8018281938152
:105510000E9452B440E050E062E070E0F801828105
:1055200093810E9452B4809127028F5F809327025B
:1055300040C02FEF30E00F94065D29E130E040E0FD
:1055400050E00F949A5C922F832FAACF858191E02F
:1055500069279EEF980F9C3020F08C52833008F022
:10556000D6C08B2D0F944802AA27BB27AE19BF09BE
:10557000F80185858823B1F12FEF30E00F94065DA7
:1055800029E130E040E050E00F949A5C922F832FA5
:10559000692F782F6F3F710519F014F06FEF70E0ED
:1055A0006634710514F466E470E0F80185810F94A7
:1055B000B20290E080E02C960FB6F894DEBF0FBEEA
:1055C000CDBFDF91CF911F910F91FF90EF90BF90D2
:1055D000AF909F908F907F906F905F904F903F9093
:1055E0002F9008959D01A1E0BFEF0F94FE5C29E18B
:1055F00030E040E050E00F949A5CBA01A9014150BC
:105600005F4F6F4F7F4F942F852FC2CFFBE0EF1678
:10561000F1040CF45ECFF801658584810F94480293
:10562000F801A280B380C5010E94E7B2672B682B06
:10563000692B59F44FEF5FEFBA0180E00F94674791
:10564000AB01BC01C5010E94A6B2F801B580658519
:105650008EEF8B0D8C3020F084ED8B0D8330B0F409
:10566000662351F09701A1E0BFEF0F94FE5C23E3A6
:1056700030E040E050E00ACF2FEF30E0D7010F9448
:10568000065D23E330E040E050E05BCF848191E0B1
:1056900069279EEF980F9C3018F08C528330B8F534
:1056A0008B2D0F944802F80185858823E1F02FEFB8
:1056B00030E0D7010F94065D29E130E040E050E092
:1056C0000F949A5C922F832F692F782F77FF02C057
:1056D00070E060E06F3F710519F014F06FEF70E05B
:1056E000F801848164CF9701A1E0BFEF0F94FE5CC5
:1056F00029E130E040E050E00F949A5CBA01A90142
:1057000041505F4F6F4F7F4F942F852FDDCF8B2DF3
:105710000F9448024ECF66246A94762C811491042B
:10572000A104B104F1F0F80127803084032C000CAF
:10573000440855080F94AD06211431044104510466
:1057400009F4BDCE681979098A099B0962157305A8
:105750008405950508F0B3CEFFEF6F167F0609F0BC
:1057600057CE4FE7E41AF10855CE712C612C4ACE82
:1057700066246A94712C46CE8F929F92AF92BF920C
:10578000CF92DF92EF92FF920F931F93CF93DF930D
:10579000CDB7DEB760970FB6F894DEBF0FBECDBFB2
:1057A000E986FA860B871C872D873E874F87588BA3
:1057B0006115710511F0011103C090E080E0CCC0CB
:1057C0007B015C01DB018D909C9019821A821B8207
:1057D0001C821D821E821F8218868A81807F8A8396
:1057E0006FEA75E0C7010E9470F16C0164EB75E02F
:1057F000C7010E9470F17C01C114D10451F1F6017E
:1058000080858F70843029F5818592850E9492234E
:10581000182F8930B1F134F48130E4F4C12CD12C4B
:10582000760168C08A30D1F7B701CE0109960E948F
:10583000088129833A834B835C836D837E838F83C6
:1058400098873F7009F4B9CFCE0101960E94F07A93
:1058500015C011E0B701CE0109960E940881298385
:105860003A834B835C836D837E838F8398873F70FD
:1058700009F4A3CFCE0101960E94AC7A6B017C01A2
:1058800039C0B701CE0109960E94088129833A8365
:105890004B835C836D837E838F8398873F7009F48D
:1058A0008CCF31503B3008F0B9CFE32FF0E08827A0
:1058B000E35AF34D8F4F0D94EF5C712C712C0E2C2D
:1058C000682C682CCC2CBF2CBF2CBF2C682C682CCF
:1058D0002D813E814F815885AAE0B0E00F94B95CDC
:1058E000CDCFCD80FAE0CF9E600111240D2C000CAD
:1058F000EE08FF0880914502893020F4809144022F
:105900008930E8F066E17FE088E290E10F942A2890
:10591000B40188E290E10F9414286FE07FE088E200
:1059200090E10F942A282AE030E0B701A60188E22E
:1059300090E10F94832788E290E10F94BE26D50171
:105940001296ED91FC9162E0848195810E9422F291
:10595000009779F581E090E060960FB6F894DEBF8D
:105960000FBECDBFDF91CF911F910F91FF90EF90B0
:10597000DF90CF90BF90AF909F908F90089520E0E0
:1059800030E040E251E46D817E818F8198850F94F3
:10599000945B0F94005E72CF6D817E818F819885BC
:1059A0002AE030E040E050E00F949A5C69017A010F
:1059B000A1CFFC0120852F70263061F6B4010E9432
:1059C00070F15C01009731F2DC0118968C91189708
:1059D0008F709BEF980F923008F0BCCF4501853057
:1059E00029F416968C90169717969C90F501808551
:1059F0008068808768EB75E0C4010E9470F1FC014B
:105A0000892B61F0C186D286E386F486812F829548
:105A1000807F10851F70182B10879CCF66E07FE079
:105A200088E290E10F942A28D5016D917C9188E25B
:105A300090E10F94142888E290E10F94BE26A7010C
:105A4000960168EB75E0C4010E9441FF68EB75E0C8
:105A5000C4010E9470F1FC01892B09F47BCF1295DF
:105A6000107F90859F70192BD7CF2F923F924F9226
:105A70005F927F928F929F92AF92BF92CF92DF926E
:105A8000EF92FF920F931F93CF93DF9300D000D03C
:105A90001F921F92CDB7DEB709831A832B833C83F5
:105AA0004D835E836F837887DC011496ED91FC91C2
:105AB0000FEF1FEF3097F9F057014C01C288D388E0
:105AC000E114F10489F1F7018081882369F1C1149F
:105AD000D10489F1B701C6010E9470F1E980FA8012
:105AE0000B811C812D813E814F815885BC01C401F1
:105AF0000E94BC2B8C01C80128960FB6F894DEBF1B
:105B00000FBECDBFDF91CF911F910F91FF90EF900E
:105B1000DF90CF90BF90AF909F908F907F905F90DD
:105B20004F903F902F900895C114D10421F0D601D9
:105B30001696CD90DC907B80F12C0FEF1FEF272C79
:105B4000312C512C412CC114D10449F166E675E089
:105B5000C6010E9470F10097E9F0FC0120852F70CA
:105B60002230C1F481859285A385B4858215930581
:105B7000A405B50579F4E980FA800B811C812D819B
:105B80003E814F815885B601C4010E94BC2B8C0117
:105B9000FF24F394D6011296CD90DC90D4CFF1106F
:105BA000AACF61E37FE081E89FE00F942A28B50146
:105BB00081E89FE00F94142865E27FE081E89FE090
:105BC0000F942A28672D70E04AE050E081E89FE0BA
:105BD0000F94CB2781E89FE00F94BE268CCF1F93B4
:105BE000CF93DF9300D000D0CDB7DEB76130710521
:105BF00009F46BC05CF4672B09F45DC064EB7CE0D6
:105C000088E290E10F942A2880E04BC06230710551
:105C100071F06330710591F79093CC0D8093CB0DAB
:105C200055275093CE0D4093CD0D84E009C090933D
:105C3000CC0D8093CB0D5093CE0D4093CD0D83E0D2
:105C40000F943C08182F4FEF5FEFBA0180E00F94DC
:105C500067476093760A7093770A8093780A9093E7
:105C6000790A1123D9F06FE97CE081E89FE00F9475
:105C70002A28812F90E0B0E0A0E089839A83AB834B
:105C8000BC8380E190E09E838D83BE016F5F7F4F78
:105C900081E89FE00E941ABC0F94BE2681E011119A
:105CA000B3CF26960FB6F894DEBF0FBECDBFDF91FF
:105CB000CF911F9108959093CC0D8093CB0D50936D
:105CC000CE0D4093CD0D81E0BBCF9093CC0D809352
:105CD000CB0D5093CE0D4093CD0D82E0B1CFCF933D
:105CE000DF93EC01EC81FD8140815181052E000C98
:105CF000660B770B228189EC9CE00F94772970E08A
:105D000060E08A819B810E9473B3E7ECFDE08283AF
:105D100089EC9CE0918380831092D70E1092D90E6B
:105D20001092D80EDF91CF910895CF93DF93611534
:105D3000710589F0EB01DC011296ED91FC9162E0B6
:105D4000848195810E9422F2BE010E9470F1DF9150
:105D5000CF910D94850190E080E0DF91CF9108957F
:105D60004F925F926F927F928F929F92AF92BF926B
:105D7000CF92DF92EF92FF920F931F93CF93DF9317
:105D8000CDB7DEB768970FB6F894DEBF0FBECDBFB4
:105D9000098B1A8B2B8B3C8B4D8B5E8B6F8B788F8B
:105DA000DC0112962D913C911397232B09F4DEC050
:105DB000CC2009F4DBC06C01ED91FC91008CF18DDD
:105DC000E02D19955C016EE07BE088E290E10F9494
:105DD0002A28CE0141960E947C7DA114B10471F461
:105DE00060E0CE0141960E944779682FF6018481D8
:105DF00095810F942A4181E090E0BAC0CE0141968E
:105E00000E943B7B4C0194E0F2E0AF16B10459F0E4
:105E100081E1A816B10409F445C091E0A1E0AA16F9
:105E2000B10409F495E019861A861B861C861D8626
:105E30001E861F86188A8A85807F892B8A87EE2492
:105E4000EA94FE2C09891A892B893C894D895E893F
:105E50006F89788DCE0109960E943EA764E07BE0B1
:105E600088E290E10F942A28CE0109960E947C7D59
:105E7000B2E0AB16B10489F0E1E1AE16B104B1F0C5
:105E8000AA94AB2809F0B7CF188963E070E0C60187
:105E90000E9409EB612F0F942A416F85F6018481DE
:105EA000958151C0888D8170888FBCCF0FE710E03D
:105EB0008FEF88169806A9F0092C000CAA08BB08D9
:105EC000A50194012959310941095109AFEFB0E009
:105ED0000F94B95C2BE531E040E050E00F949A5C00
:105EE000890163E070E0C6010E9409EB5C0128892A
:105EF00030E0D8010F94065D412C512C32014A94B8
:105F0000A30192010F949A5C622FC5010F942A415C
:105F100064E070E0C6010E9409EB5C01AFEFB0E005
:105F2000A01BB10B288930E00F94065DA3019201FC
:105F30000F949A5C622FC5010F942A416F85D60198
:105F400014968D919C910F942A411E8561E070E01A
:105F5000C6010E9409EB612F0F942A411D8562E062
:105F600070E0C6010E9409EB612F43CF90E080E012
:105F700068960FB6F894DEBF0FBECDBFDF91CF910C
:105F80001F910F91FF90EF90DF90CF90BF90AF9057
:105F90009F908F907F906F905F904F9008958F9219
:105FA0009F92AF92BF92CF92DF92EF92FF920F93A8
:105FB0001F93CF93DF9300D000D01F921F92CDB7D5
:105FC000DEB76D7F6130710509F4BDC0FC01E28070
:105FD000F380E114F10409F4B6C08C01C7010E94FA
:105FE000E7B24B015C0161E070E0C7010E942DB394
:105FF00081149104A104B10409F4A5C020E030E0AB
:106000004AE754E40F94945B0F94075E6B017C01A4
:10601000C114D104E104F10409F495C00F94AD0654
:10602000681979098A099B096C157D058E059F05FC
:1060300008F489C0F801A280B38070E060E0C50177
:106040000E942DB320E030E048EC52E40F94945BC2
:106050000F94075E6B017C014FEF5FEFBA0180E0A8
:106060000F946747AB01BC01C5010E94A6B219821B
:106070001A821B821C821D821E821F8218868A81C0
:10608000807F8A83F8016281738140E050E3CE0112
:1060900001960E948478CE0101960E94F07A4B010D
:1060A0005C016BEB75E088E290E10F9414282AE024
:1060B00030E0B501A40188E290E10F94D9266AECA2
:1060C00075E088E290E10F9414282AE030E0B701EF
:1060D000A60188E290E10F94D92688E290E10F941E
:1060E000BE26C80CD91CEA1CFB1C8A81807F8660F6
:1060F0008A83CD82DE82EF82F886F8016281738125
:1061000040E050E2CE0101960E9471776EEC75E09E
:1061100088E290E10F9414282AE030E0B701A6014C
:1061200088E290E10F94D92688E290E10F94BE2690
:1061300030E020E040E050E260E070E0F801828171
:1061400093810E942BB890E080E028960FB6F894D7
:10615000DEBF0FBECDBFDF91CF911F910F91FF909A
:10616000EF90DF90CF90BF90AF909F908F90089569
:10617000CF92DF92EF92FF920F931F93CF93DF9313
:10618000CDB7DEB762970FB6F894DEBF0FBECDBFB6
:106190006C010B871C872D873E874F87588B698B37
:1061A0007A8B6AEB7AE0C7010F943955EEE0F0E0A4
:1061B000892BF1F064EB7AE0C7010F943955E0E1E7
:1061C000F0E0892BA9F06EEA7AE0C7010F94395507
:1061D000EFE0F0E0892B61F01D856AEA7AE0C70103
:1061E0000F943955E12FF0E0892B11F4EDE0F0E048
:1061F0009B85992341F0309731F4EF2809F45CC076
:106200008FEF9FEFCAC0E131F10508F037C0882752
:10621000E35FFE4C8F4F0D94EF5C00315C311E311B
:106220003E313E313E313E310E32C5323E313E319D
:106230003E313E313E31CF320833DD32CE010B9656
:106240000E94AC7A20EF260F2931D0F6D6011496A1
:10625000ED91FC91159723A39B01AC0133274427B3
:1062600055271296ED91FC910280F381E02D60811B
:10627000718103EE15E0C6010E9473EBD6011496FE
:10628000ED91FC911597118A1496ED91FC9115975B
:1062900081E081871496ED91FC9115978DE48287BA
:1062A0001496ED91FC9115978FE5838714966D9167
:1062B0007C9145E250E04CC0F601048115814FEF1E
:1062C0005FEFBA0180E00F946747D80198966D930D
:1062D0007D938D939C939B97D601ED91FC910484C3
:1062E000F585E02D64E0C6011995EB85E150E631B6
:1062F00028F6F0E0D60114962D913C911597882749
:10630000EB57FE4C8F4F0D94EF5C9B31AC313E311F
:106310003E31AC319B313E313E313E313E313E313A
:106320003E313E31DC31F4313E313E313E313E31A1
:10633000F031EC31F231F90185A1858F1496ED91A0
:10634000FC91858D8160858F4DE050E06AE172E0BF
:10635000C6010E94B6721FC0F90185A1858F1496EF
:10636000ED91FC91858D8E7F858F4DE050E06DE045
:1063700072E0C6010E94B672D6011296ED91FC91B0
:106380000280F381E02D48EE55E06CEF76E08081ED
:1063900091810F94680781E090E062960FB6F894BF
:1063A000DEBF0FBECDBFDF91CF911F910F91FF9048
:1063B000EF90DF90CF900895F901178AD6011496D7
:1063C000ED91FC91159785A1858F1496ED91FC9127
:1063D000858D8160858F52CF81E0F901878BEECF6B
:1063E00082E0FBCF84E0F9CF83E0F901878B14963C
:1063F000ED91FC91159785A1858F1496ED91FC91F7
:106400001597858D8160858F1496ED91FC91818D16
:10641000833009F033CF82E0818F30CF1982F601CB
:10642000048115819031C1F190F4923009F440C09B
:106430009E30B9F0CE010B960E94AC7A61157105C1
:106440008105910509F058C0F80117A243C09131A8
:1064500041F1923179F782E0F801818F64E67AE0C8
:1064600006C083E0D80159968C936CE37AE0CE01A4
:1064700001960F944255D6011296ED91FC9102803F
:10648000F381E02D4DEE55E0BE016F5F7F4F8081BF
:1064900091810F946807F2CEF801118E60E57AE0E1
:1064A000E6CF81E0D80159968C936AE57AE0DFCF98
:1064B000D80197961C92048115814FEF5FEFBA01C6
:1064C00080E00F946747D80198966D937D938D93E4
:1064D0009C939B97D6011496ED91FC91159785A1FD
:1064E000858F1496ED91FC91858D8E7F858F4DE083
:1064F00050E06DE072E02CCFD80197961C9261506D
:10650000710981099109660F771F881F991F2EEF66
:1065100030E040E050E00F949A5CDA01C901019646
:10652000A11DB11D813071F0A8F2823029F18330B4
:1065300009F0A1CFD6011496ED91FC91118E60E582
:106540007AE008C0D6011496ED91FC9182E0818F2B
:1065500064E67AE0CE0101960F944255D601149676
:10656000ED91FC91159785A1858F1496ED91FC9185
:10657000858D8160858F7FCFD6011496ED91FC913A
:1065800081E0818F6AE57AE0E5CFCE010B960E942B
:10659000AC7AD6011496ED91FC91678B6FCED60143
:1065A0001496ED91FC91913029F0923009F066CE6D
:1065B000148E64CE80E5848F61CEF601048115814E
:1065C000913049F09230B1F0CE010B960E94AC7A36
:1065D000F801638F53CE83E0D8015B968C930280E1
:1065E000F381E02D0280F381E02D42EF55E06BEE68
:1065F00076E04DCFF801138ED6011296ED91FC9105
:106600000280F381E02D42EF55E06CEF76E03FCF62
:10661000D6011496ED91FC91913031F0923009F051
:106620002DCE858D877FD6CE858D8860D3CE3F9247
:106630004F925F926F927F928F929F92AF92BF9292
:10664000CF92DF92EF92FF920F931F93CF93DF933E
:10665000CDB7DEB7C75AD1090FB6F894DEBF0FBE6B
:10666000CDBFDC0114962D913C911597232B09F495
:10667000D2C58B016C01ED91FC910284F385E02D74
:1066800019958230910509F418C1C4F597FFC3C567
:10669000F60187819085DC01ED91FC910084F18504
:1066A000E02D199585970CF4F4C045E250E0BE0149
:1066B0006F5F7F4FF601878190850F944026D6014A
:1066C00017968D919C91DC01ED91FC910084F185F0
:1066D000E02D1995892B09F437C162E070E080E064
:1066E00090E00F94BB04F60187819085DC01ED9169
:1066F000FC910284F385E02D1995E1CF843091055A
:1067000009F474C0C4F1059719F60130110509F0B8
:1067100000C169E979E088E290E10F944E284DE0EC
:1067200050E060E072E0C6010E94B672F60104819A
:1067300015814FEF5FEFBA0180E00F946747D801F2
:1067400098966D937D938D939C939B97D601ED9135
:10675000FC910484F585E02D62E0C6011995D6010F
:106760001496ED91FC9115978FEF80831496ED911F
:10677000FC9181838DCFD6011496ED91FC9180A57B
:1067800091A5A2A5B3A5892B8A2B8B2B09F480CFC9
:106790000F94AD06D6011496ED91FC91159700A5C6
:1067A00011A522A533A5601B710B820B930B6639D3
:1067B00071058105910508F46BCFED91FC9104847E
:1067C000F585E02D62E0C6011995F6010481158179
:1067D0004FEF5FEFBA0180E00F946747D8019896BA
:1067E0006D937D938D939C939B9752CFD601149676
:1067F000ED91FC9180A591A5A2A5B3A5892B8A2B2B
:106800008B2BD9F10F94AD06D6011496ED91FC9126
:1068100000A511A522A533A5601B710B820B930B5C
:10682000683873418105910540F1D601ED91FC91E5
:106830000484F585E02D65E0C6011995F601048113
:1068400015814FEF5FEFBA0180E00F946747D801E1
:1068500098966D937D938D939C939B97D6011496F8
:10686000ED91FC9117A265EA79E088E290E10F943E
:106870002A2888E290E10F94BE26F6018781908550
:10688000DC01ED91FC910084F185E02D1995892BB7
:1068900019F481E090E03FC062E070E080E090E0B9
:1068A0000F94BB04F60187819085DC01ED91FC918A
:1068B0000284F385E02D1995E0CFD6011496ED9171
:1068C000FC9180A591A5A2A5B3A5892B8A2B8B2B22
:1068D000E1F00F94AD06D6011496ED91FC9140A421
:1068E00051A462A473A464197509860997096838CC
:1068F00073418105910548F0D601ED91FC91048426
:10690000F585E02D65E0C60119950130110509F402
:10691000BFCE90E080E0C955DF4F0FB6F894DEBFE0
:106920000FBECDBFDF91CF911F910F91FF90EF90E0
:10693000DF90CF90BF90AF909F908F907F906F909F
:106940005F904F903F90089565E979E088E290E18B
:106950000F942A284AE050E0F601668188E290E12F
:106960000F94E12660E979E088E290E10F942A280B
:106970008E010F5F1F4F7E01F5E2EF0EF11CD80173
:106980006D918D0140E150E06A3058F469EF75E097
:1069900088E290E10F94142840E150E0F80131972B
:1069A000608188E290E10F94E126E016F10639F764
:1069B0006EE288E290E10F947C2788E290E10F94E8
:1069C000BE26FE01339680E00E171F0719F0919145
:1069D000890FFACF9DA1981313C469E879E088E282
:1069E00090E10F942A2888E290E10F94BE268DA1B1
:1069F000D6011496ED91FC91159797A1891709F48A
:106A000048CF87A314960D90BC91A02D85E2FE017E
:106A1000319601900D928A95E1F7D6011496ED9189
:106A2000FC91C056DF4F188219821A821B82C05A0D
:106A3000D040CC55DF4F188219821A821B82C45A6B
:106A4000D040CF55DF4F8881C15AD040807FCF558D
:106A5000DF4F8883C15AD04083A190E04C01B0E160
:106A60008B0E911C499708F014CF3584878986A333
:106A7000118D738CD60114962D913C91858DD90181
:106A800095968C93E48CF12C878DD6011296ED911E
:106A9000FC910280F381E02D4BEF55E06BEE76E048
:106AA00080FD02C06CEF76E0808191810F946807D1
:106AB000B0E8EB16F10409F086C0D6011296ED910C
:106AC000FC910280F381E02D42E056E06BEE76E02F
:106AD000808191810F94680768E076E088E290E118
:106AE0000F941428D6011496ED91FC914AE050E0E1
:106AF00065A188E290E10F94E12688E290E10F948D
:106B0000BE26D6011496ED91FC91159785A112969B
:106B1000ED91FC910280F381E02D43E156E06BEEB4
:106B200076E083FD02C06CEF76E0808191810F9466
:106B30006807D6011296ED91FC9113970280F381BC
:106B4000E02D808191811496ED91FC9125A14AE17F
:106B500056E06BEE76E021FD02C06CEF76E00F941C
:106B600068071EA2113009F4F8C1E0F1123009F4EF
:106B700029C2133009F45BC269E779E0CE01869639
:106B80000F94425560E0CE0180569F4F0E943978A5
:106B9000E9962FAFE997EA963FAFEA97EB964FAFAA
:106BA000EB97EC965FAFEC97ED966FAFED97EE96A7
:106BB0007FAFEE97EF968FAFEF97C158DF4F988377
:106BC000CF57D04043C0EF2809F086CFD6011296A8
:106BD000ED91FC910280F381E02D42E056E06CEFF4
:106BE00076E076CF60E57AE0CE0186960F94425546
:106BF00060E1CE0180569F4F0E943978C856DF4F22
:106C00002883C859D040C756DF4F3883C959D04070
:106C1000C656DF4F4883CA59D040C556DF4F588308
:106C2000CB59D040C456DF4F6883CC59D040C356AF
:106C3000DF4F7883CD59D040C256DF4F8883CE597D
:106C4000D040C156DF4F9883CF59D040D60112961D
:106C5000ED91FC910280F381E02D4DEE55E0BE01F7
:106C60006A5D7F4F808191810F946807C056DF4F26
:106C7000E880C05AD040CF55DF4FF880C15AD0408D
:106C8000CE55DF4F0881C25AD040CD55DF4F188115
:106C9000C35AD040CC55DF4F2881C45AD040CB5581
:106CA000DF4F3881C55AD040CA55DF4F4881C65A98
:106CB000D040C955DF4F5881C75AD0406EEE75E0BD
:106CC000C6010E947173D6011296ED91FC9102806B
:106CD000F381E02D42EF55E06CEF76E0772011F084
:106CE0006BEE76E0808191810F946807092C000C8F
:106CF000AA08BB08D6011296ED91FC910280F3819F
:106D0000E02D6081718103EE15E0A5019401C601BB
:106D10000E9473EB432C512C712C612CBFEF3B165E
:106D200081F0D6011296ED91FC910280F381E02D65
:106D30006081718106E216E0A3019201C6010E9402
:106D400073EB18AA19AA1AAA1BAA1CAA1DAA1EAA82
:106D50001FAA89A9807F89ABB501A401CE01C09685
:106D60000E945B78E1962FAFE197E2963FAFE29702
:106D7000E3964FAFE397E4965FAFE497E5966FAF86
:106D8000E597E6967FAFE697E7968FAFE797E896A9
:106D90009FAFE89779018A019B01AC0164EE75E031
:106DA000C6010E94717318AA19AA1AAA1BAA1CAAC2
:106DB0001DAA1EAA1FAA89A9807F89ABB301A201BF
:106DC000CE01C0960E945B7828AF39AF4AAF5BAF67
:106DD0006CAF7DAF8EAF9FAF63E0CE01C8960E94CF
:106DE0001778A9962FAFA997AA963FAFAA97AB9607
:106DF0004FAFAB97AC965FAFAC97AD966FAFAD971B
:106E0000AE967FAFAE97AF968FAFAF97E0969FAF3E
:106E1000E09779018A019B01AC0167E276E0C60147
:106E20000E9471731EA2D6011496ED91FC9186A169
:106E3000811132C16CE37AE0CE0186960F944255FF
:106E40006EE0CE0180569F4F0E943978A1962FAFF9
:106E5000A197A2963FAFA297A3964FAFA397A496F0
:106E60005FAFA497A5966FAFA597A6967FAFA6979D
:106E7000A7968FAFA797A8969FAFA897D60114960D
:106E8000ED91FC91159726A130E050E040E012967C
:106E9000ED91FC910280F381E02D608171810CE223
:106EA00016E0C6010E9473EBD6011496ED91FC9199
:106EB00085A180FD14C064EC79E0CE0186960F9424
:106EC000425562E0CE0180569F4F0E94397828AB30
:106ED00039AB4AAB5BAB6CAB7DAB8EAB9FABD6013A
:106EE0001296ED91FC910280F381E02D48EE55E081
:106EF000BE016A5D7F4F808191810F946807C05603
:106F0000DF4FE880C05AD040CF55DF4FF880C15ADC
:106F1000D040CE55DF4F0881C25AD040CD55DF4F0B
:106F20001881C35AD040CC55DF4F2881C45AD04075
:106F3000CB55DF4F3881C55AD040CA55DF4F488105
:106F4000C65AD040C955DF4F5881C75AD04069EE64
:106F500075E0C6010E9471739CCC6AE57AE0CE01AF
:106F600086960F94425561E1CE0180569F4F0E9454
:106F70003978C057DF4F2883C059D040CF56DF4FF4
:106F80003883C159D040CE56DF4F4883C259D040D4
:106F9000CD56DF4F5883C359D040CC56DF4F68835E
:106FA000C459D040CB56DF4F7883C559D040CA561C
:106FB000DF4F8883C659D040C956DF4F9883C759E1
:106FC000D04044CE64E67AE0CE0186960F944255D6
:106FD00062E1CE0180569F4F0E943978C857DF4F3B
:106FE0002883C858D040C757DF4F3883C958D0408E
:106FF000C657DF4F4883CA58D040C557DF4F588324
:10700000CB58D040C457DF4F6883CC58D040C357CB
:10701000DF4F7883CD58D040C257DF4F8883CE589A
:10702000D040C157DF4F9883CF58D0400FCE6CE38C
:107030007AE0CE0186960F9442556EE0CE018056DE
:107040009F4F0E943978C058DF4F2883C058D040E6
:10705000CF57DF4F3883C158D040CE57DF4F4883DA
:10706000C258D040CD57DF4F5883C358D040CC577B
:10707000DF4F6883C458D040CB57DF4F7883C55863
:10708000D040CA57DF4F8883C658D040C957DF4F1A
:107090009883C758D040DACD813029F562E87AE08C
:1070A000CE0186960F94425565E1CE0180569F4FE2
:1070B0000E94397869962FAF69976A963FAF6A97B1
:1070C0006B964FAF6B976C965FAF6C976D966FAF8B
:1070D0006D976E967FAF6E976F968FAF6F97A096F6
:1070E0009FAFA097CBCE823029F568E77AE0CE013A
:1070F00086960F94425564E1CE0180569F4F0E94C0
:10710000397861962FAF619762963FAF6297639629
:107110004FAF639764965FAF649765966FAF65975F
:1071200066967FAF669767968FAF679768969FAFB3
:107130006897A4CE833029F566E47AE0CE0186967E
:107140000F9442556FE0CE0180569F4F0E943978D0
:1071500029962FAF29972A963FAF2A972B964FAFA4
:107160002B972C965FAF2C972D966FAF2D972E9661
:107170007FAF2E972F968FAF2F9760969FAF609718
:107180007DCE843029F56CE87AE0CE0186960F94A6
:10719000425566E1CE0180569F4F0E943978219674
:1071A0002FAF219722963FAF229723964FAF239779
:1071B00024965FAF249725966FAF259726967FAFCD
:1071C000269727968FAF279728969FAF289756CE5A
:1071D0008D3609F053CE69E779E0CE0186960F949B
:1071E000425560E0CE0180569F4F0E94397828AF0B
:1071F00039AF4AAF5BAF6CAF7DAF8EAF9FAF3ECEC6
:107200006DE779E088E290E10F942A2888E290E126
:107210000F94BE263ECB8FEF9FEF7DCB8F929F9238
:10722000AF92BF92CF92DF92EF92FF920F931F9394
:10723000CF93DF937C014A015901C091740AD09128
:10724000750A062F660F110B209709F45CC088851C
:107250008F70863009F055C062E376E0CE010E945F
:1072600070F16C0182E08816910449F067E376E0E2
:10727000E3E08E16910429F0D0E0C0E006C06BE395
:1072800076E0CE010E9470F1EC01C114D104D9F175
:10729000F60180858F708430B1F561857285A80113
:1072A000C7010F948A61A8016EEF78E0C7010F94BF
:1072B0006C61209779F188858F70843059F56985E4
:1072C0007A85A801C7010F946C61A8016EEF78E080
:1072D000C7010F946C61A114B10429F0A801B50194
:1072E000C7010F946C61C701DF91CF911F910F917E
:1072F000FF90EF90DF90CF90BF90AF909F908F90D6
:107300000895D0E0C0E0A80163EE73E1C7010F94D7
:107310007055C9CFF2E08F16910481F083E0881692
:10732000910429F06091720A7091730ACACFA80182
:107330006DED73E1C7010F945255C7CFA8016AEDF7
:1073400073E1F8CFAF92BF92CF92DF92EF92FF92AC
:107350001F93CF93DF9300D000D0CDB7DEB76C0181
:107360007C0110E08AE0A82EB12C133061F1F70106
:10737000828190E0B0E0A0E089839A83AB83BC83F4
:10738000BE82AD82BE016F5F7F4F87E79FE00E94A4
:107390001ABC68ED73E10F942A281F5FFFEFEF1A04
:1073A000FF0A143011F726960FB6F894DEBF0FBE11
:1073B000CDBFDF91CF911F91FF90EF90DF90CF90E5
:1073C000BF90AF900895F601858190E0B0E0A0E015
:1073D00089839A83AB83BC83BE82AD82BE016F5F1B
:1073E0007F4F87E79FE00E941ABC66ED73E1D3CF21
:1073F000FC01DC018D918111FDCF30E020E050E0F7
:1074000040E08AE09191992301F1443051055CF507
:107410009E3271F42F3F310509F02CF5DB01A40FEA
:10742000B51F12962C934F5F5F4F30E020E0EACFFC
:10743000829FD001839FB00D1124292F990F330B08
:10744000205331092A0F3B1FDDCF2F3F310509F0B3
:1074500054F4443051053CF4640F751FFB01228342
:1074600081E090E0089590E080E00895CF92DF926F
:10747000EF92FF920F931F93CF93DF93EC016A017A
:107480007B01CB01BA010F94005E8B011F936F93B8
:1074900084E298E09F938F93DF93CF930F94E16101
:1074A0000F900F900F900F900F900F9020E030E012
:1074B000A901C701B6010F94365E181624F0F7FA39
:1074C000F094F7F8F09409900020E9F721978EE204
:1074D0008883B80117FF03C0719561957109072E64
:1074E000000C880B990B0F94355B9B01AC01C70115
:1074F000B6010F94215D20E030E040E251E40F94AA
:10750000945B0F94005E605D69831A82DF91CF9176
:107510001F910F91FF90EF90DF90CF900895CF9340
:10752000DF931F921F92CDB7DEB78091A212909188
:10753000A312009711F48EEA92E1BE016F5F7F4FB4
:10754000681B790B072E000C880B990B0F900F907E
:10755000DF91CF9108954F925F926F927F929F92A9
:10756000AF92BF92CF92DF92EF92FF920F931F9351
:10757000CF93DF93CDB7DEB768970FB6F894DEBF31
:107580000FBECDBFFC01198A1A8A1B8A1C8A1D8A6C
:107590001E8A1F8A188E8A89807F8A8BA081B1817A
:1075A000109709F47AC08C91882309F476C0008181
:1075B0001181D8019C91992309F443C09D3209F4AB
:1075C000DAC090539A3028F00F5F1F4F1183008369
:1075D000EECFC801912CDC016D01C81AD90A2D919A
:1075E000022E000C330B205331092A303105A0F351
:1075F0007F016EE270E0C8010F945161FC010097B9
:1076000009F448C0DC015D01AE1ABF0A11968C91E5
:107610001197082E000C990BC09711960A9798F3B2
:107620008181282F082E000C330B205331092A307A
:10763000310518F480330CF057C020E030E0A90188
:1076400008C0912CD12CC12CD3CF29E030E040E0F0
:1076500050E0AAE0B0E00F94B95C2B013C0122811C
:10766000822F022E000C990BC0978A30910570F47E
:1076700020330CF441C02A330CF042C0092E000C18
:10768000AA0BBB0B480E591E6A1E7B1EA114B10427
:1076900009F088C0CD2809F073C088E0FE0171961A
:1076A000DE01199601900D928A95E1F729853A85B8
:1076B0004B855C856D857E858F85988968960FB62C
:1076C000F894DEBF0FBECDBFDF91CF911F910F9118
:1076D000FF90EF90DF90CF90BF90AF909F907F9002
:1076E0006F905F904F9008958A330CF0AECF032EC9
:1076F000000C440B550BADCF80E090E0DC01C2CF15
:1077000089E090E0A0E0B0E0BDCFB8E0CB16D104B6
:107710000CF04DC0C8010F94EB549B01AC01A4E6E2
:10772000B0E00F94B95C992041F07094609450944B
:107730004094411C511C611C711C2A89207F2660C9
:107740002A8B460E571E681E791E4D8A5E8A6F8AE6
:10775000788E6CE270E0F701808191810F94516125
:10776000009721F4D7011D921C9297CF0196F70143
:107770009183808392CFC8010196992493942BCF53
:10778000C8010F94EB54AB01BC01CE0141960E949D
:107790005B7829833A834B835C836D837E838F83FD
:1077A0009887D7CFF3E0AF16B1040CF4AECFC80181
:1077B0000F94C9542A89207F27602A8B6D8B7E8B7A
:1077C0008F8B988FC6CFCF92DF92EF92FF920F935D
:1077D0001F93CF93DF93EC01A881B981109781F1BA
:1077E0008C91882369F108811981F801908199238E
:1077F00051F09D3241F090539A3028F00F5F1F4FA7
:1078000019830883F0CFC8010F94EB546B017C01FE
:107810006CE270E0C8010F945161009769F419821D
:107820001882C701B601DF91CF911F910F91FF9090
:10783000EF90DF90CF900895019699838883F1CFE0
:10784000C12CD12C7601EDCF0097B1F1FC01DB0109
:10785000AC01405F5F4F80E090812FE9290F263017
:1078600098F497559295907F9C9321813FE9320F30
:107870003630B0F42755922B9D933296E417F507D6
:1078800059F791E0892708952FEB290F263010F43E
:107890009753E8CF90539A3028F381E090E0E2CFFD
:1078A0003FEB320F363010F42753E5CF20532A3008
:1078B00010F381E020E0DFCF80E008950097D1F061
:1078C000DC011696ED91FC913097A1F080858F70C8
:1078D000843021F481859285009771F40680F781C8
:1078E000E02D309739F080858F70843019F48185D0
:1078F0009285089590E080E0089508950F931F9376
:10790000CF93DF93EC010A811B8170E060E0C80136
:107910000E9473B31816D4F48A8761E070E0C8013E
:107920000E9473B3181619069CF49987888762E041
:1079300070E0C8010E9473B31816190664F49C879E
:107940008B87DF91CF911F910F91089583E0E4CF52
:107950008BE290E0EACF88E590E0F1CF08950895BA
:10796000089508950F931F93CF93DF93EC011D8625
:107970000A811B8170E060E0C8010E9473B387FD3B
:1079800044C08C838C818150853410F080E28C83DC
:1079900061E070E0C8010E9473B387FD3BC08D8336
:1079A0008D818150853410F081E28D8362E070E03A
:1079B000C8010E9473B3863490F58E8363E070E053
:1079C000C8010E9473B39C01215031092115344034
:1079D00040F59A87898764E070E0C8010E9473B31C
:1079E000813024E0920700F59C878B8765E070E08A
:1079F000C8010E9473B318161906CCF498878F83B8
:107A0000DF91CF911F910F91089581958C8381E033
:107A10008D87B8CF81958D8381E08D87C1CF1E8200
:107A2000CDCF1A861986D7CF80E094E0DDCF80E1F4
:107A300097E2E4CF08950895CF93DF93EC0165E7D3
:107A400072E188E290E10F942A2860E772E188E20F
:107A500090E10F942A286C817D814AE050E088E211
:107A600090E10F94CB276AE672E188E290E10F94EF
:107A70002A2888E290E10F94BE2661E08C810F9461
:107A800076026E818C810F9448028A819B810097D7
:107A900029F040E050E0BA010E94A6B2E881F981E5
:107AA0000484F585E02D62E0CE0119958A819B81E1
:107AB000009799F00E94F3D11816190674F40A8001
:107AC000DB81C02D4FEF5FEFBA0180E00F94674775
:107AD000AB01BC01CE010E94A6B281E090E0DF9133
:107AE000CF910895CF93DF93EC0167E472E188E2D0
:107AF00090E10F942A286C817D814AE050E088E271
:107B000090E10F94CB2765E472E188E290E10F9455
:107B10002A28EA81FB810280F381E02D6081718156
:107B200088E290E10F9414286FE372E188E290E11B
:107B30000F942A2888E290E10F94BE268A819B81C7
:107B4000892B09F451C08C819D81892B09F04CC08F
:107B5000E881F981008CF18DE02DCE0119958130FD
:107B6000910529F0029759F061E08C811AC063E019
:107B700070E0CE010E9409EB61E00F94760261E0B3
:107B80008C810F94760261E070E0CE010E9409EBD7
:107B900061E00F94760262E070E0CE010E9409EB92
:107BA00061E00F9476028091A100887F8093A1000C
:107BB00080919100887F809391008091A1008260E4
:107BC0008093A10080919100826080939100E88170
:107BD000F9810484F585E02D62E0CE01199581E0FC
:107BE00090E0DF91CF91089590E080E0FACF2F925E
:107BF0003F924F925F926F927F928F929F92AF923D
:107C0000BF92CF92DF92EF92FF920F931F93CF9389
:107C1000DF93CDB7DEB760970FB6F894DEBF0FBE27
:107C2000CDBF9A838983DC011496ED91FC91309746
:107C300009F45DC1868097808114910409F41DC107
:107C4000D401ED91FC91309709F413C18081882310
:107C500009F40FC12FEF3FEFA9016EEE75E0C401EB
:107C60000E94252922E030E040E050E069EE75E016
:107C7000C4010E9425292FEF3FEFA90167E376E0B9
:107C8000C4010E94252965E675E0C4010E9470F1D7
:107C9000988B8F87009709F4ECC0FC0180858F706A
:107CA000853009F0E6C0CF010E94B3F2833008F4BA
:107CB000E0C020E030E040EA51E464EE75E0C40149
:107CC0000E94F0288C010E94EF1B20E030E040EA87
:107CD00051E460E476E0C4010E94F0286C010E9447
:107CE000EF1B20E030E040E050EC64E476E0C401BB
:107CF0000E94F0287C010E94EF1B20E030E040E869
:107D00005FE370E060E08F8598890F9476462B01E1
:107D10003C0120E030E0A9010F942E5BB12C87FFDD
:107D200006C077FA709477F87094BB24B39420E07F
:107D300030E0A90161E070E08F8598890F94764664
:107D40006B837C838D839E8320E030E0A90162E019
:107D500070E08F8598890F9476466F83788789873E
:107D60009A8720E030E040EA50E463E070E08F85DD
:107D700098890F9476466B877C878D879E878CE3E6
:107D800090E00F9400531C019801275F3F4FA7011B
:107D9000475F5F4FB601675F7F4F1F92BF92FA85C3
:107DA000FF9389858F9398859F93AF81AF93AB8025
:107DB000BC80CD80DE8083017201C1010F94162C3E
:107DC000C101032C000CAA0BBB0BEF85F88981873E
:107DD0009287A387B48761E070E0C1010F94772B8D
:107DE00020E030E04AE754E46B857C858D859E85F4
:107DF0000F94945B0F94005EAF85B88919968D91AE
:107E00009C910F94C92B6AE97FE088E290E10F947E
:107E10002A28B301A20188E290E10E94B6F667E445
:107E200076E088E290E10F9414284B815C816D81AB
:107E30007E8188E290E10E94B6F66BE476E088E20B
:107E400090E10F9414283F81288599858A85432FD6
:107E5000522F692F782F88E290E10E94B6F688E2CF
:107E600090E10F94BE260F900F900F900F900F90FF
:107E70000F90F40182809380DFCE6FE87FE088E28C
:107E800090E10F942A2888E290E10F94BE2640E00A
:107E900050E0BA01A981BA8112968D919C910E94FD
:107EA000A6B2A981BA81ED91FC9111970484F58560
:107EB000E02D62E0CD01199581E090E060960FB66B
:107EC000F894DEBF0FBECDBFDF91CF911F910F9110
:107ED000FF90EF90DF90CF90BF90AF909F908F90EA
:107EE0007F906F905F904F903F902F9008956BE739
:107EF0007FE088E290E10F942A2888E290E10F94D5
:107F0000BE2690E080E0DACFCF93DF93EC010E94B1
:107F1000B23C6FE476E088E290E10F94C22661E023
:107F20008C810F94760261E08D810F9476026D85CD
:107F30008C810F9448026D858D810F94480260E01A
:107F40008E810F94760240E050E0BA018A819B81D5
:107F50000E94A6B240E050E061E070E08A819B811F
:107F60000E9452B440E050E062E070E08A819B8160
:107F70000E9452B4E881F9810484F585E02D62E025
:107F8000CE01199582E08093270281E090E0DF9195
:107F9000CF9108956F927F928F929F92AF92BF92EE
:107FA000CF92DF92EF92FF920F931F93CF93DF93C5
:107FB0003C01DC0114968D919C911597892B71F4ED
:107FC0001296CD91DC9184E190E00F940053BC01B6
:107FD000CE010E9463B2E3019D838C83F301C481CF
:107FE000D581209769F46BE87CE081E89FE00F94ED
:107FF0002A2881E89FE00F94BE2690E080E0B4C27A
:108000004FEF5FEFBA0180E00F9467476E837F8385
:1080100088879987D3011496ED90FC901597E11409
:10802000F104D1F01296ED91FC913097A9F0C48142
:10803000D581209789F088858F70853069F4CE01CD
:108040000E94B3F2823040F000916D0A10916E0AE6
:108050000115110509F096C06EE47CE081E89FE00F
:108060000F942A2861E070E0E3018C819D81892BC7
:1080700011F470E060E04AE050E081E89FE00F9486
:10808000CB276CE47CE081E89FE00F942A2861E034
:1080900070E0F30182819381892B11F470E060E03C
:1080A0004AE050E081E89FE00F94CB276AE47CE04F
:1080B00081E89FE00F942A28D3011296ED91FC915C
:1080C00061E070E084819581892B11F470E060E0BB
:1080D0004AE050E081E89FE00F94CB2768E47CE021
:1080E00081E89FE00F942A28E301EA81FB81048064
:1080F000F581E02D80858F7061E070E0853011F4AE
:1081000070E060E04AE050E081E89FE00F94CB2708
:1081100066E47CE081E89FE00F942A28D301129660
:10812000ED91FC91848195810E94B3F261E070E051
:10813000823010F070E060E04AE050E081E89FE0BB
:108140000F94CB2781E89FE00F94BE2663E67CE086
:1081500081E89FE00F942A2881E89FE00F94BE26D3
:10816000D301ED91FC910484F585E02D61E0C3011C
:108170001995E301E881F9810084F185E02DC301BF
:1081800019953BCF61E0CE010E9422F2EC01888577
:108190008F70843029F469857A856115710539F409
:1081A0006EE27CE081E89FE00F942A28CBCFC801E3
:1081B0000E9470F18C01009769F46CE07CE081E82A
:1081C0009FE00F942A2869857A8581E89FE00F94C3
:1081D0001428B8CF6BE576E00E9470F1009709F49F
:1081E000D2C0EC0128852F70243009F0CCC0C9849E
:1081F000DA84D0E0C0E0C114D10409F4B7C0BE01F4
:108200006859744FC6010F943955892B09F0A9C0DC
:10821000FE01E459F44F25913491922F832FF701F9
:108220009283838362E676E0C8010E9470F1E301E5
:10823000EC81FD81009709F4AEC0DC0118962C9109
:1082400018972F70223009F0A6C019968D919D9134
:108250000D90BC91A02D0097A105B10509F49BC01C
:108260009183808340815181052E000C660B770B32
:10827000228189EC9CE00F94772967E676E0C801BB
:108280000E9470F17C01F301C481D581009709F44B
:1082900088C0DC0118968C918F70863009F081C0FF
:1082A0006CE676E0C7010E9470F19B878A8761E7E0
:1082B00076E0C7010E9470F19D878C8765E776E0C4
:1082C000C7010E9470F19F878E876BE776E0C70138
:1082D0000E9470F1998B888B60E876E0C7010E945C
:1082E00070F1009709F45AC0FC01818592859D8345
:1082F0008C8366E876E0C8010E9470F19B8B8A8BC4
:10830000892B09F40FC166EF7BE088E290E10F94BE
:108310002A2888E290E10F94BE26D3011496ED91AD
:10832000FC910288F389E02DC681D781209709F45A
:1083300041C06AE876E0CE010E9470F1009769F0D2
:10834000FC0120852F70213041F48185882329F09C
:1083500068817981C3010E94952E0A80DB81C02D3E
:10836000E5CF2696C834D10509F045CF6BE47BE014
:1083700088E290E10F942A2888E290E10F94BE26CB
:1083800096E080E04CCF86E090E0D70113969C9376
:108390008E93129747CF80E895E262CF88EE93E004
:1083A000A6CF1B861A8688EE93E09D838C831D865C
:1083B0001C869FCF60EE7BE088E290E10F942A2834
:1083C00088E290E10F94BE26D3011496ED91FC91C2
:1083D0000288F389E02DE680F780E114F10409F4C6
:1083E0007BC064EB75E0C7010E9470F1009709F44F
:1083F00068C063E976E00E9470F18C01009709F48F
:1084000060C0EC0188858F70823009F04EC0C9844D
:10841000DA84D3011496ED91FC910288F389E02D62
:10842000309709F456C0C681D78146010D2C000C47
:10843000AA08BB08209709F44CC067E976E0CE0192
:108440000E9470F1009709F440C0FC0120852F7054
:108450002230D9F581859285A385B4858815990543
:10846000AA05BB0591F56FEB7BE088E290E10F94E4
:108470002A286881798188E290E10F94142860EBC2
:108480007BE088E290E10F942A284AE050E0B601B0
:1084900088E290E10F94CB2788E290E10F94BE260A
:1084A00068817981C3010E94952EF80180858F70C3
:1084B000843039F4D80119966D917C91C3010E94E2
:1084C000952EE701EA80FB8088CF0A80DB81C02DF2
:1084D000B1CF70E060E0E6CF66EC7BE088E290E14F
:1084E0000F942A2888E290E10F94BE26D3011296B9
:1084F000ED91FC9162E0848195810E9422F20097C7
:1085000089F0FC01C681D781209761F0CE010E94DD
:108510000F1C882319F0CE010F9485010A80DB819E
:10852000C02DF2CF66E77CE087E79FE00F942A2812
:10853000D3011296ED91FC910280F381E02D6081D0
:10854000718187E79FE00F94142887E79FE00F94DD
:10855000BE26E301E881F9810484F585E02D62E01F
:10856000C301199581E090E0DF91CF911F910F91A8
:10857000FF90EF90DF90CF90BF90AF909F908F9043
:108580007F906F900895CF93DF93EC0166EE7AE0D1
:1085900088E290E10F942A28EA81FB810280F3812E
:1085A000E02D6081718188E290E10F94142888E2C7
:1085B00090E10F94BE26E881F9810484F585E02DD1
:1085C00062E0CE01199581E090E0DF91CF910895AE
:1085D000DC01ED91FC910484F585E02D62E01995B4
:1085E00081E090E008950F931F93CF93DF93DC0118
:1085F00012962D913C91232B81F1EC0160E679E0FC
:1086000088E290E10F942A284AE050E06E8188E2E7
:1086100090E10F94E12688E290E10F94BE268C81D0
:108620009D81892B61F40A811B818CE290E00F947B
:108630000053BC01C8010E9463B29D838C83EC810E
:10864000FD81309769F46EE479E081E89FE00F9452
:108650002A2881E89FE00F94BE2690E080E04BC07E
:1086600085E2DF011D928A95E9F7EC81FD8182E2C6
:108670008283EC81FD8116A2EC81FD8115A2EC8143
:10868000FD8117A20C811D814FEF5FEFBA0180E0E1
:108690000F946747F80160A771A782A793A78E81FF
:1086A000811116C062E00F94760265E179E087E7F8
:1086B0009FE00F942A2887E79FE00F94BE268BE85F
:1086C0009FE00F947E1F1092450281E08093751108
:1086D00026E040E855E260E070E08F8198850F94D5
:1086E0007729E881F9810484F585E02D62E0CE01E7
:1086F000199581E090E0DF91CF911F910F9108953E
:108700002F923F924F925F926F927F928F929F92A1
:10871000AF92BF92CF92DF92EF92FF920F931F938F
:10872000CF93DF93CDB7DEB7CB57D1090FB6F8940F
:10873000DEBF0FBECDBFE296EFAEE297E396FFAE8F
:10874000E397E4960FAFE497E5961FAFE597E696BB
:108750002FAFE697E7963FAFE797E8964FAFE897DA
:10876000E9965FAFE9970097B9F124012B2CEC96BD
:10877000AFAEEC97EB96DFAEEB97EA96CFAEEA970B
:10878000362E8C0180914502893020F4809144027C
:108790008930C0F0C8010E942DFA7C01892B91F02C
:1087A0006BE976E088E290E10F941428B70188E243
:1087B00090E10F94142888E290E10F94BE26C7013F
:1087C0000F949C53F80180858F70843009F461C147
:1087D00028F4882309F466C180E02FC0853009F4AD
:1087E00046C08630C9F761EA76E0C8010E9470F1A0
:1087F0003C01009709F476C0912C812CB12CA12C5E
:10880000D12CC12CE296EFACE297E396FFACE39754
:10881000E4960FADE497E5961FADE597E6962FAD8C
:10882000E697E7963FADE797E8964FADE897E9966C
:108830005FADE997632D0E948043C558DF4F0FB6A7
:10884000F894DEBF0FBECDBFDF91CF911F910F9186
:10885000FF90EF90DF90CF90BF90AF909F908F9060
:108860007F906F905F904F903F902F9008958091F0
:108870008D118F5F80938D116680778061147104F4
:1088800059F14201EC96AFACEC97B22CEA96CFAC22
:10889000EA97EB96DFACEB97E296EFACE297E396C4
:1088A000FFACE397E4960FADE497E5961FADE5972F
:1088B000E6962FADE697E7963FADE797E8964FAD82
:1088C000E897E9965FADE997632DC3010E94804365
:1088D000F30162807380D2CF80918D11815080939B
:1088E0008D117ACF65EA76E0C8010E9470F12C0103
:1088F0006AEA76E0C8010E9470F17C016FEA76E0D6
:10890000C8010E9470F1332039F0F1E03F1609F4FC
:10891000A1C0D12CC12C0CC063EB76E0C8010E9431
:1089200070F13C0168EB76E0C8010E9470F16C01C7
:108930006114710409F43801C114D10409F4680107
:108940004114510431F4EA964FACEA97EB965FACD0
:10895000EB97E114F10421F4EC96EFACEC97F22CD8
:108960006114710409F4A7C0F30180858F7084300D
:1089700009F0A1C061847284C114D10409F49EC0BD
:10898000F60180858F70843009F098C0C184D2844C
:1089900010E000E04114510409F4F5C061147104C1
:1089A00009F4B3C060E374E188E290E10F942A28EF
:1089B000F2016185728588E290E10F9414286BE2E0
:1089C00074E188E290E10F942A28B30188E290E1F3
:1089D0000F94142888E290E10F94BE26CE018F58A0
:1089E0009F4F0E947C7DE114F10409F0D5C0F20193
:1089F00080858F70843009F085C14091911150912C
:108A0000921161857285CE0101960E9432BBCE0122
:108A100001960E9456B28823C1F00E948F3A6B01E2
:108A2000683C71050CF085C06AEE73E181E89FE057
:108A30000F942A284AE050E0B60181E89FE00F94A5
:108A4000CB2781E89FE00F94BE26CE0101960E94BD
:108A5000CFBB58C16DEB76E0C8010E9470F13C01BC
:108A600062EC76E0C8010E9470F16C01611471043F
:108A700009F04AC163EB76E0C8010E9470F13C0145
:108A8000C114D10409F44ECF892B09F059CF380114
:108A900057CFD12CC12C712C612CF12CE12C512CF5
:108AA000412C46CFD12CC12C712C612CF12CE12C06
:108AB000512C412C45CF712C612C5ECF00E020E081
:108AC00030E340E150E0BE016F597F4FCE018F5837
:108AD0009F4F0E945C7B6C01E4960FADE49710E021
:108AE0000115110509F056CFE2968FADE29781117D
:108AF00009C0E3968FADE3978F7009F44BCF02E086
:108B000010E048CF01E010E045CF61E274E188E277
:108B100090E10F942A28F2016185728588E290E144
:108B20000F9414286CE174E188E290E10F942A28F4
:108B300055CF6114710431F0B301CE0101960E944A
:108B40006CFA83CFA12CC12CF12CE12CE2960FAD55
:108B5000E297E3961FADE397E4962FADE497E59691
:108B60003FADE597E6964FADE697E7965FADE797A1
:108B7000E8966FADE897E9967FADE997CE0101964B
:108B80000E9473BE62CFE114F10409F4BBC0C114AA
:108B9000D10409F4B7C004C0C114D10409F427CF2B
:108BA000F70180858F70843009F0A8C08185928597
:108BB00025961FAE1EAE259748EE53E060E070E0AC
:108BC00029964CAF5DAF6EAF7FAF299724E532E0B9
:108BD00023963FAF2EAF23972F969FAF8EAF2F9741
:108BE00061961FAE1EAE619763961FAE1EAE639771
:108BF00065961FAE1EAE659767961FAE1EAE679751
:108C000069961FAF0EAF69976A961FAE6A9740E4E8
:108C100050E0BE016F5F7F4FCE018F5B9F4F0E9480
:108C200018F321E030E02C0F3D1F820F931FFC0151
:108C3000108264E174E188E290E10F942A28F70140
:108C40006185728588E290E10F94142867EC76E0E4
:108C500088E290E10F941428BE016F5F7F4F88E295
:108C600090E10F9414286FE074E188E290E10F9492
:108C70002A28B60188E290E10F94142888E290E156
:108C80000F94BE260E948EF18823C1F18091280C9A
:108C9000811134C06FE270E0CE0101960F945161F2
:108CA000892B51F4F7012185328543E050E060E4DF
:108CB000CE0101960E940E3968E074E188E290E1ED
:108CC0000F942A28BE016F5F7F4F88E290E10F94D6
:108CD000142863E074E188E290E10F942A28B60139
:108CE00088E290E10F94142888E290E10F94BE2668
:108CF00041E0B601CE0101960F944A074114510498
:108D000009F075CE81E099CD892B09F019CE0ACEF4
:108D10008F929F92AF92BF92CF92DF92EF92FF928B
:108D20000F931F93CF93DF9300D000D01F921F9219
:108D3000CDB7DEB7DC011296ED91FC91309709F4C6
:108D400068C024813581232B09F463C08C0166231C
:108D500009F472C00E94B427E62EB72E6C01D80128
:108D60001296ED91FC910280F381E02D608171817A
:108D700081E89FE00F94142863ED71E181E89FE0A2
:108D80000F942A2881E89FE00F94BE2620E030E06F
:108D9000A9016E2D7B2DC6010F94365E87FD39C06B
:108DA00067EC71E181E89FE00F942A284E2D5B2D3E
:108DB000B60181E89FE00E94B6F681E89FE00F943B
:108DC000BE26D8011296ED91FC9161E084819581D7
:108DD0000E9422F219821A821B821C822A81207F21
:108DE0002760F22E2E2D4E2D5B2DB6014D835E8316
:108DF0006F837887912C812CB12CA12CD12CC12C84
:108E0000E9800B811C813E814F8158856FEF0E9464
:108E1000804328960FB6F894DEBF0FBECDBFDF911A
:108E2000CF911F910F91FF90EF90DF90CF90BF9067
:108E3000AF909F908F9008950280F381E02D608124
:108E4000718187E79FE00F94142860EE71E187E756
:108E50009FE00F942A2887E79FE028960FB6F894A2
:108E6000DEBF0FBECDBFDF91CF911F910F91FF905D
:108E7000EF90DF90CF90BF90AF909F908F900D9428
:108E8000BE264F925F926F927F928F929F92AF9287
:108E9000BF92CF92DF92EF92FF920F931F93CF93E7
:108EA000DF93CDB7DEB7E8970FB6F894DEBF0FBEFD
:108EB000CDBF09AB1AAB2BAB3CAB4DAB5EAB6FABD5
:108EC00078AFDC011496ED91FC91309719F490E0A5
:108ED00080E0CBC020813181232BC9F33C01DC0130
:108EE000ED91FC910284F385E02D1995029779F7B5
:108EF0008BA9E82EF12C19A9112321F0E114F1041A
:108F000009F433C1823009F4D9C0B8F4882309F4D4
:108F1000D5C08130B9F063EF71E188E290E10F9440
:108F20002A284AE050E0B70188E290E10F94CB276D
:108F300088E290E10F94BE26CACF833009F447C07F
:108F4000893049F7D3011296ED91FC9161E084815B
:108F500095810E9422F22C0119A61AA61BA61CA616
:108F60001DA61EA61FA618AA8AA5807F8AA719A7D4
:108F700061E0CE0189960E94177829A33AA34BA3FA
:108F80005CA36DA37EA38FA398A71150163108F0A0
:108F9000FDC1E12FF0E08827EF52F84B8F4F0D9481
:108FA000EF5CFB48B948C649C649C649C649C649E7
:108FB000C649C6492A498A49C649C649FB48FB48A9
:108FC000C649C649C649FB48FB48FB48FB488AA935
:108FD0008F7009F47CCFCE01C1960E94667AD301CE
:108FE0001496ED91FC91668377838087918769E37E
:108FF00072E188E290E10F942A28D3011296ED9154
:10900000FC910280F381E02D6081718188E290E122
:109010000F9414286BE272E188E290E10F942A2801
:10902000D3011496ED91FC9146815781608571853D
:1090300088E290E10E94B6F688E290E10F94BE26A5
:10904000F301E480F5800F94AD06D70152966D933D
:109050007D938D939C935597D3011496ED91FC913C
:109060008689811119C081E090E0E8960FB6F894E6
:10907000DEBF0FBECDBFDF91CF911F910F91FF904B
:10908000EF90DF90CF90BF90AF909F908F907F90A8
:109090006F905F904F900895168A60E0C3010E9420
:1090A0008846D3011496ED91FC9180E090E0A0E019
:1090B000B0EC86879787A08BB18BD5CF8AA98F70AC
:1090C00009F405CFCE01C1960E94667AD3011496A9
:1090D000ED91FC91628773878487958765E272E1E1
:1090E00088E290E10F942A28D3011296ED91FC9129
:1090F0000280F381E02D6081718188E290E10F941C
:1091000014286AE172E188E290E10F942A28D301E1
:109110001496ED91FC91428553856485758588E2AE
:1091200090E10E94B6F688E290E10F94BE26D3014A
:109130001296ED91FC9162E0848195810E9422F269
:10914000009709F490CF912C812CB12CA12CD12C1B
:10915000C12CE9A8FAA80BA91CA92DA93EA94FA9C1
:1091600058AD6FEF0E9480437ECFEE24E394F12C44
:10917000E9CE8091290C90912A0C0597F1F0198283
:109180001A821B821C821D821E821F8218868A817F
:10919000807F8A836BE0CE0101960E943978912C02
:1091A000812CB12CA12CD12CC12C79018A019B01DD
:1091B000AC016FEFC2010E948043912C812CB12C35
:1091C000A12CD12CC12CE9A4FAA40BA51CA52DA57A
:1091D0003EA54FA558A96FEFC2010E94804330E021
:1091E00020E040E050E460E070E0F3018281938190
:1091F0000E942BB838CF19821A821B821C821D82D2
:109200001E821F8218868A81807F8A8340E051E017
:1092100060E070E0D30112968D919C910E94A4B4FD
:10922000672B682B692BA1F06BE0CE0101960E94A1
:109230003978912C812CB12CA12CD12CC12C790105
:109240008A019B01AC016FEFC2010E948043BBCF3A
:109250006AE0EBCF8091290C90912A0C059791F050
:1092600061E0D30112968D919C910E94C7BA30E0C3
:1092700020E040E050E160E070E0F3018281938102
:109280000E942BB840E050E061E070E0D3011296FC
:109290008D919C910E947BB4912C812CB12CA12C9E
:1092A000D12CC12CE9A4FAA40BA51CA52DA53EA583
:1092B0004FA558A96FEFC2010E948043D301ED91E1
:1092C000FC910288F389E02DC3011995892B09F4DB
:1092D000E8CE19821A821B821C821D821E821F8286
:1092E00018868A81807F8A8361E0CE0101960E9480
:1092F000397829873A874B875C876D877E878F8788
:10930000988B79018A019B01AC016FEFC2010E9429
:109310008043C7CE912C812CB12CA12CD12CC12CF7
:10932000E9A4FAA40BA51CA52DA53EA54FA558A9F7
:109330006FEFC2010E948043D301ED91FC9102883E
:10934000F389E02DC3011995892B09F08CCE19867C
:109350001A861B861C861D861E861F86188A8A858D
:10936000807F8A8762E0CE0109960E94397829833E
:109370003A834B835C836D837E838F8398877901E7
:109380008A019B01AC016FEFC201ECCE68E072E193
:1093900088E290E10F942A284AE050E069A988E227
:1093A00090E10F94E12688E290E10F94BE26B3CDC0
:1093B0002F923F924F925F926F927F928F929F92E5
:1093C000AF92BF92CF92DF92EF92FF920F931F93D3
:1093D000CF93DF93CDB7DEB764970FB6F894DEBFB7
:1093E0000FBECDBF1C01DC0114968D919C91159789
:1093F000892B99F41296ED91FC91FA83E98389E126
:1094000090E00F940053BC0189819A810E9463B25D
:10941000D10115969C938E931497F10104811581C7
:109420000115110569F468E671E181E89FE00F9488
:109430002A2881E89FE00F94BE2690E080E09CC33C
:10944000D8011D921C920280F381E02DFC8BEB8BE6
:10945000309791F0848195819A838983009761F098
:10946000DC0118968C9118978F70853029F4CD0106
:109470000E94B3F2811190C06EE271E181E89FE039
:109480000F942A2861E070E0F10184819581892B95
:1094900011F470E060E04AE050E081E89FE00F9452
:1094A000CB276CE271E181E89FE00F942A2861E00C
:1094B00070E0D10112968D919C91892B11F470E08E
:1094C00060E04AE050E081E89FE00F94CB276AE239
:1094D00071E181E89FE00F942A28D1011296ED9165
:1094E000FC9161E070E084819581892B11F470E03A
:1094F00060E04AE050E081E89FE00F94CB2768E20B
:1095000071E181E89FE00F942A28D1011296ED9134
:10951000FC910480F581E02D80858F7061E070E022
:10952000853011F470E060E04AE050E081E89FE0AF
:109530000F94CB2766E271E181E89FE00F942A281F
:10954000D1011296ED91FC91848195810E94B3F234
:1095500061E070E0823010F070E060E04AE050E0DE
:1095600081E89FE00F94CB2781E89FE00F94BE260F
:1095700062E471E181E89FE00F942A2881E89FE08E
:109580000F94BE26D101ED91FC910484F585E02D68
:1095900061E0C101199551CF60E089819A810E94F3
:1095A00022F29F838E83009729F0FC0180858F70C3
:1095B000853039F06CE071E181E89FE00F942A2852
:1095C000D3CF8E819F810E94B3F28150883008F002
:1095D000A3C1E82FF0E08827EF50F54B8F4F0D9493
:1095E000EF5C5D4C334C064C814B694B694B524BE5
:1095F000F94A67E08E819F810E9422F2FC019085EA
:109600009F70933009F041C0418452846384748414
:10961000F1E0FD8366E08E819F810E9422F2FC01D1
:1096200090859F70933009F045C081859285A38510
:10963000B48589839A83AB83BC8391E09D8364E086
:109640008E819F810E9422F2FC0190859F70933051
:1096500009F050C061857285838594850F94075EFB
:109660004B0163E08E819F810E9422F2FC01808584
:109670008F70833009F060C081859285A385B485A1
:109680008A879B87AC87BD8764C0923059F4618517
:109690007285838594850F94355B2B013C0181E0B5
:1096A0008D83B8CF412C512C8FE7682E83E4782E20
:1096B0001D82B0CF9230C9F461857285838594850F
:1096C0000F94355B69837A838B839C83A1E0AD83A0
:1096D000B6CF412C512CBFE76B2EB3E47B2E198201
:1096E0001A821B821C821D82AACF19821A821B82B7
:1096F0001C82A5CF9230C1F481849284A384B48467
:10970000B0CFF0EC8F2EF7E29F2EF9E0AF2EB12C08
:10971000412C512CAFE76A2EA3E47A2E19821A82CB
:109720001B821C821D829DCFE0EC8E2EE7E29E2ED6
:10973000E9E0AE2EB12C95CF823009F082C0618570
:109740007285838594850F94355B6A877B878C87C8
:109750009D8762E08E819F810E9422F2FC018085BC
:109760008F70833009F072C091859E87A285AF8784
:10977000B385B88B8485898B61E08E819F810E943F
:1097800022F2FC0180858F70833009F08BC0C18488
:10979000D284E384F48460E08E819F810E9422F26F
:1097A000FC0180858F70833009F0A9C08185928586
:1097B000A385B4858E839F83A887B98720E030E096
:1097C000A9016E817F81888599850F942E5B87FF23
:1097D000D0C08E819F81A885B985B0588E839F8324
:1097E000A887B98791E09A8BAB89BC891696ED91D1
:1097F000FC9180858F70823009F4BDC0833009F4FC
:10980000D4C180E090E0A0EAB1E4D3C160EC862E40
:1098100067E2962E69E0A62EB12C80E090E0A0EAE7
:10982000B0E48A879B87AC87BD87412C512C7FE7AA
:10983000672E73E4772E19821A821B821C821D8286
:1098400088CF80E090E0A0EAB0E41ACF823029F51A
:1098500061857285838594850F94355B6E877F87DC
:10986000888B998B89CF40EC842E47E2942E49E077
:10987000A42EB12C80E090E0A0EAB0E48A879B8718
:10988000AC87BD87412C512C5FE7652E53E4752EC4
:1098900019821A821B821C821D821E861F86188ACC
:1098A000198A6ACF823039F56185728583859485FE
:1098B0000F94355B6B017C016ECF20EC822E27E28A
:1098C000922E29E0A22EB12C80E090E0A0EAB0E434
:1098D0008A879B87AC87BD87412C512C3FE7632E3D
:1098E00033E4732E19821A821B821C821D821E860B
:1098F0001F86188A198AC12CD12C76014CCF823050
:1099000091F561857285838594850F94355B6E83AF
:109910007F838887998752CF80EC882E87E2982EA4
:1099200089E0A82EB12C80E090E0A0EAB0E48A871C
:109930009B87AC87BD87412C512C9FE7692E93E410
:10994000792E19821A821B821C821D821A8A1E8617
:109950001F86188A198AC12CD12C7601CE82DF820B
:10996000E886F98641CF1A8A1E821F8218861986D8
:109970003BCF1A8A39CF61857285838594850F9490
:10998000355BF8016287738784879587D8011696BF
:109990001D921D921D921C921997F801128213823A
:1099A000148215820F94AD06D80152966D937D9363
:1099B0008D939C935597D1011496ED91FC9181E084
:1099C000868B908E878A61E0C1010E948846F101F2
:1099D00004811581D8018D919C9163EF70E1892BF1
:1099E00009F0EACD8CE390E00F9400539C8B8B8BB5
:1099F0009801265F3F4FA8014E5F5F4FB8016A5F35
:109A00007F4F1F92BA89BF93E989EF93F889FF933B
:109A10008F858F939E859F9356016701EE80FF800F
:109A2000088519858B899C890F94162CD101149671
:109A3000ED91FC918B899C89918380830F900F908D
:109A40000F900F900F900F90009709F491CD61E067
:109A500070E00F94772BD1011496ED90FC90BD81AE
:109A6000BB2309F44AC0A301920169817A818B81E9
:109A70009C810F94365E87FF40C0F7010190F08112
:109A8000E02DFF83EE8389819A81AB81BC8182AB1B
:109A900093ABA4ABB5AB46AA57AA60AE71AE82AD8C
:109AA000882359F1068D178DF80180809180A2805E
:109AB000B380A5019401C301B2010F942E5B87FF0F
:109AC0007EC0D8014D925D926D927C921397AE81CB
:109AD000BF8196968D909D90AD90BC909997A50171
:109AE0009401C301B2010F942E5B87FF7DC0EE810C
:109AF000FF8146A257A260A671A620E030E04AE7A7
:109B000054E46A857B858C859D850F94945B0F94C6
:109B1000005ED7018D919C910F94C92B64E571E192
:109B200087E79FE00F942A28D1011296ED91FC91CE
:109B30000280F381E02D6081718187E79FE00F94BF
:109B4000142887E79FE00F94BE26D1011496ED916B
:109B5000FC9180E090E0A0E0B0EC86879787A08B36
:109B6000B18BD101ED91FC910484F585E02D62E08B
:109B7000C101199581E090E064960FB6F894DEBFBC
:109B80000FBECDBFDF91CF911F910F91FF90EF904E
:109B9000DF90CF90BF90AF909F908F907F906F900D
:109BA0005F904F903F902F90089581859285A38577
:109BB000B485F80182879387A487B587E7CEA5018E
:109BC000940169817A818B819C810F94365E18168D
:109BD0000CF07DCF89819A81AB81BC81F8018083B3
:109BE0009183A283B38373CFA501940169817A81A4
:109BF0008B819C810F94365E18160CF07ECF898184
:109C00009A81AB81BC81EE81FF8186A397A3A0A737
:109C1000B1A773CF4F925F926F927F928F929F9274
:109C2000AF92BF92CF92DF92EF92FF920F931F936A
:109C3000CF93DF93CDB7DEB760970FB6F894DEBF52
:109C40000FBECDBF6130710509F4DBC1DC01149694
:109C5000ED91FC913097C9F481E090E060960FB6E9
:109C6000F894DEBF0FBECDBFDF91CF911F910F9152
:109C7000FF90EF90DF90CF90BF90AF909F908F902C
:109C80007F906F905F904F90089520813181232BBA
:109C900019F33C01DC01ED91FC910284F385E02D88
:109CA00019950297C9F6F301E280F380E114F104FB
:109CB00099F2C7010E94E6BA823071F240E051E0A9
:109CC00060E070E0C7010E94A4B4672B682B692B89
:109CD00019F6D3011496ED91FC9180819181FC01DC
:109CE00022AD222309F455C10F94D929882309F400
:109CF00050C1D3011496ED91FC9186898823A1F07F
:109D0000C3010E94B4276B017C0120E030E0A9016F
:109D10000F94365E87FD08C0D3011496ED91FC9137
:109D2000C282D382E482F58267EA71E188E290E13F
:109D30000F942A28D3011296ED91FC910280F381B1
:109D4000E02D6081718188E290E10F94142861EA2E
:109D500071E188E290E10F942A28D3011496ED91E5
:109D6000FC91428553856485758588E290E10E9467
:109D7000B6F66CE971E188E290E10F942A28D301EC
:109D80001496ED91FC91468157816085718588E23A
:109D900090E10E94B6F66AEC76E088E290E10F94DA
:109DA0001428D3011496ED91FC9142815381648172
:109DB000758188E290E10E94B6F668E971E188E277
:109DC00090E10F942A28D3011496ED91FC91019013
:109DD000F081E02D408151816281738188E290E1C0
:109DE0000E94B6F664E971E188E290E10F942A28B6
:109DF000D3011496ED91FC910190F081E02D448106
:109E000055816681778188E290E10E94B6F660E92B
:109E100071E188E290E10F942A28D3011496ED9124
:109E2000FC910190F081E02D40855185628573851C
:109E300088E290E10E94B6F6D3011496ED91FC9170
:109E40008689882331F069E871E188E290E10F9416
:109E50002A2888E290E10F94BE26F301E480F58081
:109E6000D70156968C918111F7CE0281138161E062
:109E7000F801848195810E9422F22C0120E030E0DB
:109E8000A901D7011E966D917D918D919C9151975D
:109E90000F942E5B81110CC020E030E0A901F70186
:109EA00062817381848195810F94365E18165CF00F
:109EB00040E050E061E070E0C8010E94A4B4672B6C
:109EC000682B692B31F119861A861B861C861D8624
:109ED0001E861F86188A8A85807F8A8761E0CE0168
:109EE00009960E94397829833A834B835C836D837A
:109EF0007E838F839887912C812CB12CA12CD12C1F
:109F0000C12C79018A019B01AC016FEFC2010E9453
:109F1000804340E050E061E070E0D30112968D9103
:109F20009C910E9452B4D3011496ED91FC91328120
:109F300063815481458119861A861B861C868A8511
:109F4000807F8760F82E8A87232F832F962FA52F57
:109F5000B42F8D879E87AF87B88B912C812CB12C25
:109F6000A12CD12CC12CE9840B851C853E854F8505
:109F700058896FEFC2010E948043D3011496ED917E
:109F8000FC9182819381A481B58186879787A08B7C
:109F9000B18BD3011496ED91FC91868981115CCE31
:109FA0008789908D009709F457CE28EE33E0829F81
:109FB0002001839F500C929F500C11240F94AD06EA
:109FC000D3011496ED91FC914114510499F0620172
:109FD000F12CE12C0289138924893589AB01BC015C
:109FE000401B510B620B730B4C155D056E057F0515
:109FF00008F432CE81E0868B61E0C3010E9488467E
:10A000002BCE90E080E02ACE2F923F924F925F922B
:10A010006F927F928F929F92AF92BF92CF92DF9278
:10A02000EF92FF920F931F93CF93DF93CDB7DEB7DD
:10A03000C458D1090FB6F894DEBF0FBECDBFFC01E6
:10A04000902FA2960FAFA297A3961FAFA397A496A7
:10A050002FAFA497A5963FAFA597A6964FAFA6970B
:10A06000A7965FAFA797A8966FAFA897A9967FAF5F
:10A07000A99786EF800F823008F4A0C6EB96FFAE5A
:10A08000EEAEEB97AD96FFAFEEAFAD97822F422EBF
:10A09000512C002309F4A0C64114510409F491C6BF
:10A0A000EB96AEADBFADEB97AB2B09F49CC68730FA
:10A0B00051F5913109F429C2923109F446C2903127
:10A0C000F9F46FEF70E0CE018F599F4F0E94137922
:10A0D0006A962FAF6A976B963FAF6B976C964FAFB0
:10A0E0006C976D965FAF6D976E966FAF6E976F962C
:10A0F0007FAF6F97A0968FAFA097A1969FAFA197C4
:10A1000067E0462E512CAD96AEADBFADAD9714961F
:10A11000ED91FC91309709F474C466807780CF5735
:10A12000DF4F19821882C158D040E9961FAE1EAE8B
:10A13000E997E3961FAE1EAEE397312C212CE796EC
:10A140001FAE1EAEE7976114710409F468C46EEE89
:10A1500075E0C3010E9470F1E1969FAF8EAFE19769
:10A1600069EE75E0C3010E9470F1AB969FAF8EAFB0
:10A17000AB9769ED76E0C3010E9470F1CD57DF4FD8
:10A1800099838883C358D04065E675E0C3010E9477
:10A1900070F1ED969FAF8EAFED97E196EEADFFAD0E
:10A1A000E197309709F4C0C0AB962EAD3FADAB97A9
:10A1B0002115310509F4B8C080858F70823009F00F
:10A1C000B3C0D90118968C918F70823009F0ACC061
:10A1D0002CE330E040E050E069EB75E0C3010F9400
:10A1E000A246C358DF4F688379838A839B83CD5708
:10A1F000D040EB96EEADFFADEB973097F1F1BF019C
:10A20000D3018D919C910F945C61892BB1F5B2E0E3
:10A210004B16510409F4ABC30CF09FC1F1E04F168B
:10A22000510409F43CC2CD57DF4FE881F981C3588E
:10A23000D040309711F1912C812CB12CA12CD12C34
:10A24000C12CA296EFACA297A396FFACA397A496BD
:10A250000FADA497A5961FADA597A6962FADA6976F
:10A26000A7963FADA797A8964FADA897A9965FADC3
:10A27000A9976FEFCF010E948043AB96EEADFFAD83
:10A28000AB9781859285A385B48582309105A10520
:10A29000B10509F443C08F3F9F4FAF4FBF4FF1F15E
:10A2A000E196EEADFFADE19781859285A385B485FA
:10A2B000EF964EAD5FADEF97849F9001859F300D77
:10A2C000949F300D1124E796EEADFFADE797E20FB6
:10A2D000F31FE796FFAFEEAFE797CF57DF4FE88169
:10A2E000F981C158D040AF01FF0F660B770B4817BB
:10A2F00059076A077B0794F4CF57DF4F9983888308
:10A30000C158D040E9963FAF2EAFE997EF962EADFA
:10A310003FADEF97E3963FAF2EAFE397EF964EAD8D
:10A320005FADEF97240E351ED30112966D907C9091
:10A330000ACFA3968FADA3978F70E1F481E090E0F0
:10A34000CC57DF4F0FB6F894DEBF0FBECDBFDF9105
:10A35000CF911F910F91FF90EF90DF90CF90BF9022
:10A36000AF909F908F907F906F905F904F903F90B5
:10A370002F9008956DEE70E188E290E10F942A2805
:10A380006FED70E188E290E10F942A28CE018F5999
:10A390009F4F0E94667AAB01BC0188E290E10E9467
:10A3A000B6F688E290E10F94BE26AD96AEADBFAD95
:10A3B000AD9712960D911C914FEF5FEFBA0180E0BF
:10A3C0000F946747AB01BC01C8010E94A6B2CE0141
:10A3D0008F599F4F0E94667A6B017C016BE17AE096
:10A3E000AD96EEADFFADAD97848195810E9470F181
:10A3F000A701960160E476E00E94C2289FCF69ED34
:10A4000070E188E290E10F942A286FEC70E188E215
:10A4100090E10F942A284AE050E0A2966FADA297EF
:10A4200088E290E10F94E12688E290E10F94BE2645
:10A43000A2960FADA2976BE17AE0AD96AEADBFAD3F
:10A44000AD9714968D919C910E9470F16DE276E02B
:10A450000F944F467C01009709F470CFFC01808572
:10A46000982F9F70923039F0933081F0911166CF20
:10A47000807F8260808710E030E020E0D70119966D
:10A480000D931D932D933C931C9758CF602F70E034
:10A4900090E080E00F94335BD70119966D937D9324
:10A4A0008D939C931C974ACF69EC70E188E290E110
:10A4B0000F942A2867EB70E188E290E10F942A2834
:10A4C000CE018F599F4F0E94667AAB01BC0188E292
:10A4D00090E10E94B6F688E290E10F94BE26CE018C
:10A4E0008F599F4F0E94667A6B017C016BE17AE085
:10A4F000AD96EEADFFADAD97848195810E9470F170
:10A50000A701960160ED76E077CF60E870E0CE01BC
:10A510008F599F4F0E94137962962FAF629763966F
:10A520003FAF639764964FAF649765965FAF65974B
:10A5300066966FAF669767967FAF679768968FAF9F
:10A54000689769969FAF6997DBCD6AE070E0CE01AE
:10A550008F599F4F0E94137AD3CD23E042165104A6
:10A5600009F429C237E04316510409F05CCEA396E2
:10A570008FADA3978F7009F48CC0CE018F599F4F78
:10A580000E94AC7AAB96AEADBFADAB9719960D916C
:10A590001D912D913C911C97672B682B692B09F419
:10A5A000A6C00230110521053105B1F56DED76E04B
:10A5B00088E290E10F94142888E290E10F94BE267F
:10A5C00021E030E040E050E0AB96AEADBFADAB97E0
:10A5D00019962D933D934D935C931C9761E0CE01AA
:10A5E0008F599F4F0E9439782A962FAF2A972B9622
:10A5F0003FAF2B972C964FAF2C972D965FAF2D9793
:10A600002E966FAF2E972F967FAF2F9760968FAFB6
:10A61000609761969FAF6197CE018F599F4F0E94BF
:10A62000AC7AE196EEADFFADE197618772878387E3
:10A6300094878091290C90912A0C059751F1D301B0
:10A64000AD90BC9088248394C12C50E3D52EE12C8E
:10A65000F12CA2960FADA297A3961FADA397A49637
:10A660002FADA497A5963FADA597A6964FADA697FB
:10A67000A7965FADA797A8966FADA897A9967FAD4F
:10A68000A997AD96EEADFFADAD97828193810E9403
:10A69000C8B4A2968FADA297882309F4C4CDA29620
:10A6A0009FADA297992309F4BECDEFEFE90FE631F4
:10A6B00008F059C1F0E08827EF59FC4A8F4F0D94FC
:10A6C000EF5CBB535554B354B354B354B354B35465
:10A6D000B354B35473548D54B354B354A154A154CC
:10A6E000B354B354B354A154A154A154A154013050
:10A6F000110521053105B1F56EEE76E088E290E1B5
:10A700000F94142888E290E10F94BE2622E030E0F6
:10A7100040E050E0AB96AEADBFADAB9719962D9330
:10A720003D934D935C931C9762E0CE018F599F4FF0
:10A730000E94397822962FAF229723963FAF239716
:10A7400024964FAF249725965FAF259726966FAF37
:10A75000269727967FAF279728968FAF2897299619
:10A760009FAF2997E196EEADFFADE1971186128676
:10A77000138614865ECFE196AEADBFADE197199614
:10A780006D917C91CE018F599F4F0E94137929AF13
:10A790003AAF4BAF5CAF6DAF7EAF8FAF21969FAF3F
:10A7A000219767E0CE018F599F4F0E94177829AB00
:10A7B0003AAB4BAB5CAB6DAB7EAB8FAB98AFA296BD
:10A7C0008FADA29790E0B0E0A0E0AB96EEADFFAD0C
:10A7D000AB9781879287A387B487C12C40E3D42E9F
:10A7E000E12CF12C8091290C90912A0C059779F19C
:10A7F000AB96EEADFFADAB9781859285A385B48511
:10A800000197A105B10519F5E196EEADFFADE19710
:10A8100081859285A385B4854497A105B105BCF4D3
:10A820002EE130E040E050E02187328743875487B3
:10A830006EE170E0CE018F599F4F0E941379298FEE
:10A840003A8F4B8F5C8F6D8F7E8F8F8F98A3809107
:10A85000290C90912A0C059709F4E5CCF301A0800E
:10A86000B18088248394A2960FADA297A3961FADC2
:10A87000A397A4962FADA497A5963FADA597A696AE
:10A880004FADA697A7965FADA797A8966FADA8976F
:10A89000A9967FADA997AD96AEADBFADAD97129617
:10A8A0008D919C910E94C8B4BECC70E060E0CE0156
:10A8B0008F599F4F0E94137929A73AA74BA75CA7EE
:10A8C0006DA77EA78FA798AB67E0CE018F599F4FEA
:10A8D0000E94177829A33AA34BA35CA36DA37EA380
:10A8E0008FA398A76CCFED962EAD3FADED972115B8
:10A8F000310569F0F90181859285A385B4850097BA
:10A90000A105B10521F061E070E00F94772BC12C17
:10A9100020E4D22EE12CF12C65CFED962EAD3FAD8B
:10A92000ED972115310599F3F90181859285A3856C
:10A93000B4850097A105B10551F3DC01DA961C92AC
:10A94000E6CF892F90E0B0E0A0E0AB96EEADFFAD92
:10A95000AB9781879287A387B487C12C30E1D32E30
:10A96000E12CF12C3FCFC12CD12C76013BCFA3960B
:10A970008FADA3978F7009F456CCCE018F599F4F9E
:10A980000E94667A9B01AC0164EE75E0C3010E94EF
:10A99000C2288091290C90912A0C059709F443CC88
:10A9A000F301A080B18088248394C12C90E2D92E39
:10A9B000E12CF12C58CFA3968FADA3978F7009F49B
:10A9C000BDCC6AEA70E188E290E10F942A28CE01BA
:10A9D0008F599F4F0E94667AAB01BC0188E290E1DB
:10A9E0000E94B6F688E290E10F94BE26CE018F5900
:10A9F0009F4F0E94667A9B01AC0160E476E0C30140
:10AA0000FBCCE9961FAE1EAEE997E3961FAE1EAED5
:10AA1000E397312C212CE7961FAE1EAEE797211449
:10AA2000310409F4CBC1E7968EAD9FADE797B10134
:10AA30000F94DB5C3B016BE970E188E290E10F94DD
:10AA40002A284AE050E0B10188E290E10F94CB2738
:10AA500060E970E188E290E10F942A280FEF10E09E
:10AA6000E7968EAD9FADE797B8010F94DB5C4AE0A7
:10AA700050E088E290E10F94CB2769E870E188E22A
:10AA800090E10F942A284AE050E0B30188E290E177
:10AA90000F94CB276FE770E188E290E10F942A28AA
:10AAA000E9968EAD9FADE997B8010F94DB5C4AE063
:10AAB00050E088E290E10F94CB2768E770E188E2EC
:10AAC00090E10F942A284AE050E0E3966EAD7FAD06
:10AAD000E39788E290E10F94CB2764E770E188E286
:10AAE00090E10F942A2888E290E10F94BE26198203
:10AAF0001A821B821C821D821E821F8218868A81F6
:10AB0000807F8A83B301CE0101960E941379298741
:10AB10003A874B875C876D877E878F87988B67E046
:10AB2000CE0109960E94177879018A011B012C0138
:10AB3000298BFA8A4B8B1C8B6D8B3E8A8F8B588EA0
:10AB40006BE17AE0AD96EEADFFADAD978481958176
:10AB50000E9470F1912C812CB12CA12CD12CC12CF4
:10AB60009101A2016FEF0E948043672809F4E6CBB0
:10AB7000AD96AEADBFADAD971496ED91FC9130970B
:10AB800009F4DCCB66807780E3962EAD3FADE3978A
:10AB9000032E000C440B550BE5962CAF3DAF4EAF8A
:10ABA0005FAFE597E9968EAD9FADE997092E000C52
:10ABB000AA0BBB0BAF968CAF9DAFAEAFBFAFAF973D
:10ABC0006114710409F4BACB2CE330E040E050E0AA
:10ABD00069EB75E0C3010F94A2466B0167E376E071
:10ABE000C3010E9470F1AB969FAF8EAFAB976EEE34
:10ABF00075E0C3010E9470F18C0169EE75E0C3013C
:10AC00000E9470F1AB96AEADBFADAB97109709F453
:10AC1000CDC00115110509F4C9C0009709F4C6C0DB
:10AC200018962C912F70223009F0C0C0F8012085B1
:10AC30002F70223009F0BAC0DC0118962C911897B9
:10AC40002F70223009F0B2C0C114D10409F4AEC093
:10AC500019968D919D910D90BC91A02D82309105FA
:10AC6000A105B10509F4A6C08F3F9F4FAF4FBF4F5D
:10AC700009F4A0C0E9962EAD3FADE997232B09F466
:10AC800099C0D80119968D919C918C9D80018D9DC4
:10AC9000100D9C9D100D11242FEF30E0D8010F9462
:10ACA000065D9601DD0C440B550B0F949A5CE596FE
:10ACB0006CAD7DAD8EAD9FADE5970F94685CAF96A2
:10ACC0002CAD3DAD4EAD5FADAF970F949A5C1901C1
:10ACD0002A016DE670E188E290E10F942A28F301E1
:10ACE0006081718188E290E10F94142867E670E139
:10ACF00088E290E10F942A28C8016FEF70E00F946A
:10AD0000DB5C4AE050E088E290E10F94CB2761E6FB
:10AD100070E188E290E10F942A282AE030E0B20145
:10AD2000A10188E290E10F94832788E290E10F94DB
:10AD3000BE26AB96EEADFFADAB9781859285A38520
:10AD4000B48582159305A405B50581F119861A8687
:10AD50001B861C861D861E861F86188A8A85807F14
:10AD60008A87B101CE0109960E94137929833A831B
:10AD70004B835C836D837E838F839887912C812C9A
:10AD8000B12CA12CD12CC12C79018A019B01AC01E1
:10AD90006FEFC3010E948043AB96AEADBFADAB97E2
:10ADA00019962D923D924D925C921C97F301628010
:10ADB000738006CF212C312C2101BBCF90E080E0A5
:10ADC000BFCAEB962EAD3FADEB9744244394512C74
:10ADD000232B09F098C9B2CAEB964EAD5FADEB9745
:10ADE000452B09F090C9833009F4A3CA20F48130BF
:10ADF00008F489C9A3CA883009F401CB8C3009F45E
:10AE000053CB873009F07FC999CA4F925F926F92F6
:10AE10007F928F929F92AF92BF92CF92DF92EF92EA
:10AE2000FF920F931F93CF93DF93CDB7DEB7689751
:10AE30000FB6F894DEBF0FBECDBF3B016BE17AE0E9
:10AE4000FC01848195810E9470F12C01009709F426
:10AE50007BC020E030E0A90160E077E00F94A246DB
:10AE60008B0120E030E0A9016DE276E0C2010F9491
:10AE7000A2460115110541F00617170709F064C035
:10AE80000615170509F460C019861A861B861C86EC
:10AE90001D861E861F86188A8A85807F8A87662D72
:10AEA000CE0109960E943978298B3A8B4B8B5C8BAB
:10AEB0006D8B7E8B8F8B988F61E0CE0141960E94C7
:10AEC000177829833A834B835C836D837E838F83DA
:10AED0009887912C812CB12CA12CD12CC12C7901DB
:10AEE0008A019B01AC016FEFC2010E94804360E0C8
:10AEF00077E0C2010F944F468C01009711F1FC01DD
:10AF00008085982F9F70923039F0933079F09111AD
:10AF100018C0807F82608087C301770CAA0BBB0BAF
:10AF2000F80181879287A387B4870BC0B301770CA0
:10AF3000880B990B0F94355BF801618772878387C3
:10AF4000948781E090E002C090E080E068960FB6C0
:10AF5000F894DEBF0FBECDBFDF91CF911F910F914F
:10AF6000FF90EF90DF90CF90BF90AF909F908F9029
:10AF70007F906F905F904F9008952F923F924F92E5
:10AF80005F926F927F928F929F92AF92BF92CF9279
:10AF9000DF92EF92FF920F931F93CF93DF93CDB782
:10AFA000DEB7E6970FB6F894DEBF0FBECDBF4C01FB
:10AFB00061307105D9F5DC0112968D919C910E944A
:10AFC000E7B2672B682B692B89F14FEF5FEFBA016E
:10AFD00080E00F9467476B017C01F40102811381CB
:10AFE000C8010E94E7B2C61AD70AE80AF90AF0E6D1
:10AFF000CF16FAEEDF06E104F104C0F040E050E0C5
:10B00000BA01C8010E94A6B26BE17AE0D40114969D
:10B010008D919C910E9470F160E476E00E9470F145
:10B02000009721F0FC012085207F2087D401149611
:10B030000D911C910115110509F4C0C36BE17AE073
:10B04000C8010E9470F13C01009709F4DAC3FC01C9
:10B0500080858F70863009F0D4C360E476E0C30148
:10B060000E9470F1FC01892B09F4CBC390859F707D
:10B07000933009F0C3C3C184D284E384F48420E014
:10B0800030E0A9016DE276E0C3010F94A2467EABE9
:10B090006DAB20E030E040EF51E4C701B6010F9402
:10B0A000365E18160CF43FC120E030E040E751E472
:10B0B000C701B6010F942E5B87FF3AC125E130E04E
:10B0C0003CAB2BABF80166807780B12C1AAA19AA89
:10B0D0006114710409F450C3D301ED91FC913097D0
:10B0E00009F414C18081882309F410C120E030E004
:10B0F000A90169EE75E0C3010F94A2468B0120E01F
:10B1000030E0A90164EE75E0C3010F94A2461B0173
:10B110002C0120E030E0A90160E476E0C3010F9447
:10B12000A2466B017C010F30110509F434C10CF00B
:10B1300004C10230110521F00E30110509F005C1DE
:10B1400065E675E0C3010E9470F16C01009709F497
:10B15000DDC0FC0181859285A385B4850097A1059A
:10B16000B10509F4D3C07C01FC0122AD222309F40E
:10B17000CDC00F94D929882309F4C8C064E476E0CF
:10B18000C3010E9470F12C01009709F4BFC0DC01DB
:10B1900018968C918F70833009F0B8C06AE570E121
:10B1A00088E290E10F942A28D4011296ED91FC9147
:10B1B0000280F381E02D6081718188E290E10F943B
:10B1C00014286EEF78E088E290E10F941428F301E0
:10B1D0006081718188E290E10F94142865E570E147
:10B1E00088E290E10F942A28D7015C96ED91FC91BA
:10B1F000408151816281738188E290E10E94B6F6BC
:10B200006FE470E188E290E10F942A28D7019096CC
:10B21000ED91FC91408151816281738188E290E1DE
:10B220000E94B6F669E470E188E290E10F942A2862
:10B23000D7015E96ED91FC914081518162817381CD
:10B2400088E290E10E94B6F667E177E088E290E15B
:10B250000F941428F701408151816281738188E243
:10B2600090E10E94B6F66BE177E088E290E10F94FE
:10B270001428D70114964D915D916D917C9117978B
:10B2800088E290E10E94B6F66FE177E088E290E113
:10B290000F941428F701408551856285738588E2F3
:10B2A00090E10E94B6F6D70158968D919C916FE07F
:10B2B00077E0892B11F069E077E088E290E10F9464
:10B2C0001428F70182AD65E177E0811102C06BE4DB
:10B2D00079E088E290E10F94142888E290E10F94DD
:10B2E000BE260431110509F443C10531110509F4E5
:10B2F000CEC10E30110551F42BA93CA924313105E2
:10B3000009F44CC02531310509F4C2C0F301628053
:10B310007380DECE61857285838594850F94355B5D
:10B320006B017C01ACCE84E190E09CAB8BABCACED0
:10B33000AFE0B0E0BCABABABC5CE0331110541F023
:10B3400024F0063111050CF4FBCE10E000E0F8CE3D
:10B35000C201B1010F94355B1B012C01C701B6017D
:10B360000F94355B6B017C01AC019B01C201B10103
:10B370000F94365E04E110E0181614F010E000E0BF
:10B38000A7019601C201B1010F942E5B87FFD8CEB1
:10B3900005E110E0D5CEBB24B394D2CE70E060E0DE
:10B3A000D60119968D919C910F943B2B68E370E127
:10B3B00088E290E10F942A28D4011296ED91FC9135
:10B3C0000280F381E02D6081718188E290E10F9429
:10B3D00014286EEF78E088E290E10F941428F301CE
:10B3E0006081718188E290E10F94142867E270E136
:10B3F00088E290E10F942A2888E290E10F94BE261B
:10B400002DA93EA92230310509F480CFD401ED9158
:10B41000FC9120883188F301E080F18019821A8242
:10B420001B821C821D821E821F8218868A81807F59
:10B430008A83D20119966D917D918D919C911C9773
:10B440000F94005ECE0101960E94137929873A87F6
:10B450004B875C876D877E878F87988B67E0CE01EF
:10B4600009960E941778022F242F09A73AA74BA705
:10B470005CA76DA77EA78FA798ABA12CCC24C39403
:10B48000132F352FAB01BC01C401F10119953ECF3B
:10B4900061E070E0D60119968D919C910F943B2B41
:10B4A00066E170E188E290E10F942A28D4011296B7
:10B4B000ED91FC910280F381E02D6081718188E241
:10B4C00090E10F9414286EEF78E088E290E10F94F9
:10B4D0001428F3016081718188E290E10F941428AF
:10B4E00064E070E188E290E10F942A2888E290E11C
:10B4F0000F94BE262DA93EA92230310509F406CFAE
:10B50000D401ED91FC9120883188F301E080F18035
:10B5100019821A821B821C821D821E821F8218863B
:10B520008A81807F8A83D20119966D917D918D9158
:10B530009C911C970F94005ECE0101960E94137996
:10B5400029873A874B875C876D877E878F87988BA3
:10B5500067E0CE0109960E941778022F242F09A3D5
:10B560003AA34BA35CA36DA37EA38FA398A785CF1B
:10B5700070E060E0D60119968D919C910F943B2B61
:10B5800068EF7FE088E290E10F942A28D4011296B8
:10B59000ED91FC910280F381E02D6081718188E260
:10B5A00090E10F9414286EEF78E088E290E10F9418
:10B5B0001428F3016081718188E290E10F941428CE
:10B5C00067EE7FE088E290E10F942A2888E290E11C
:10B5D0000F94BE262DA93EA92431310509F041C0A2
:10B5E000D401ED91FC9120883188F301E080F18055
:10B5F00019821A821B821C821D821E821F8218865B
:10B600008A81807F8A83D20119966D917D918D9177
:10B610009C911C970F94005ECE0101960E941379B5
:10B6200029873A874B875C876D877E878F87988BC2
:10B6300067E0CE0109960E941778022F242F098F08
:10B640003A8F4B8F5C8F6D8F7E8F8F8F98A3A12C3D
:10B65000CC24C394132F352FAB01BC01C401F101DD
:10B66000199529A93AA9B901330F880B990B0F94A1
:10B67000355BD20119962D913D914D915C911C97AE
:10B680000F94225D0F94005E7AAB69AB3FCE61E010
:10B6900070E0F601818592850F943B2B6BED7FE086
:10B6A00088E290E10F942A28D4011296ED91FC9142
:10B6B0000280F381E02D6081718188E290E10F9436
:10B6C00014286EEF78E088E290E10F941428F301DB
:10B6D0006081718188E290E10F94142869EC7FE029
:10B6E00088E290E10F942A2888E290E10F94BE2628
:10B6F0002DA93EA92531310569F519821A821B82CF
:10B700001C821D821E821F8218868A81807F8A8306
:10B71000D20119966D917D918D919C911C970F94FA
:10B72000005ECE0101960E94137929873A874B87E4
:10B730005C876D877E878F87988B67E0CE0109963F
:10B740000E941778298B3A8B4B8B5C8B6D8B7E8B91
:10B750008F8B988FE9A9FAA9BF01FF0F880B990B6E
:10B760000F94355BD20119962D913D914D915C91CD
:10B770001C970F94215D86CF29A93AA9232BC9F1E3
:10B7800065EB7FE088E290E10F942A284AE050E0E0
:10B7900069A97AA988E290E10F94CB2788E290E129
:10B7A0000F94BE2689A99AA964E170E018161906BB
:10B7B00014F065E170E0C4010E94055781E090E05B
:10B7C000E6960FB6F894DEBF0FBECDBFDF91CF91E6
:10B7D0001F910F91FF90EF90DF90CF90BF90AF90AF
:10B7E0009F908F907F906F905F904F903F902F90A1
:10B7F0000895BB2019F36FE070E0DDCF923009F4BB
:10B8000089CDC12CD12C80ECE82E8FE7F82E37CCD7
:10B810002F923F924F925F926F927F928F929F9260
:10B82000AF92BF92CF92DF92EF92FF920F931F934E
:10B83000CF93DF93CDB7DEB7CF58D1090FB6F894C9
:10B84000DEBF0FBECDBF3C011A01CD57DF4F2883AD
:10B85000C358D040C457DF4F19830883CC58D04019
:10B86000C257DF4FF982E882CE58D040C957DF4F28
:10B87000C882C758D040CB57DF4FB982A882C5587D
:10B88000D040DC011496ED91FC910288F389E02D03
:10B8900086809780AB2849F4FE01EE57FF4FCB57C7
:10B8A000DF4FF983E883C558D04081E0CB57DF4FA5
:10B8B000A881B981C558D0408C936B01F12CE12C43
:10B8C0008114910409F4F6C5CD57DF4FB881C358F0
:10B8D000D040B13009F488C008F47FC0B23041F0E4
:10B8E000B33009F477C0D40112968D909C90E8CFC4
:10B8F00067E976E0C4010E9470F111E0009799F3C6
:10B90000FC0181859285A385B4858C159D05AE05C6
:10B91000BF0549F766E675E0C4010E9470F1C8579B
:10B92000DF4F99838883C858D040D3011296ED9198
:10B93000FC9162E0848195810E9422F2C657DF4F1C
:10B9400099838883CA58D040822D0E94D9FE7C01F9
:10B95000CF57DF4F1882C158D04019AA1AAA1BAA84
:10B960001CAA1DAA1EAA1FAA18AE8AA9807F8AAB8C
:10B970006FEA75E0C4010E9470F16C0164EB75E040
:10B98000C4010E9470F15C01C114D10451F0F601B0
:10B9900080858F70843029F4818592850E9492235E
:10B9A000182FEFEFE10FEB3008F09DC10E2E000CC9
:10B9B000FF0B8827E152F34A8F4F0D94EF5CF75C41
:10B9C000855D635DAA5D735E735EF25DCF5D165E3D
:10B9D000275E3F5E63E277E08DCF66E277E0C401E9
:10B9E0000E9470F11BE08ACF6BE277E0F8CF17017D
:10B9F000512C412CA701FF0C660B770BCE01C19691
:10BA00000E945B78EA962FAFEA97EB963FAFEB97F1
:10BA1000EC964FAFEC97ED965FAFED97EE966FAF6C
:10BA2000EE97EF967FAFEF97C158DF4F8883CF57E0
:10BA3000D040C058DF4F9883C058D0408091450215
:10BA4000893020F4809144028930B8F16CE87DE0BF
:10BA500088E290E10F942A2800E020E030E340E102
:10BA600050E0BE016F5F7F4FCE01C1960E945C7BAC
:10BA7000BC0188E290E10F94142860E87DE088E240
:10BA800090E10F942A28612F110F770B4AE050E0C4
:10BA900088E290E10F94CB276EE77DE088E290E1A9
:10BAA0000F942A28D4016D917C9188E290E10F9443
:10BAB000142888E290E10F94BE26A114B10409F085
:10BAC00016C1D12C71C31701512C412CB201A70111
:10BAD000CE01C1960E945B78E2962FAFE297E39683
:10BAE0003FAFE397E4964FAFE497E5965FAFE597F6
:10BAF000E6966FAFE697E7967FAFE797E8968FAF4A
:10BB0000E897E9969FAFE99799CFFE24EF24FE24AA
:10BB10001701512C412CB201A101CE01C1960E9406
:10BB20005B78AA962FAFAA97AB963FAFAB97AC9630
:10BB30004FAFAC97AD965FAFAD97AE966FAFAE9788
:10BB4000AF967FAFAF97E0968FAFE097E1969FAF4C
:10BB5000E19774CFFE24EF24FE241701512C412CD1
:10BB6000B201A101CE01C1960E945B78A2962FAFCF
:10BB7000A297A3963FAFA397A4964FAFA497A5967D
:10BB80005FAFA597A6966FAFA697A7967FAFA7972B
:10BB9000A8968FAFA897A9969FAFA9974FCFFF24DC
:10BBA0001701512C412CB201A701CE01C1960E9470
:10BBB0005B786A962FAF6A976B963FAF6B976C96E0
:10BBC0004FAF6C976D965FAF6D976E966FAF6E9738
:10BBD0006F967FAF6F97A0968FAFA097A1969FAFFC
:10BBE000A1972CCFEF2CFF241701512C412CB2012F
:10BBF000A701CE01C1960E945B7862962FAF629733
:10BC000063963FAF639764964FAF649765965FAF57
:10BC1000659766966FAF669767967FAF67976896EA
:10BC20008FAF689769969FAF699708CF1701512C1E
:10BC3000412C8AA9807F86608AAB2AE030E0D70158
:10BC40000F94065D6DAB7EAB8FAB98AFF7CE17014F
:10BC5000512C412C8AA9807F87608AABB701FF0CE9
:10BC6000880B990B0F94355B20E030E048EC52E4F0
:10BC70000F948E5D6DAB7EAB8FAB98AFDFCEC10105
:10BC800024E0969587952A95E1F70E94D9FEFFE07A
:10BC90002F22332402C0969587952A94E2F781706B
:10BCA00099271C01512C412CB201AC01CE01C19647
:10BCB0000E945B782A962FAF2A972B963FAF2B973F
:10BCC0002C964FAF2C972D965FAF2D972E966FAF7A
:10BCD0002E972F967FAF2F9760968FAF60976196C4
:10BCE0009FAF6197ABCE212C312C2101A7CEF5015E
:10BCF00080858F708550823008F0E3CEB501CE018B
:10BD0000C1960E94997E29A33AA34BA35CA36DA37D
:10BD10007EA38FA398A788E0FE01B196DE019996D5
:10BD200001900D928A95E1F788E0FE01B996DE0157
:10BD3000D19601900D928A95E1F789A9811103C0EE
:10BD40008AA98F7009F180914502893008F4B9C23F
:10BD500069EF7CE088E290E10F942A2800E020E07F
:10BD600030E340E150E0BE016F5F7F4FCE01C196EE
:10BD70000E945C7BBC0188E290E10F94142888E269
:10BD800090E10F94BE269DCE63E976E0C5010E9446
:10BD900070F17C01009709F494CEDC0118968C9127
:10BDA0008F70823009F41DC1843009F08ACE8091F1
:10BDB0004502893020F480914402893090F06FE28E
:10BDC0007DE088E290E10F942A28D70119966D91C1
:10BDD0007C9188E290E10F94142888E290E10F941E
:10BDE000BE26C657DF4FE881F981CA58D040309748
:10BDF00009F471C380858F70863009F06AC3D7015A
:10BE00001996CD90DC90C114D10409F462C3D3011A
:10BE10001296ED91FC9162E0848195810E9422F25C
:10BE2000B6010E9470F10F94CA016C01892B09F4CC
:10BE300050C380914502893020F4809144028930BA
:10BE4000A8F06DE17DE088E290E10F942A28F601E8
:10BE500041855285638574852AE030E088E290E16F
:10BE60000F94832788E290E10F94BE26D70119969C
:10BE70006D917C91D3011496ED91FC918289938907
:10BE80000E9470F17C01009709F423C36FEA75E00A
:10BE90000E9470F1009749F0FC0120852F7024303A
:10BEA00021F4818592850E949223D60119964D91A5
:10BEB0005D916D917C911C97CE01C1960E945B783B
:10BEC00022962FAF229723963FAF239724964FAF0A
:10BED000249725965FAF259726966FAF26972796CE
:10BEE0007FAF279728968FAF289729969FAF2997DE
:10BEF00064EB75E0C7010E9470F1BC01009721F16D
:10BF0000FC0190859F7095509230F0F4CE01C1965F
:10BF10000E94997E298B3A8B4B8B5C8B6D8B7E8B31
:10BF20008F8B988F88E0FE017196DE015996019003
:10BF30000D928A95E1F788E0FE017996DE01D196AF
:10BF400001900D928A95E1F780914502893020F4A5
:10BF5000809144028930D8F068E07DE088E290E189
:10BF60000F942A2800E020E030E340E150E0BE01D9
:10BF70006F5F7F4FCE01C1960E945C7BBC0188E25F
:10BF800090E10F94142888E290E10F94BE26D60128
:10BF900018968C911897982F92959F7090FD99C242
:10BFA00021E0CF57DF4F2883C158D0409160929550
:10BFB000907F8F70892B18968C93DD24D394C9576A
:10BFC000DF4FB881C758D040BB2309F406C1C8571A
:10BFD000DF4F48815981C858D040452B09F4FDC036
:10BFE0008CC280914502893020F4809144028930CE
:10BFF000A8F068E67DE088E290E10F942A28F70136
:10C0000041855285638574852AE030E088E290E1BD
:10C010000F94832788E290E10F94BE26D7011996EA
:10C020006D917D918D919C911C97C457DF4FE88154
:10C03000F981CC58D0408F0130E020E060177107C3
:10C04000820793070CF455C0C257DF4F48815981CE
:10C05000CE58D0408A0130E020E0061717072807A5
:10C0600039070CF446C0AB014E1B5F0BDE01AF5726
:10C07000BF4F5D01C12CC257DF4FE880F980CE5819
:10C08000D0408F01CD57DF4F2881C358D040C30126
:10C090000E94085C29AB3AAB4BAB5CAB6DAB7EABA3
:10C0A0008FAB98AF80914502893020F48091440293
:10C0B0008930E0F06FE277E088E290E10F94142895
:10C0C0006CE477E088E290E10F941428CF57DF4FBB
:10C0D0006881C158D04070E04AE050E088E290E1C9
:10C0E0000F94CB2788E290E10F94BE26DD24D394F1
:10C0F0005BC06EE57DE088E290E10F942A28F701AD
:10C1000041855285638574852AE030E088E290E1BC
:10C110000F9483276FE37DE088E290E10F942A2853
:10C1200088E290E10F94BE2681E08093CA0DCE0193
:10C1300041969093500E80934F0ECD57DF4FF8816C
:10C14000C358D0406F2F70E041E050E0D7011996FE
:10C150008D919C910E94EF2DD82E8823E1F0F7015C
:10C16000618572859E012F573F4F5901C12C7B017C
:10C170008B01CD57DF4F2881C358D04050E040E0BD
:10C18000C3010E94085C29AB3AAB4BAB5CAB6DAB17
:10C190007EAB8FAB98AF80E48093CA0D8FEC9DE0AF
:10C1A0009093500E80934F0EC957DF4FB881C758F8
:10C1B000D040BB2349F0C857DF4FE881F981C85808
:10C1C000D040EF2B09F099C1C657DF4FE881F981C4
:10C1D000CA58D040EF2B09F447C0C657DF4FA8819B
:10C1E000B981CA58D04018968C9118978F708630B4
:10C1F000D9F5F40160817181CD010E9470F13C019B
:10C20000009791F10F94CA017C01009709F4D6C000
:10C21000FC0181859285A385B48582159305A405CB
:10C22000B50509F09CC0C957DF4FF881C758D04009
:10C23000F11157C0D70118968C91189782958F707D
:10C2400080FD4FC091E0CB57DF4FE881F981C558A1
:10C25000D040908381608295807F18969C9118973A
:10C260009F70892B18968C9388E0FE01F196DE0171
:10C27000D99601900D928A95E1F729AD3AAD4BAD73
:10C280005CAD6DAD7EAD8FAD21969FAD2197C15751
:10C29000DF4F0FB6F894DEBF0FBECDBFDF91CF9159
:10C2A0001F910F91FF90EF90DF90CF90BF90AF90D4
:10C2B0009F908F907F906F905F904F903F902F90C6
:10C2C000089580914402893008F4FBCB41CDF301FD
:10C2D0006281738140E050E1CE01C1960E94717786
:10C2E00073CFCB57DF4FA881B981C558D0401C927E
:10C2F000DD2009F4B9CFC957DF4FB881C758D04006
:10C30000BB2309F4B1CFCF57DF4F8881C158D0404C
:10C3100081110AC0CB57DF4FA881B981C558D040E1
:10C320008C91882309F4A0CF912C812CB12CA12CC5
:10C33000D12CC12CE9A8FAA80BA91CA92DA93EA9AA
:10C340004FA958AD6FEFC3010E94804381E0CB57E6
:10C35000DF4FE881F981C558D040808385CF2186A1
:10C3600032864386548680914502893020F480913C
:10C3700044028930F8F061E577E088E290E10F94BB
:10C3800014282AE030E0B201A10188E290E10F9484
:10C39000D9266FE577E088E290E10F941428D40164
:10C3A0006D917C9188E290E10F94142888E290E1ED
:10C3B0000F94BE26F70180858F7E8087D1109BCF9A
:10C3C000CB57DF4FA881B981C558D0408C918823C5
:10C3D00009F44ACFC957DF4FB881C758D040BB23B3
:10C3E00009F442CFF30180858F708530D1F58681C5
:10C3F000978168EB75E00E9470F1CD57DF4F99830C
:10C400008883C358D040009771F1DC0118968C9155
:10C4100018978F70823039F519968D919D910D90F6
:10C42000BC91A02D82159305A405B505E1F480917A
:10C430004502893020F480914402893050F062ED49
:10C440007CE088E290E10F942A2888E290E10F9442
:10C45000BE26CB57DF4FE881F981C558D040108206
:10C4600003CFC301C6CF912C812CB12CA12CD12C90
:10C47000C12CE9A8FAA80BA91CA92DA93EA94FA96E
:10C4800058AD6FEFC3010E948043CD57DF4F288125
:10C490003981C358D0402115310509F4E5CED301C7
:10C4A00018968C9187FDE0CEF9012186328643866D
:10C4B0005486DACE19821A821B821C828A81807F7E
:10C4C0008A831D821E821F82188688E0FE013196B3
:10C4D000CECED12C74CDC957DF4FE881C758D0409C
:10C4E000EE2309F4C1CEC857DF4F28813981C858DF
:10C4F000D040D12C232B09F4B7CEC857DF4FA881E9
:10C50000B981C858D04018968C9118978F70823096
:10C5100009F05ACE19968D919D910D90BC91A02D48
:10C5200081309105A105B10509F4D1CE0297A1058D
:10C53000B10509F049CED30112966D917C9140E08E
:10C5400050E2CACE2F923F924F925F926F927F92AB
:10C550008F929F92AF92BF92CF92DF92EF92FF9213
:10C560000F931F93CF93DF93CDB7DEB768970FB6C6
:10C57000F894DEBF0FBECDBF6115710509F491C0FF
:10C580005E8B498B9D8B8C8BFB0186809780811401
:10C59000910409F486C0F40180858F70823031F0F7
:10C5A000853031F1F40182809380F1CF618472840F
:10C5B00041E050E069897E89C3010E94EF2D882304
:10C5C00089F3B12CA12CCC24C39473018301298954
:10C5D00050E040E0B3018C899D890E94085C298766
:10C5E0003A874B875C876D877E878F87988BDACFFA
:10C5F000C4010E94B3F28230A9F660E0C4010E9437
:10C6000022F2FC01C184D284E384F48461E0C40199
:10C610000E9422F2FC012184328443845484388EA7
:10C620002F8ADB8ACA8AA1014C195D094F5F5F4FCF
:10C6300069897E89C6010E94EF2D882309F4B2CF53
:10C6400080914502893020F480914402893020F0A5
:10C6500088E290E10F94BE26712C612C6A897B8957
:10C66000660D771D8F89988D861797070CF49ACFE2
:10C67000B12CA12CCC24C39471010A891B8929896E
:10C68000A3018C899D890E94085C29833A834B838E
:10C690005C836D837E838F8398879FEF691A790A05
:10C6A000DDCF68960FB6F894DEBF0FBECDBFDF9129
:10C6B000CF911F910F91FF90EF90DF90CF90BF909F
:10C6C000AF909F908F907F906F905F904F903F9032
:10C6D0002F9008952F923F924F925F926F927F9288
:10C6E0008F929F92AF92BF92CF92DF92EF92FF9282
:10C6F0000F931F93CF93DF9300D01F921F92CDB75C
:10C70000DEB761307105D1F490E080E00F900F90BA
:10C710000F900F900F90DF91CF911F910F91FF908D
:10C72000EF90DF90CF90BF90AF909F908F907F90D1
:10C730006F905F904F903F902F90089520916F0AD7
:10C740003091700A232B01F78C01DC01ED91FC91F3
:10C750000284F385E02D19950297B1F68091760A4F
:10C760009091770AA091780AB091790A892B8A2B47
:10C770008B2B79F4D8011296ED91FC9162E08481C3
:10C7800095810E9422F29C838B83892BB1F4B12C7A
:10C790000BC40F94AD06C090760AD090770AE09053
:10C7A000780AF090790A6C197D098E099F09683C16
:10C7B000710581059105F0F6A7CFEB81FC8180859D
:10C7C0008F70863021F7C680D7801D82B12CC114AE
:10C7D000D10409F4E5C3D60118968C91982F9F7067
:10C7E0002BEF290F223008F0DBC3BD81B111D8C374
:10C7F000282F22952F7087FF7AC522FD78C59530A6
:10C8000009F0A7C0F6018681978168EB75E00E9468
:10C8100070F11C01892B09F46AC581E090E09093C6
:10C82000700A80936F0AB11003C0C8010E946F2E76
:10C83000D10119964D905C906AE677E088E290E12C
:10C840000F941428D8011296ED91FC910280F38187
:10C85000E02D6081718188E290E10F9414286EEFE1
:10C8600078E088E290E10F941428F60160817181EC
:10C8700088E290E10F9414286DE476E088E290E17C
:10C880000F941428D10119964D915D916D917C9171
:10C890001C972AE030E088E290E10F94832788E239
:10C8A00090E10F94BE26F60180809180D801149605
:10C8B000ED91FC9161E77EE0309759F0B4018289F7
:10C8C00093890E9470F17C01009709F044C06EE4E6
:10C8D0007EE081E89FE00F942A2881E89FE00F9492
:10C8E000BE26EE24EA94FE2C4201550CAA08BB0891
:10C8F000D10119964D905D906D907C901C97841499
:10C900009504A604B70409F4A7C48091760A90910F
:10C91000770AA091780AB091790A892B8A2B8B2B00
:10C9200009F486CF0F94AD062091760A3091770AEC
:10C930004091780A5091790A621B730B840B950B16
:10C94000683C71058105910508F072CF0E942DA702
:10C95000D6CFC6015ACF67E976E00E9470F13C015C
:10C96000892B79F466E277E0C7010E9470F13C01FF
:10C970006BE27EE0892B69F0F10180858F70806B1E
:10C980008087D30118968C918F70823079F065E1A1
:10C990007EE081E89FE00F942A2881E89FE00F94D1
:10C9A000BE26EEEFEE2EFF24FA949ECF6AE876E0E4
:10C9B000C7010E9470F17C01009709F442C1FC019B
:10C9C00080858F70813009F061C18185882309F4E9
:10C9D0005DC1D10118968C91807FF12CE12C803BB8
:10C9E00019F072E0E72EF12C6AE07EE088E290E137
:10C9F0000F942A28B40188E290E10F94142867E08C
:10CA00007EE088E290E10F942A28F3014185528567
:10CA1000638574852AE030E088E290E10F948327F3
:10CA200066E777E088E290E10F9414284AE050E04E
:10CA3000B70188E290E10F94CB276CEC75E088E2B7
:10CA400090E10F941428F1E0F093CA0D81E090E09A
:10CA50008C0F9D1F9093500E80934F0E41E050E03D
:10CA6000B701D30119968D919C910E94EF2DF82E5C
:10CA70004FEF5FEFBA0180E00F9467476093760A4B
:10CA80007093770A8093780A9093790AFF2009F4CB
:10CA9000FAC0D8011296ED91FC9162E084819581F3
:10CAA0000E9422F27C01009709F4C2C0FC0180853B
:10CAB0008F70863009F0E7C0B401C7010E9470F1A1
:10CAC0007C01009709F4B4C00F94CA017C01892B42
:10CAD00009F4AEC080914502893020F4809144026F
:10CAE000893028F160E07EE088E290E10F942A2806
:10CAF000D70119964D915D916D917C911C972AE01B
:10CB000030E088E290E10F9483276AEF7DE088E2CD
:10CB100090E10F942A2869817A814AE050E088E206
:10CB200090E10F94DB2688E290E10F94BE26F70196
:10CB3000418552856385748589819A81B0E0A0E042
:10CB4000481759076A077B0719F164EF7DE088E20F
:10CB500090E10F942A28B40188E290E10F94142800
:10CB600066EE7DE088E290E10F942A2888E290E169
:10CB70000F94BE26F0E4F093CA0D8FEC9DE09093E5
:10CB8000500E80934F0E6DEFE62EFF24FA94ACCE3C
:10CB9000F10181859285A385B485481759076A07F5
:10CBA0007B0789F560EE7DE088E290E10F942A280A
:10CBB000B40188E290E10F9414286EED7DE088E2E4
:10CBC00090E10F942A2869817A814AE050E088E256
:10CBD00090E10F94DB266DEC7DE088E290E10F940C
:10CBE0002A2888E290E10F94BE26F0E4F093CA0D63
:10CBF0008FEC9DE09093500E80934F0E5CEFE52EEE
:10CC0000FF24FA9471CE67EC7DE088E290E10F9406
:10CC10002A28B40188E290E10F9414286CEA7DE0A0
:10CC200088E290E10F942A2888E290E10F94BE26D2
:10CC300090E49093CA0DAFECBDE0B093500EA0937A
:10CC40004F0ED1011896EC91E295EF70E150AA24B5
:10CC5000AA94BA2CEB3008F066C0F0E0D301199624
:10CC60002D913C918827E85CF9498F4F0D94EF5C3A
:10CC700049665E6649665E6608670367086703671C
:10CC8000496649661467F12CE12CD2CFF12CE12CD6
:10CC9000D8CFF101818592853093520E2093510EA9
:10CCA0001092540E1092530E9093560E8093550E80
:10CCB00086E00F943C08A82EB12C35C0D1011996FE
:10CCC0008D919C919827892798273093520E209315
:10CCD000510E1092540E1092530E9093560E809354
:10CCE000550E86E00F943C08A82EB12CF1018185E9
:10CCF0009285A385B4853A2F2B2FD30119968D9158
:10CD00009C9101969093520E8093510E1092540E66
:10CD10001092530E3093560E2093550E86E00F94CA
:10CD20003C08A80EB11C4FEF5FEFBA0180E00F94F2
:10CD300067476093760A7093770A8093780A909396
:10CD4000790A61EA7DE088E290E10F942A284AE0BE
:10CD500050E0B50188E290E10F94CB276FE97DE0C8
:10CD600088E290E10F942A28B40188E290E10F94C0
:10CD700014286DE777E088E290E10F941428F3011E
:10CD800041855285638574852AE030E088E290E130
:10CD90000F94832769E97DE088E290E10F942A28C7
:10CDA000D10119964D915D916D917C911C972AE06E
:10CDB00030E088E290E10F94832788E290E10F94BD
:10CDC000BE26A114B104B9F4F10180858F708230C0
:10CDD00091F4E114F10479F0D70118968C918F70D9
:10CDE000823049F481859285A385B485F7018187D6
:10CDF0009287A387B48791E080E0AB2809F090E0A8
:10CE0000E92EF82E71CDF10181859285992744CFC5
:10CE1000F10181859285A385B485892F9A2FAB2F47
:10CE2000BB27A7FDBA95F2CFD10119968C9130930B
:10CE3000520E2093510E882341F080E09FEF909393
:10CE4000540E8093530E85E034CF90E080E0F7CF0E
:10CE5000D60118968C911897806418968C936EEF73
:10CE60007EE081E89FE00F942A28D8011296ED9188
:10CE7000FC910280F381E02D6081718181E89FE067
:10CE80000F9414286EEF78E081E89FE00F94142847
:10CE9000F6016081718181E89FE00F94142860EFB2
:10CEA0007EE081E89FE00F942A28D60118968C91A5
:10CEB0001897982F92959F70292F2370233039F05F
:10CEC0009F5F9295907F8F70892B18968C9368EE58
:10CED0007EE081E89FE00F942A28D8011296ED9118
:10CEE000FC910280F381E02D6081718181E89FE0F7
:10CEF0000F9414286EEF78E081E89FE00F941428D7
:10CF0000F6016081718181E89FE00F94142863E845
:10CF100077E081E89FE00F941428D60118966C9171
:10CF20006295637070E04AE050E081E89FE00F9402
:10CF3000CB2781E89FE00F94BE26D7C16AED7EE043
:10CF400081E89FE00F942A28D8011296ED91FC9178
:10CF50000280F381E02D6081718181E89FE00F9470
:10CF600014286EEF78E081E89FE00F941428F60112
:10CF70006081718181E89FE00F94142867EC7EE066
:10CF800081E89FE00F942A2881E89FE00F94BE2655
:10CF9000D60118968C9118978F7018968C93A5C10E
:10CFA0001092700A10926F0AD8011496ED91FC91BC
:10CFB000C480D580F12CE12C0F94AD06C114D104AE
:10CFC000E104F10491F0D8011496ED91FC914680B2
:10CFD00057806084718464197509860997096C15F6
:10CFE0007D058E059F0508F4C3C08091760A909157
:10CFF000770AA091780AB091790A892B8A2B8B2B1A
:10D0000009F0A2C0EB81FC81EF2B09F0B8C0D80178
:10D010001496ED91FC9182859385892B69F4848522
:10D020009585892B49F486859785892B29F48089F4
:10D030009189892B09F4FFC080914502893020F441
:10D04000809144028930B8F061EA7EE088E290E1A4
:10D050000F942A28D8011296ED91FC910280F38159
:10D06000E02D6081718188E290E10F94142888E2BC
:10D0700090E10F94BE2681E090E09093700A809337
:10D080006F0AB11003C0C8010E946F2ED801149618
:10D09000ED91FC916285738542E050E0C8010E94E9
:10D0A000A262D8011496ED91FC916485758543E0E8
:10D0B00050E0C8010E94A262D8011496ED91FC9143
:10D0C0006685778550E040E0C8010E94A262D801E1
:10D0D0001496ED91FC916089718941E050E0C8019E
:10D0E0000E94A26280914502893020F4809144021E
:10D0F0008930B8F061E97EE088E290E10F942A2857
:10D10000D8011296ED91FC910280F381E02D6081AF
:10D11000718188E290E10F94142888E290E10F94E5
:10D12000BE260F94AD066B017C010F94AD066C1901
:10D130007D098E099F09623371058105910508F00B
:10D1400076C00E942DA7F1CF0F94AD06C090760A4D
:10D15000D090770AE090780AF090790A6C197D09EE
:10D160008E099F09683C71058105910508F04ACF39
:10D17000D8011496ED91FC9184819581C7CAAB8149
:10D18000BC8118968C9118978F70863009F03FCF2C
:10D190001696ED90FC90E114F10409F438CFF701F4
:10D1A0008085982F9F702BEF290F223008F02FCF0A
:10D1B00082958F7082FF05C08B708295807F892B4E
:10D1C0008087D70118968C9182958370833059F5AA
:10D1D0006EE877E081E89FE00F941428D80112965A
:10D1E000ED91FC910280F381E02D6081718181E8F5
:10D1F0009FE00F9414286EEF78E081E89FE00F9491
:10D200001428F7016081718181E89FE00F94142850
:10D2100081E89FE00F94BE26D70118968C9118974D
:10D220008F7018968C93F701E280F380B4CF109240
:10D23000700A10926F0AF801E480F5804FEF5FEFFB
:10D24000BA0180E00F946747D70116966D937D93DE
:10D250008D939C9319978CCFBDEFEB16BFEFFB0618
:10D2600009F46CCEACF5FCEFEF16FFEFFF06B9F159
:10D2700069EB7EE081E89FE00F942A28D80112969E
:10D28000ED91FC910280F381E02D6081718181E854
:10D290009FE00F9414286EEF78E081E89FE00F94F0
:10D2A0001428F6016081718181E89FE00F941428B1
:10D2B0006EEA7EE081E89FE00F942A2881E89FE0F3
:10D2C0000F94BE26D60118968C9118978F7765CE4D
:10D2D000E114F10409F4BCCDEA94EF2849F6F60113
:10D2E00080858F708087F1E0FD83BB24B394F601C5
:10D2F000C280D3806CCA0F931F93CF93DF93EC014E
:10D300000E947E3C61EA77E088E290E10F94C226B9
:10D3100080917A0A90917B0A892B19F586E190E039
:10D320000F9400538C012B853C854A85042E000CFC
:10D33000550B688579850F94792D10937B0A00939E
:10D340007A0AF8018681978197FD1AC061E00F94EF
:10D35000760260E0F80186810F94480281E0F801CE
:10D360008183E881F9810484F585E02D62E0CE01B6
:10D37000199581E090E0DF91CF911F910F91089571
:10D380001182EFCF8FE090E090932A0C8093290CCC
:10D3900088EC90E00895FC018481958108956BEDFF
:10D3A00073E2811102C06DED73E287E79FE00D9497
:10D3B0002A2863E77FE187E79FE00F942A28F0E0BF
:10D3C000E0E0199584EF91E008958091520B882355
:10D3D000B1F0E091530BF091540B309731F086810E
:10D3E00097819093510B8093500B68EC7CE187E719
:10D3F0009FE00F942A2887E79FE00D94BE260895AA
:10D40000CF93C1E068EE73E080E090E00F94BB043E
:10D410004AE050E06C2F87E79FE00F94E126CF5F52
:10D42000C43181F784EF91E0CF9108952F923F921C
:10D430004F925F926F927F928F929F92AF92BF9224
:10D44000CF92DF92EF92FF920F931F93CF93DF93D0
:10D45000CDB7DEB768970FB6F894DEBF0FBECDBF6D
:10D460003C018091630B60E079E2882309F46AC192
:10D4700061E070E080E090E00F94BB04BE016F5F5C
:10D480007F4F80E00E948AFD892B09F059C1898174
:10D4900083FF56C144E0BE016F5F7F4F82E00E9470
:10D4A00084FE009791F429813A813227232732277D
:10D4B0003093940D2093930D2B813C8132272327A9
:10D4C00032273093920D2093910D0E9457FD6FEDFE
:10D4D00078E288E290E10F942A286091930D709190
:10D4E000940D90E080E00F94335B562E798B8A8BFD
:10D4F000492E462F572F682F792F88E290E10E94FE
:10D50000B6F667ED78E288E290E10F942A28609100
:10D51000910D7091920D90E080E00F94335B6B8BD6
:10D520007C8B8D8B9E8BAB01BC0188E290E10E94CD
:10D53000B6F66BEC78E288E290E10F942A2842E09C
:10D54000BE016F5F7F4F81E10E9484FE49815A8155
:10D55000542745275427892B11F050E040E070E014
:10D5600060E040935F0B5093600B6093610B70938E
:10D57000620B2AE030E088E290E10F94832720E0FC
:10D5800030E44CE156E4652D79898A89942D0F9415
:10D590002E5B87FF7AC0D3011296ED91FC9120801B
:10D5A00031806EEA77E0C1010E9470F1988F8F8B15
:10D5B00062EB77E0C1010E9470F11C0119821A82AE
:10D5C0001B821C828A81807F8760F82E8A83252DAA
:10D5D000852D9989AA89B42D8D839E83AF83B887C1
:10D5E000912C812CB12CA12CD12CC12CE9800B8148
:10D5F0001C813E814F8158856FEF8F89988D0E94E5
:10D60000804319821A821B821C828A81807F8760F4
:10D61000F82E8A832B89822F9C89AD89BE898D83C0
:10D620009E83AF83B887E9800B811C813E814F8147
:10D6300058856FEFC1010E94804327EB37E0452DED
:10D6400059896A89742DC3010E944BEB2CEB37E09A
:10D650004B895C896D897E89C3010E944BEB609187
:10D660005F0B7091600B8091610B9091620B2AE0CF
:10D67000AE014F5F5F4F0F94DD5542EC57E0BE01A6
:10D680006F5F7F4FC3010E9421EB68EC77E088E277
:10D6900090E10F94C226BE016F5F7F4F80EE0E9423
:10D6A0008AFD892B19F419811F3F49F462EA78E257
:10D6B00081E89FE00F944E2881E090E04DC0112357
:10D6C00031F063E978E281E89FE00F942A2815FFA2
:10D6D00006C066E878E281E89FE00F942A2814FFEC
:10D6E00006C06AE778E281E89FE00F942A2813FFDA
:10D6F00006C06CE678E281E89FE00F942A2812FFCA
:10D7000006C06CE578E281E89FE00F942A2811FFBB
:10D7100006C06DE478E281E89FE00F942A2810FFAC
:10D720000BC062E478E281E89FE00F942A2881E848
:10D730009FE00F94BE26C0CF112309F4BDCFF7CFD1
:10D7400065EE78E288E290E10F942A2888E290E181
:10D750000F94BE2690E080E068960FB6F894DEBF86
:10D760000FBECDBFDF91CF911F910F91FF90EF9032
:10D77000DF90CF90BF90AF909F908F907F906F90F1
:10D780005F904F903F902F9008952F923F924F922D
:10D790005F926F927F928F929F92AF92BF92CF9241
:10D7A000DF92EF92FF920F931F93CF93DF93CDB74A
:10D7B000DEB760970FB6F894DEBF0FBECDBF613005
:10D7C000710579F42C0180915E0B811125C069E20D
:10D7D00078E281E89FE00F942A2881E89FE00F9487
:10D7E000BE2690E080E060960FB6F894DEBF0FBED4
:10D7F000CDBFDF91CF911F910F91FF90EF90DF9000
:10D80000CF90BF90AF909F908F907F906F905F90E0
:10D810004F903F902F90089568E178E288E290E180
:10D820000F942A2882E00F94EE04692E712C40E1B7
:10D8300050E0B30188E290E10F94CB278FEF681698
:10D84000710409F42DC16AEC77E088E290E10F944D
:10D85000142880E00F94EE04BC0190E080E00F9467
:10D86000335B20E030E040E857E30F94945B20E026
:10D8700030E045E253E40F94945B20E030E040E276
:10D8800052E40F94215D762E272E382E692E462FD6
:10D89000572F682F792F88E290E10E94B6F661E158
:10D8A00078E288E290E10F942A2881E00F94EE0458
:10D8B000BC0190E080E00F94335B20E030E040E872
:10D8C00057E30F94945B20E030E048EC52E40F946F
:10D8D000945B69877A878B879C87AB01BC0188E260
:10D8E00090E10E94B6F66EEC77E088E290E10F944A
:10D8F000C226D2011296ED91FC91E080F18067E2A0
:10D9000076E0C7010E9470F19E878D8760ED77E019
:10D91000C7010E9470F1988B8F87272D322D432DE0
:10D92000562D672D722D832D962D0F94965E8111A5
:10D9300040C019821A821B821C828A81807F876084
:10D94000F82E8A83272D872D922DA32DB62D8D831A
:10D950009E83AF83B887912C812CB12CA12CD12C24
:10D96000C12CE9800B811C813E814F8158856FEF6E
:10D970008D859E850E94804319821A821B821C829B
:10D980008A81807F8760F82E8A832985822F9A85F5
:10D99000AB85BC858D839E83AF83B887E9800B817F
:10D9A0001C813E814F8158856FEF8F8598890E9439
:10D9B000804324ED37E0472D522D632D762DC20193
:10D9C0000E944BEB27ED37E049855A856B857C85B6
:10D9D000C2010E944BEB8091630B882309F45DC068
:10D9E00020E030E048EC51EC672D722D832D962D10
:10D9F0000F942E5B87FD51C020E030E048E452E4F4
:10DA0000672D722D832D962D0F94365E18160CF40B
:10DA100044C020E030E048EC52E469857A858B858B
:10DA20009C850F94365E1816C4F120E030E04AE77A
:10DA300054E469857A858B859C850F94945B0F945B
:10DA4000075E66507F4F8F4F9F4F24EFC22EDD241D
:10DA5000D394E12CF12CA70196010F94785C2983D3
:10DA60001A8220E030E04AE754E4672D722D832DBE
:10DA7000962D0F94945B0F94075E6E557D498F4FE2
:10DA80009F4FA70196010F94785C2B831C82BE01E7
:10DA90006F5F7F4F85E00E94DAFD88EE93E0A3CEB2
:10DAA00088E290E10F94BE260F94ED46F6CFEF92F8
:10DAB000FF920F931F93CF93DF93CDB7DEB760979D
:10DAC0000FB6F894DEBF0FBECDBF80915E0B8823EA
:10DAD000C9F06DEA77E288E290E10F942A2888E2A3
:10DAE00090E10F94BE2690E080E060960FB6F89427
:10DAF000DEBF0FBECDBFDF91CF911F910F91FF9081
:10DB0000EF90089561E078E288E290E10F942A288E
:10DB10000E9414FE80E480939D0D0E9414FE10E08C
:10DB20001B7F80919D0D0E9480FD62E08AE79DE051
:10DB30000F94CB21612F8AE79DE00F94CB2160E009
:10DB40008AE79DE00F94CB218AE79DE00F94FD4288
:10DB50006AE070E080E090E00F94BB046EEE77E244
:10DB600088E290E10F942A288EEF0F94EE0440E1B2
:10DB700050E0BC0188E290E10F94DB2660EE77E292
:10DB800088E290E10F942A288FEF0F94EE0440E191
:10DB900050E0BC0188E290E10F94DB2688E290E13E
:10DBA0000F94BE266AEC77E287E79FE00F942A285D
:10DBB0008BEF0F94EE04182F092F8CEF0F94EE04C7
:10DBC000F82EE92E8DEF0F94EE049F938F93EF9232
:10DBD000FF920F931F938AED97E09F938F938E018F
:10DBE0000F5F1F4F1F930F930F94E161B80187E7F9
:10DBF0009FE00F94C22681E080935E0B0FB6F894ED
:10DC0000DEBF0FBECDBF81E090E06FCF0F931F93BB
:10DC1000CF93DF9300D000D01F92CDB7DEB78091B5
:10DC2000630B882369F060E777E281E89FE00F9457
:10DC30002A2881E89FE00F94BE2690E080E0B0C0E3
:10DC400060EA77E287E79FE00F944E280E9414FE77
:10DC50008091640290916502A0916602B091670282
:10DC600089839A83AB83BC838AE79DE09093870D79
:10DC70008093860D1E8280E197E22E812F5F2E8396
:10DC80000197D9F71D82BE016B5F7F4F80E20E9432
:10DC90008AFD8C01892BF1F48D8101E010E081383F
:10DCA000C9F4BE016F5F7F4F8FEF0E94DAFD1F82C4
:10DCB00080E89EE32F812F5F2F830197D9F7BE0164
:10DCC0006B5F7F4F80E00E948AFD8D8180FF0CC0DA
:10DCD00003E010E06CE877E281E89FE00F942A28E7
:10DCE000C8010E9457FDA9CFBE016B5F7F4F80E046
:10DCF0000E948AFD892B61F78D8184FFE9CF809195
:10DD0000880D0E9480FD8091860D9091870DDC0129
:10DD1000ED91FC910190F081E02D64EF19958091D7
:10DD2000860D9091870D0F94FD42882319F002E033
:10DD300010E0D0CFBE016B5F7F4F81E00E948AFD73
:10DD40008C01892B39F61D811F7810611D8380910C
:10DD5000880D0E9480FD8091860D9091870DDC01D9
:10DD6000ED91FC910190F081E02D61E01995809199
:10DD7000860D9091870DDC01ED91FC910190F08171
:10DD8000E02D612F19958091860D9091870D0F944C
:10DD9000FD428111CCCF81E08093630B81E090E064
:10DDA00027960FB6F894DEBF0FBECDBFDF91CF919F
:10DDB0001F910F910895CF93DF9300D000D01F9251
:10DDC0001F92CDB7DEB7E1E6FFE0128A118A80E04C
:10DDD00090E19587848784E890E0948B838B81E041
:10DDE000868787E7858B1C821B8286E193E09A8376
:10DDF0008983FE83ED838FEF9FEF98878F8366E59E
:10DE000077E287E79FE00F942A286091DD0A7091FE
:10DE1000DE0ACE0101960E94E6F881E69FE00E94AC
:10DE2000EDAD66E477E287E79FE00F942A2887E765
:10DE30009FE00F94BE260F94D40F28960FB6F89447
:10DE4000DEBF0FBECDBFDF91CF91089560E08DE0C2
:10DE50000D94480261E08DE00D944802892B71F029
:10DE6000FB01828193810E9442F364EC73E287E7B5
:10DE70009FE00F942A2888EC90E0089590E080E0DD
:10DE8000F2CF0F931F93CF93DF93EB0102970CF424
:10DE90009FC00A811B8169EA72E2C8010F941B5579
:10DEA000892B61F40E94A8F57E7F0E9402F688EC1F
:10DEB00090E0DF91CF911F910F91089563EB72E293
:10DEC000C8010F941B55892B21F40E94A8F571609D
:10DED000ECCF6FE772E287E79FE00F942A280E9459
:10DEE000A8F5672F609561704AE050E070E087E721
:10DEF0009FE00F94CB2787E79FE00F94BE26809189
:10DF0000530F9091540F892B09F452C00A811B8141
:10DF10000E94C3F2882309F44BC0F801019000204D
:10DF2000E9F73197E01BF10BB09708F041C0A091E1
:10DF3000530FB091540F52961C921E9251975496C3
:10DF40001C921E92539784E890E01D969C938E93AA
:10DF50001C971E961C921E9782E755968C93559798
:10DF6000ED91FC9111970088F189E02D60E270E05D
:10DF7000CD011995B8018091530F9091540F0F94D2
:10DF800014288091530F9091540FDC01ED91FC9176
:10DF90000190F081E02D60E019958091530F9091F0
:10DFA000540FDC01ED91FC910488F589E02D199561
:10DFB0006A817B8187E79FE00F94142868E772E20B
:10DFC00087E79FE00F942A2887E79FE00F94BE26FB
:10DFD0008091290C90912A0C02973CF080EF9FEFE2
:10DFE00090932A0C8093290C62CF6BE672E281E851
:10DFF0009FE00F942A2881E89FE00F94BE2684EFCB
:10E0000091E057CFCF93DF93EB010297BCF169EA20
:10E0100072E28A819B810F941B55892B29F40E94FF
:10E02000A8F57D7F0E9402F663EB72E28A819B81F4
:10E030000F941B55892B29F40E94A8F572600E9449
:10E0400002F664E072E287E79FE00F942A280E94BC
:10E05000A8F571FB662760F971E0672770E04AE078
:10E0600050E087E79FE00F94CB2787E79FE00F946E
:10E07000BE2688EC90E0DF91CF9108950E94DB6E80
:10E08000F8CF892B71F0FB01828193810E94A3F369
:10E0900065E572E287E79FE00F942A2888EC90E01C
:10E0A000089590E080E0F2CFEF92FF920F931F93DC
:10E0B000CF93DF93CDB7DEB72C970FB6F894DEBFC2
:10E0C0000FBECDBF8C017B0180E495E09A838983EC
:10E0D0001B821C821D821E8298878F8319861A8656
:10E0E0001B861C8605301105ECF0BE01695F7F4F71
:10E0F000F701808591850E94F839892B99F0CE012E
:10E1000007960E946DF4BE01695F7F4FF70186811B
:10E1100097810E94F839892B61F0CE0107960E9401
:10E120003FF50EC0CE0101960E946DF4043011053A
:10E1300054F7CE0101960E943FF503301105A4F17A
:10E14000BE01695F7F4FF701848195810E94F83994
:10E15000892B51F1CE0107960E94D6F4BE01695F6A
:10E160007F4FF701828193810E94F839892B19F141
:10E17000CE0107960E9404F46EE372E287E79FE007
:10E180000F942A2880E00E9466F688EC90E02C9696
:10E190000FB6F894DEBF0FBECDBFDF91CF911F91B8
:10E1A0000F91FF90EF900895CE0101960E94D6F452
:10E1B000023011059CF6CE0101960E9404F4013054
:10E1C0001105D1F6CE0101960E9404F465E472E2D5
:10E1D00087E79FE00F942A28CFCF0F931F93CF9309
:10E1E000DF938C01EB010297C4F08A819B810F942D
:10E1F000CD548093450299270E946FF60230110595
:10E2000049F08C819D810F94CD54809344029927CD
:10E210000E9479F6C8ECD0E002C0C0E9D1E06AE221
:10E2200072E287E79FE00F942A284AE050E060916D
:10E23000450287E79FE00F94E12665E172E287E7F8
:10E240009FE00F942A284AE050E06091440287E75B
:10E250009FE00F94E12687E79FE00F94BE26CE0152
:10E26000DF91CF911F910F9108950F931F93CF933B
:10E27000DF93CDB7DEB769970FB6F894DEBF0FBE58
:10E28000CDBFE0918911F0918A11309709F460C0F7
:10E290008091931190919411892B09F459C08FEFBB
:10E2A0008387148613821482158216821782108641
:10E2B0001186128664E97FE187E79FE00F942A28A0
:10E2C00087E79FE00F94BE26BE016E5E7F4F809170
:10E2D000891190918A110F9484451816CCF5A89550
:10E2E000AE014F5F5F4F68E0CE0142960F94264625
:10E2F000198ABE016F5F7F4F8091931190919411A5
:10E300000E9470F18C016FE87FE187E79FE00F9436
:10E310002A28BE016F5F7F4F87E79FE00F94142884
:10E320000115110591F0C8010E945E3C8C01892BFA
:10E3300059F26AE87FE187E79FE00F942A28B80145
:10E3400087E79FE00F941428BBCF65E87FE1B4CF47
:10E3500088EC90E069960FB6F894DEBF0FBECDBF93
:10E36000DF91CF911F910F910895CF92DF92EF929D
:10E37000FF920F931F93CF93DF9300D000D0CDB7C0
:10E38000DEB78091710A81119CC08091290C909117
:10E390002A0C02970CF495C08091DD0A9091DE0A58
:10E3A000009709F48EC06BEE77E00E9470F18C014B
:10E3B000009709F486C00E94B3F2E82EF12CE11414
:10E3C000F10409F47EC070E060E0C8010F94D74604
:10E3D0006C01EA94EF2809F483C061E0C8010E944F
:10E3E00022F2FC0101851285CE0101960E948CFF6C
:10E3F000CE0101960E94AAFF67E478E187E79FE0DB
:10E400000F942A28B60187E79FE00F94142861E251
:10E4100077E087E79FE00F9414284AE050E0B801C6
:10E4200087E79FE00F94CB2761E277E087E79FE0E3
:10E430000F94142862EC7BE087E79FE00F94142888
:10E4400087E79FE00F94BE2662E072E086E490E1E9
:10E450000F94F237D0923C10C0923B1010933E10B4
:10E4600000933D1082EC9BE0892BE9F589EE97E063
:10E470009093401080933F108091500B9091510BDE
:10E48000009741F070E060E00F94D7469093730AD4
:10E490008093720A8091720A9091730A009731F109
:10E4A00090934210809341101092441010924310A8
:10E4B00081E08093710A6EE278E187E79FE00F9434
:10E4C0002A2826960FB6F894DEBF0FBECDBFDF9187
:10E4D000CF911F910F91FF90EF90DF90CF90089513
:10E4E00002E012E081CF82EC9BE0C2CF8FEC92E0A1
:10E4F000D7CFCF92DF92EF92FF920F931F93CF93DC
:10E50000DF93CDB7DEB7C154D1090FB6F894DEBFA3
:10E510000FBECDBF6C01AB0130E020E060E4CE0166
:10E5200001967C010E940E39F70101900020E9F765
:10E5300031978F010E191F09A801B701C6010F9469
:10E540007C61892B11F010E000E0C801CF5BDF4F48
:10E550000FB6F894DEBF0FBECDBFDF91CF911F91F4
:10E560000F91FF90EF90DF90CF900895CF92DF92C0
:10E57000EF92FF920F931F93CF93DF93EC01EC8107
:10E58000FD81309709F4A4C08A819B81892B09F40D
:10E590009FC08081882309F49BC07A016B01E881C8
:10E5A000F9810284F385E02DCE0119950397D9F402
:10E5B000EC81FD8180A591A5A2A5B3A5892B8A2B0D
:10E5C0008B2B89F00F94AD06EC81FD8100A511A580
:10E5D00022A533A5601B710B820B930B6639710565
:10E5E0008105910528F38F81988521E0E21AF108D1
:10E5F000DC01ED91FC910280F381E02DA701B601D1
:10E6000019958F819885DC01ED91FC910190F08145
:10E61000E02DD601129660E09D012C193D092E15C2
:10E620003F0518F42D91620FF7CF19950C811D81CC
:10E630004FEF5FEFBA0180E00F946747F80160A7E2
:10E6400071A782A793A76CE179E288E290E10F9429
:10E650002A284AE050E06E8188E290E10F94E1269A
:10E6600067E179E288E290E10F942A288601C801E7
:10E670008C199D098E159F05B8F4D8016C9140E165
:10E6800050E06A3050F469EF75E088E290E10F9451
:10E69000142840E150E0F801608188E290E10F9495
:10E6A000E1260F5F1F4FE3CF88E290E10F94BE2673
:10E6B000E881F9810484F585E02D63E0CE01DF91E6
:10E6C000CF911F910F91FF90EF90DF90CF90199411
:10E6D000DF91CF911F910F91FF90EF90DF90CF903E
:10E6E00008958F929F92AF92BF92CF92DF92EF9256
:10E6F000FF920F931F93CF93DF9300D000D01F9210
:10E700001F92CDB7DEB7E982FA820B831C832D837B
:10E710003E834F835887DC011296ED91FC91309730
:10E7200091F1048115810115110569F1F8018085C8
:10E730008F70853041F57B01C8010E94B3F28230B1
:10E7400010F161E0C8010E9422F20097E1F0DC01C3
:10E7500018962C912F702630B1F4B7010E9470F1F9
:10E76000009789F0912C812CB12CA12CD12CC12C9B
:10E77000E980FA800B811C812D813E814F81588573
:10E780006FEF0E94804328960FB6F894DEBF0FBE4D
:10E79000CDBFDF91CF911F910F91FF90EF90DF9050
:10E7A000CF90BF90AF909F908F900895EF92FF927F
:10E7B0001F93CF93DF93192F7B01C82FD92FD7FF3A
:10E7C00003C0D195C195D10961E08C2F0F947602D9
:10E7D00082E0E816F10499F460E08C2F0F9448026F
:10E7E0006EE377E288E290E10F942A2888E290E1D4
:10E7F000DF91CF911F91FF90EF900D94BE26612F76
:10E80000EF2851F46095661F6627661F8C2F0F94C2
:10E8100048026AE377E2E6CF661F6627661F8C2F01
:10E820000F94480265E377E2DDCFAF92BF92DF92AB
:10E83000EF92FF920F931F93CF93DF93CDB7DEB785
:10E840002E970FB6F894DEBF0FBECDBF20918F116B
:10E8500030919011232B09F4B8C020918E11211111
:10E86000B4C07C0180918E118F5F80938E11809156
:10E870008D118F5F80938D110F94AD0600915A0B0F
:10E8800010915B0B20915C0B30915D0B601B710B49
:10E89000820B930B6B3071058105910508F48BC0D9
:10E8A00083E0E816F104A9F00F94AD060091560B31
:10E8B0001091570B2091580B3091590B601B710B25
:10E8C000820B930BDD24D394643671058105910589
:10E8D00008F4D12CE0918F11F091901106811781ED
:10E8E0000115110509F449C0F80180858F70863043
:10E8F00009F03FC01987088770E060E0CE010896F4
:10E900000E94CDDBB701CE0108960E940DDFDD200D
:10E9100031F064E070E0CE0108960E940DDF61EAFC
:10E9200076E0C8010E9470F1FC01892B11F19085FD
:10E930009F7095509230E8F4A680B780A114B1047E
:10E94000C1F0BA82A982B801CE0101960E94CDDB46
:10E95000B701CE0101960E940DDFDD2031F064E0A9
:10E9600070E0CE0101960E940DDFF501A280B38018
:10E97000E5CFF80102811381B3CFF3E0EF16F10484
:10E9800051F00F94AD0660935A0B70935B0B80931C
:10E990005C0B90935D0BDD2051F00F94AD066093FE
:10E9A000560B7093570B8093580B9093590B109202
:10E9B00095101092961080918D11815080938D1139
:10E9C00080918E11815080938E112E960FB6F894FF
:10E9D000DEBF0FBECDBFDF91CF911F910F91FF9092
:10E9E000EF90DF90BF90AF900895A89582E090E0FF
:10E9F0000C9415748091280C8F5F8093280CA89537
:10EA000083E090E00E9415740F94BB2F8091280C36
:10EA100081508093280C089563E177E287E79FE0B7
:10EA20000F942A2860E077E287E79FE00F942A2876
:10EA300062EF76E287E79FE00F942A286AEE76E29B
:10EA400087E79FE00F942A2887E79FE00F94BE2670
:10EA50006AED76E287E79FE00F942A286EEC76E273
:10EA600087E79FE00F942A2861EC76E287E79FE032
:10EA70000F942A286CEA76E287E79FE00F942A2811
:10EA80006DE976E287E79FE00F942A2865E976E250
:10EA900087E79FE00F942A2864E876E287E79FE003
:10EAA0000F942A286EE576E287E79FE00F942A28E4
:10EAB00061E576E287E79FE00F942A2867E476E233
:10EAC00087E79FE00F942A2868E376E287E79FE0D4
:10EAD0000F942A2860E376E287E79FE00F942A28C4
:10EAE00064E276E287E79FE00F942A286AE076E204
:10EAF00087E79FE00F942A286BEE75E287E79FE097
:10EB00000F942A2866ED75E287E79FE00F942A2884
:10EB10006EEB75E287E79FE00F942A2860EB75E2C1
:10EB200087E79FE00F942A2864EA75E287E79FE071
:10EB30000F942A286CE975E287E79FE00F942A2852
:10EB400061E975E287E79FE00F942A2864E875E29F
:10EB500087E79FE00F942A286CE775E287E79FE03C
:10EB60000F942A2861E775E287E79FE00F942A282F
:10EB700062E675E287E79FE00F942A2869E575E26F
:10EB800087E79FE00F942A286BE475E287E79FE010
:10EB90000F942A286DE375E287E79FE00F942A28F7
:10EBA00061E375E287E79FE00F942A2869E275E246
:10EBB00087E79FE00F942A2866E175E287E79FE0E8
:10EBC0000F942A286CE075E287E79FE00F942A28CB
:10EBD00087E79FE00D94BE260F931F93CF93DF939B
:10EBE00000D000D0CDB7DEB70E940C756FED7CE190
:10EBF00087E79FE00F942A28CE0101960E948CFFA0
:10EC0000CE0101960E94A23900E415E01A8309831F
:10EC10008091740D9091750DA091760DB091770D46
:10EC20008B839C83AD83BE83CE0101960E94A23963
:10EC30001A8309831B821C821D821E8280E590E05C
:10EC40000E9489FF44E050E0BE016D5F7F4F81E08C
:10EC500090E00F94A8320F949F33CE0101960E944A
:10EC6000A2391A8309831B821C821D821E8280E5C1
:10EC700090E00E9489FF44E050E0BE016D5F7F4F4D
:10EC800085E090E00F94A8320F949F33CE01019657
:10EC90000E94A23965E07DE187E79FE00F942A2872
:10ECA00088EC90E026960FB6F894DEBF0FBECDBF7D
:10ECB000DF91CF911F910F910895CF92DF92EF9244
:10ECC000FF921F93CF93DF9300D000D0CDB7DEB774
:10ECD00069E278E187E79FE00F942A288BE5E82E28
:10ECE0008FE0F82E10E090E1C92ED12CF701819130
:10ECF0007F01803130F469EF75E087E79FE00F9482
:10ED00001428153041F1F7013197808190E0B0E08F
:10ED1000A0E089839A83AB83BC83DE82CD82BE016F
:10ED20006F5F7F4F87E79FE00E941ABC67E278E140
:10ED30000F942A281F5F1630C9F626960FB6F8944E
:10ED4000DEBF0FBECDBFDF91CF911F91FF90EF903F
:10ED5000DF90CF9008958091600F90E0B0E0A0E048
:10ED600089839A83AB83BC83DE82CD82BE016F5FD1
:10ED70007F4F87E79FE00E941ABC0F94BE26DACF30
:10ED8000EF92FF920F931F93CF93DF9300D000D0A9
:10ED90001F92CDB7DEB77B01CE0107969F938F936D
:10EDA00001979F938F9301979F938F9301979F93C1
:10EDB0008F9301979F938F9301979F938F938E01CA
:10EDC0000F5F1F4F1F930F9382EF97E09F938F93D7
:10EDD000DB0113968C9113978F9312968C918F93DE
:10EDE0000F9411620FB6F894DEBF0FBECDBF069729
:10EDF000ECF469E973E281E89FE00F942A28D701D7
:10EE000012966D917C9181E89FE00F94142880E91F
:10EE100091E027960FB6F894DEBF0FBECDBFDF910D
:10EE2000CF911F910F91FF90EF9008958091530F14
:10EE30009091540F892B09F449C00E94C3F2882392
:10EE400009F444C0A091530FB091540F52961C92F4
:10EE50001E92519754961C921E92539784E890E00C
:10EE60001D969C938E931C971E961C921E9782E76C
:10EE700055968C935597ED91FC9111970088F189E7
:10EE8000E02D64E070E0CD0119958091530F9091D1
:10EE9000540FDC01ED91FC910280F381E02D46E0FE
:10EEA00050E0B801199586E0F801ABE5BFE00190AC
:10EEB0000D928A95E1F78091530F9091540FDC01E8
:10EEC000ED91FC910488F589E02D19950E945D76FD
:10EED0006BEA73E287E79FE00F942A2888EC90E0C2
:10EEE00098CFCF92DF92FF920F931F93CF93DF9330
:10EEF000F12C6115710509F48DC06A01EB018C01DB
:10EF0000CB010E9456B2F82E882309F483C0D6FEA6
:10EF10000EC0D8018C918B3009F450C008F041C06C
:10EF200040E051E060E070E08A3009F450C0D4FE67
:10EF300009C0F801608186EF860F843018F0CE0199
:10EF40000E94C7BAD5FE66C0D80114964D915D9156
:10EF50006D917C91179711968C918F70873030F05E
:10EF60008930C8F18A50823008F45DC0CE010E9419
:10EF700003B3EE81FF81309709F44CC080858F7018
:10EF80009EEF980F923010F0811144C0D801119675
:10EF90008C91982F9295907F80858F70892B808798
:10EFA00039C08C3081F040E056E060E070E08D3098
:10EFB00009F0BDCFCE010E947BB4B9CF40E051E053
:10EFC00060E070E0F7CF40E056E060E070E0CE0136
:10EFD0000E9452B4ACCFEE81FF813097D9F080858A
:10EFE0008F709EEF980F923010F0811113C04187FF
:10EFF000528763877487EE81FF818085807F83607D
:10F000008087EE81FF818085982F907F8F70806749
:10F01000903629F28F2DDF91CF911F910F91FF90A4
:10F02000DF90CF900895CE010E9403B3F3CFCF932A
:10F03000DF9300D000D01F921F92CDB7DEB7FC0146
:10F04000628398E0DE01119601900D929A95E1F7A6
:10F0500029813A814B815C816D817E818F81988588
:10F0600028960FB6F894DEBF0FBECDBFDF91CF91CB
:10F070000895CF93DF9300D000D01F921F92CDB799
:10F08000DEB7FC01608398E0DE01119601900D92DD
:10F090009A95E1F729813A814B815C816D817E816E
:10F0A0008F81988528960FB6F894DEBF0FBECDBF2E
:10F0B000DF91CF910895CF93DF9300D000D01F92BE
:10F0C0001F92CDB7DEB7FC019181907F9A6091834A
:10F0D000448355836683778388E0DE01119601902F
:10F0E0000D928A95E1F729813A814B815C816D818E
:10F0F0007E818F81988528960FB6F894DEBF0FBE6B
:10F10000CDBFDF91CF910895AF92BF92CF92DF92A2
:10F11000EF92FF920F931F93CF93DF9300D000D015
:10F120001F921F92CDB7DEB76115710509F45FC05C
:10F130005A016B017C01CB010E9456B2082F882333
:10F1400069F1D60116968D919C91009709F443C000
:10F15000FC011085212F2F703EEF320F323010F05E
:10F1600021112EC012951F70B4FE59C0C6010E9415
:10F17000E6BAF7018083112381F18181807F182B0A
:10F180001183D6011696ED91FC9181859285A38518
:10F19000B485F70184839583A683B783802F28964F
:10F1A0000FB6F894DEBF0FBECDBFDF91CF911F9198
:10F1B0000F91FF90EF90DF90CF90BF90AF900895A8
:10F1C000253049F460E00E9422F2009721F0DC0132
:10F1D00018961C91C7CF10E0C7CFD6011696ED91B7
:10F1E000FC9180858F70823021F0833051F000E0F7
:10F1F000D5CF4185528563857485C7010E945B78B0
:10F20000CDCF4185528563857485F7018181807FEB
:10F21000876081834483558366837783BFCF1123BF
:10F22000E1F2F701AACFCF93DF9300D000D01F9275
:10F230001F92CDB7DEB7FC016F3F710519F014F0D6
:10F240006FEF70E077FD60E09181892F8F708150C2
:10F250008230C8F4648388E0DE01119601900D923B
:10F260008A95E1F729813A814B815C816D817E81AC
:10F270008F81988528960FB6F894DEBF0FBECDBF5C
:10F28000DF91CF910895907F91609183E3CFCF92EA
:10F29000DF92EF92FF92DC01362F1196EC911197DD
:10F2A000EF70EC3008F0B6C0F0E08827E55AF64879
:10F2B0008F4F0D94EF5C0D7A937993790A7A0A7ADD
:10F2C0000A7AD8799A790A7A0A7A677967791496E4
:10F2D0008D919D910D90BC91A02D662399F0B7FD65
:10F2E0009FC08F3F9105A105B10529F024F08FEF54
:10F2F00090E0A0E0B0E02FEF30E0A901481B590BEF
:10F30000CA010CC0B7FD89C08F3F9105A105B105A9
:10F3100029F024F08FEF90E0A0E0B0E0FF90EF90B4
:10F32000DF90CF90089514962C91822F90E0662361
:10F33000A9F3E1CF1496CD90DD90ED90FC90179756
:10F34000662301F120E030E0A901C701B6010F9466
:10F350002E5B87FD65C020E030E04FE753E4C70136
:10F36000B6010F94365E18160CF457C0A70196012B
:10F3700060E070E08FE793E40F94215D0F94005EEE
:10F38000CB01CCCF20E030E0A901C701B6010F943A
:10F390002E5B87FD42C020E030E04FE753E4C70119
:10F3A000B6010F94365E1816DCF1C701B601E6CF40
:10F3B00014966D917D918D919C9117973323B1F0A7
:10F3C0006D395FEF75078507950754F1611524E6E0
:10F3D0007207810591050CF52CE93FEF4FEF5FEFC8
:10F3E0000F949A5CC90181509F4F98CF6D394FEFB0
:10F3F0007407840794078CF0611554E6750781053E
:10F40000910574F424E630E040E050E00F949A5CFB
:10F41000C90184CF8FEF9FEF81CF90E080E07ECF56
:10F420008FEF90E07BCFCF93DF93EC01DB018981FD
:10F430008F708630E1F128F481508230C8F080E08E
:10F4400014C0873009F18A508230C8F72FEF30E0BE
:10F450000F94065D24E630E040E050E00F949A5CA3
:10F460002C833D834E835F8381E0DF91CF910895AC
:10F470002FEF30E00F94065D24E630E040E050E0EE
:10F480000F949A5C2C83F0CF2FEF30E00F94065D41
:10F4900024E630E040E050E00F949A5CCA01B901E4
:10F4A0000F94355B6C837D838E839F83DDCF2CE946
:10F4B00033E60F94065D24E630E040E050E00F9420
:10F4C0009A5C2C833D834E835F83B9CFDC01119618
:10F4D000EC911197EF70E150EB3008F039C0F0E09B
:10F4E0008827EA58F5488F4F0D94EF5C997A997AFE
:10F4F000A87A817A817A8A7AA17AA17AA17A817AA4
:10F50000817A14966D917D918D919C9117970F94AE
:10F51000355B089514966D917D918D919C9117970F
:10F5200024E630E040E050E00F949A5CCA01B90153
:10F53000EECF14966C9170E090E080E00F94335B16
:10F54000089514966D917D918D919C9117970895D2
:10F5500060E070E0CB010895DC011196EC91119709
:10F56000EF70E150EB3008F037C0F0E08827E4544A
:10F57000F5488F4F0D94EF5CCE7ACE7AEC7AC77A4D
:10F58000C77ADD7AD47AD47AD47AC77AC77A1496CD
:10F590006D917D918D919C911797089514966C9122
:10F5A00070E090E080E0089514966D917D918D91CA
:10F5B0009C9117970F94005E089514966D917D911C
:10F5C0008D919C91179724E630E040E050E00F9435
:10F5D0009A5CCA01B901089560E070E0CB0108951A
:10F5E000DC011196EC911197EF70E150EB3008F0CF
:10F5F0003EC0F0E08827E050F5488F4F0D94EF5C57
:10F60000167B167B377B0B7B0B7B307B217B217B37
:10F61000217B0B7B0B7B14962D913D914D915C9141
:10F620001797A4E6B0E00F94B95C089514966C9116
:10F6300084E6689FB0011124072E000C880B990BFB
:10F64000089520E030E048EC52E414966D917D91ED
:10F650008D919C9117970F94945B0F94005E089581
:10F6600014966D917D918D919C911797089560E00E
:10F6700070E0CB010895FC01A7812A2F2E7FC9F0ED
:10F6800081818F7081508330A0F4A695A150BB0B6F
:10F690002BE531E00F94065D24E630E040E050E0D9
:10F6A0000F949A5CDA01C90187569F4FAF4FBF4F45
:10F6B00008958FEF9FEF08952F923F924F925F92A0
:10F6C0006F927F928F929F92AF92BF92CF92DF9272
:10F6D000EF92FF920F93CF93DF9300D01F92CDB79D
:10F6E000DEB77C017A8369835C834B83DB011C92E8
:10F6F000FC0160818FEF860F883108F04BC034FF2A
:10F7000049C0FAE06F9FB0011124605C794ECD01D1
:10F710000F947055D70111968C918F7041F04B81E9
:10F720005C816CEC75E089819A810F946C61E98150
:10F73000FA8101900020E9F7319729813A81E21B93
:10F74000F30B19012E0E3F1E4B815C814E1B5F0B8C
:10F75000415051095C834B83D7011196EC9111976D
:10F76000EF7009F4F5C0E150EC3008F0F1C0F0E0C2
:10F770008827E254F4488F4F0D94EF5CCD7B707C6A
:10F78000DD7C3C7D577D1B7CED7CED7CED7C097C3C
:10F79000F17B737D29803A80DFCFF7018481282FA8
:10F7A00030E050E040E0002359F030E0A4E6B0E063
:10F7B0000F94CC5C2FEF30E040E050E00F949A5C67
:10F7C0005F934F933F932F9386E098E09F938F939F
:10F7D000FC81FF932B812F933F922F920F94A46172
:10F7E000B2C017968C9117978F9316968C91169797
:10F7F0008F9315968C9115978F9314968C918F9368
:10F8000089E098E09F938F93BC81BF93EB81EF9346
:10F81000E3CF17968C9117978F9316968C91169726
:10F820008F9315968C9115978F9314968C918F9337
:10F830008DE098E0E7CF1496CD90DD90ED90FC90B0
:10F840001797F7FE34C084E6882E912CA12CB12C9A
:10F85000C701B601A50194010F949A5C9B01AC010C
:10F8600088279927DC01821B930BA40BB50BBF9350
:10F87000AF939F938F9366277727CB016C197D09F0
:10F880008E099F09A50194010F949A5C5F934F9391
:10F890003F932F9381E198E09F938F933C813F9317
:10F8A0004B814F933F922F920F94A4614CC0C7019C
:10F8B000B60124E630E040E050E00F949A5C9F935C
:10F8C0008F937F936F935F934F933F932F9382E137
:10F8D00098E09F938F939C819F93AB81AF93E2CFEE
:10F8E000C7010E943B7BBC01D7011696CC901697AE
:10F8F0001796DC901797D0FADD24D0F814969C91D7
:10F9000014971596FC90EB80BC80292F30E050E0D6
:10F9100040E077FD35C0011135C07F936F931F9292
:10F920001F921F929F931F92FF92DF92CF928BE1C3
:10F9300098E09F938F93FC81FF932B812F933F92AD
:10F940002F920F94A4610FB6F894DEBF0FBECDBF07
:10F9500089819A810F900F900F900F90DF91CF9136
:10F960000F91FF90EF90DF90CF90BF90AF909F905E
:10F970008F907F906F905F904F903F902F90089561
:10F98000002361F0292F30E0A4E6B0E00F94CC5CB6
:10F990002FEF30E040E050E00F949A5C5F934F937C
:10F9A0003F932F931F92FF92DF92CF928EE198E0C8
:10F9B0009F938F93BF92EF9275CF15968C91159769
:10F9C0001F928F9316969C91169717968C91817023
:10F9D0008F939F9381E298E015CF14968D909D9020
:10F9E000AD90BC90179720E030E0A901C501B401AB
:10F9F0000F942E5B2401350187FF04C077FA7094C1
:10FA000077F87094C301B2010F94005E6B01072E6A
:10FA1000000C880B990B0F94355B9B01AC01C30163
:10FA2000B2010F94215D20E030E04AE754E40F94E6
:10FA3000945B0F948B5E0F94005E062F772E20E070
:10FA400030E0A901C501B4010F942E5B87FF07C008
:10FA50007F920F93DF92CF9287E298E0D3CE7F928E
:10FA60000F93DF92CF9288E298E09F938F933C812F
:10FA70003F934B814F93B0CE14968C9114971F9265
:10FA80008F9315968C9115971F928F9316968C9144
:10FA90001F928F938EE198E09F938F93BC81BF93C9
:10FAA000EB81EF933F922F920F94A4614CCF179666
:10FAB0008C9117971F928F9314968C9114971F9285
:10FAC0008F9315968C9115971F928F9316968C9104
:10FAD0001F928F938BE198E09F938F93BC81BF938C
:10FAE000EB81EF93DFCE14966D917C914B815C811D
:10FAF000C1010F948A612CCFEF92FF920F93CF93A5
:10FB0000DF93CDB7DEB7A0970FB6F894DEBF0FBE78
:10FB1000CDBF7C0100E020E030E340E250E0BE01D8
:10FB20006F5F7F4F0E945C7BBE016F5F7F4F88E2FB
:10FB300090E10F94142861E477E188E290E10F945A
:10FB40002A28F70161816F704AE050E088E290E175
:10FB50000F94E1266AE377E188E290E10F942A2886
:10FB60004AE050E0F701628188E290E10F94E126DB
:10FB700088E290E10F94BE26A0960FB6F894DEBFFF
:10FB80000FBECDBFDF91CF910F91FF90EF90089501
:10FB9000CF93DF93EC016115710539F48F8181708A
:10FBA0008F8381E0DF91CF9108958981982F9F7095
:10FBB00029F180E09430B0F79B01770F440B550B8F
:10FBC0002959310941095109A4E6B0E00F94B95C03
:10FBD0002BE531E040E050E00F949A5C37FF02C023
:10FBE00030E020E02536310514F024E630E02F5FC8
:10FBF000220F8F818170282B2F83D3CF807F82604B
:10FC00008983DACFFC019181892F8F7021F08230B6
:10FC100029F080E00895907F926091839B0177FFA7
:10FC200002C030E020E02E3681E0380714F02DE6E7
:10FC300031E02683878130FB80F9878381E0089556
:10FC4000EF92FF920F931F93CF93DF93FC01892BC9
:10FC500069F19081992351F19D3291F180ED890FE5
:10FC60008A3070F1C8E0D0E0953211F1CEEFDFEFCD
:10FC70009B37F1F0C7E1D0E09332D1F08F018AE4F5
:10FC8000E82E86E1F82EC1E0D0E0C7010F94495577
:10FC9000AC01B701C8010F946255892B49F0219638
:10FCA0008AE0E80EF11CC931D10579F7CFEFDFEF1B
:10FCB000CE01DF91CF911F910F91FF90EF900895AA
:10FCC000D0E0C0E0F5CFEF92FF920F931F93CF9358
:10FCD000DF93EC01892B51F188858F70843009F511
:10FCE000E984FA84C7010E94207E8C011816190647
:10FCF000ECF4C7010F940F30C801012E000CAA0BC1
:10FD0000BB0B89879A87AB87BC878885807F826099
:10FD10008887C801DF91CF911F910F91FF90EF90DD
:10FD20000895823019F409851A85F3CF10E000E0B8
:10FD3000F0CF2F923F924F925F926F927F928F926D
:10FD40009F92AF92BF92CF92DF92EF92FF920F936A
:10FD50001F93CF93DF93CDB7DEB7A4970FB6F89478
:10FD6000DEBF0FBECDBF7C016B0169EE75E0C60141
:10FD70000E9470F1FC01892B09F422C180858F70EB
:10FD8000843009F455C0853009F01AC10681178105
:10FD90000115110509F414C1D80118968C91189712
:10FDA0008F70823019F412960D911C910115110576
:10FDB00009F406C1F80180858F70853011F0D801F3
:10FDC000F2CFC8010E94B3F28230C9F760E0C801E7
:10FDD0000E9422F25C010E94637E61E0C8010E94E1
:10FDE00022F24C01FC0180858F70823041F7C701FF
:10FDF0000E94AC7AD40119964D905D906D907C90E4
:10FE00001C976415750586059705C9F6A114B104FC
:10FE100009F4D6C019861A861B861C861D861E8686
:10FE20001F86188A8A85807F8A87F50161854DC083
:10FE30006EEE75E0818592850F945C61892B09F0E7
:10FE4000BFC0C7010E94AC7A61157105810591059B
:10FE500009F49CC0660F771F881F991F2FEF30E0B1
:10FE600040E050E00F949A5C57FD16C023303105F6
:10FE7000410551050CF070C0DA01C9010196A11DC0
:10FE8000B11D82309105A105B10509F44BC003975E
:10FE9000A105B10509F460C0198A1A8A1B8A1C8A57
:10FEA0001D8A1E8A1F8A188E8A89807F8A8B67E046
:10FEB000CE0141960E94177829873A874B875C8745
:10FEC0006D877E878F87988B62E1CE0109960E94AD
:10FED000397829833A834B835C836D837E838F8358
:10FEE000988729813A814B815C816D817E818F81E8
:10FEF0009885A4960FB6F894DEBF0FBECDBFDF91F4
:10FF0000CF911F910F91FF90EF90DF90CF90BF9016
:10FF1000AF909F908F907F906F905F904F903F90A9
:10FF20002F900895198A1A8A1B8A1C8A1D8A1E8A94
:10FF30001F8A188E8A89807F8A8B67E0CE0141965E
:10FF40000E94177829873A874B875C876D877E8761
:10FF50008F87988B61E1B9CF198A1A8A1B8A1C8A0C
:10FF60001D8A1E8A1F8A188E8A89807F8A8B67E085
:10FF7000CE0141960E94177829873A874B875C8784
:10FF80006D877E878F87988B60E19FCF198A1A8A49
:10FF90001B8A1C8A1D8A1E8A1F8A188E8A89807F66
:10FFA0008A8B67E0CE0141960E94177829873A87AD
:10FFB0004B875C876D877E878F87988B62E085CFC4
:10FFC00060E476E0C6010E9470F18C01009709F4AC
:10FFD0001CC1DC0118968C918F70853009F0FEC031
:10FFE000C8010E94B3F2843008F40FC160E0C80178
:10FFF0000E9422F25C0161E0C8010E9422F23C01F1
:020000021000EC
:1000000062E0C8010E9422F2DC0119962D913D9117
:100010004D915C911C97298F3A8F4B8F5C8F63E0D9
:10002000C8010E9422F24C0165E0C8010E9422F240
:100030006C0167E0C8010E9422F28C01C7010E9496
:10004000AC7A298D3A8D4B8D5C8D621773078407CE
:10005000950714F5C114D10409F4C2C0D60118964D
:100060008C9118978F70823009F0BAC019861A8661
:100070001B861C861D861E861F86188A8A85807FA1
:100080008A8719964D915D916D917C911C97CE0157
:1000900009960E945B781DCFD40119962D913D9150
:1000A0004D915C911C972D8F3E8F4F8F58A3261733
:1000B000370748075907D4F40115110509F490C012
:1000C000F80180858F70823009F08AC019861A86FF
:1000D0001B861C861D861E861F86188A8A85807F41
:1000E0008A874185528563857485D1CFD50119965C
:1000F000CD90DC90F3012184328419861A861B8608
:100100001C861D861E861F86188A8A85807F8A87A0
:100110002101032C000C6608770846010D2C000C09
:10012000AA08BB08098D1A8D012E000C220B330B77
:1001300009A31AA32BA33CA3C7010E94AC7A9B017D
:10014000AC01E9A0FAA00BA11CA12E193F09400B9C
:10015000510BC301B201681979098A099B090F94EF
:10016000685C0D8D1E8D9801110F440B550BE9A095
:10017000FAA00BA11CA12E193F09400B510B0F94A3
:100180009A5C820E931EA41EB51EC1018C199D0996
:100190006D8D7E8D098D1A8D601B710B0F94DB5C4C
:1001A00077FF02C06F5F7F4F75956795CB01770F23
:1001B000AA0BBB0B880D991DAA1DBB1D40E050E08A
:1001C000BA01B7FD64CFB301A20184179507A60752
:1001D000B7070CF05CCFAC01BD0159CF811115C040
:1001E00019861A861B861C868A85807F8A871D86CB
:1001F0001E861F86188A88E0FE013996DE01119658
:1002000001900D928A95E1F76CCE88E0F701F6CF68
:100210002F923F924F925F926F927F928F929F9216
:10022000AF92BF92CF92DF92EF92FF920F931F9304
:10023000CF93DF93CDB7DEB765970FB6F894DEBFE7
:100240000FBECDBF6115710549F528E0FC01DE0147
:10025000119601900D922A95E1F729813A814B81FF
:100260005C816D817E818F81988565960FB6F8944B
:10027000DEBF0FBECDBFDF91CF911F910F91FF90D9
:10028000EF90DF90CF90BF90AF909F908F907F9036
:100290006F905F904F903F902F9008953B018C019D
:1002A00069EE75E0C3010E9470F16C01D801FC9009
:1002B000FF2009F45AC0009709F457C0FC0180855B
:1002C0008F70843009F4DEC0853009F04EC0809113
:1002D0004502893020F480914402893050F060E377
:1002E00078E088E290E10F94142888E290E10F947E
:1002F000BE26D6011696ED90FC90E114F104A9F10A
:10030000F70180858F705701823069F0B12CA12CE4
:10031000E114F10409F436C1D70118968C918F705D
:10032000853021F0F701E280F380F2CFC7010E940F
:10033000B3F28230B9F760E0C7010E9422F20E9456
:10034000637E4C0161E0C7010E9422F26C01D8017A
:100350008C918815190431F7F60180858F708230F1
:1003600009F7C114D10409F017C160E476E0C301B4
:100370000E9470F17C01D80111968C918F7009F464
:100380003BC1E114F10409F43BC1F70180858F7092
:10039000853009F0D0C1C7010E94B3F2843008F45F
:1003A000CAC164E0C7010E9422F26C0166E0C70185
:1003B0000E9422F21C01C8010E94AC7A4B015C0130
:1003C00060E0C7010E9422F2DC0119964D905D9019
:1003D0006D907C901C97B0914502B98B8414950464
:1003E000A604B7040CF016C1B93020F48091440281
:1003F000893050F160E276E188E290E10F942A289A
:10040000C8010E94AC7AAB01BC012AE030E088E26E
:1004100090E10F9483276AE076E188E290E10F94FF
:100420002A2860E0C7010E9422F2FC014185528522
:10043000638574852AE030E088E290E10F94832799
:1004400088E290E10F94BE26C114D10409F479C169
:10045000D60118968C9118978F70823009F071C16F
:1004600019821A821B821C821D821E821F8218869C
:100470008A81807F8A8319964D915D916D917C91DF
:100480001C9743C06EEE75E0818592850F945C6188
:10049000892B09F06ACFB0E1FB1609F463C0BF15E0
:1004A00080F0E2E0FE1619F1D8014D915D916D9159
:1004B0007C91139714968D919D910D90BC91A02DD8
:1004C00038C0F1E1FF16F1F122E1F212EDCF19820D
:1004D0001A821B821C821D821E821F8218868A81BC
:1004E000807F8A8344E150E060E070E00EC01982B2
:1004F0001A821B821C821D821E821F8218868A819C
:10050000807F8A8340E050E0BA01CE0101960E94CC
:100510005B7829873A874B875C876D877E878F87D3
:10052000988B49855A856B857C858D859E85AF85A1
:10053000B88949835A836B837C838D839E83AF8381
:10054000B8878BCE19821A821B821C821D821E8262
:100550001F8218868A81807F8A8340E850E060E0AD
:1005600070E0D3CF19821A821B821C821D821E82E8
:100570001F8218868A81807F8A834FEF50E060E077
:1005800070E0C3CFA114B10409F4EFCEF50180856A
:100590008F7009F4EACE650180914502893020F41C
:1005A000809144028930B8F06CE276E188E290E113
:1005B0000F942A28D60119964D915D916D917C91E9
:1005C0001C972AE030E088E290E10F94832788E2CC
:1005D00090E10F94BE2619821A821B821C821D8212
:1005E0001E821F8218868A81807F8A83F601418558
:1005F00052856385748589CFE114F10409F09BC0AD
:10060000F801408151816281738184819581A68145
:10061000B7818FCF61E0C7010E9422F2DC011996F9
:100620002D913D914D915C911C972A8B3B8B4C8B6E
:100630005D8B281539054A055B053CF5B989B9304C
:1006400020F480914402893050F06CEE75E188E22C
:1006500090E10F942A2888E290E10F94BE2621149D
:10066000310409F46EC0F10180858F70823009F089
:1006700068C019821A821B821C821D821E821F8200
:1006800018868A81807F8A83B2CF63E0C7010E9487
:1006900022F28C0162E0C7010E9422F2DC0119966D
:1006A000CD90DD90ED90FC901C97F801218532856E
:1006B000438554852C193D094E095F09C501B401D4
:1006C00064197509860997090F94685C2A893B8922
:1006D0004C895D8924193509460957090F949A5C9C
:1006E000C20ED31EE41EF51EF989F93020F4809164
:1006F0004402893090F067ED75E188E290E10F9453
:100700002A282AE030E0B701A60188E290E10F94A0
:10071000832788E290E10F94BE2619821A821B82F9
:100720001C821D821E821F8218868A81807F8A8396
:10073000B701A601EACED70118968C918F7009F007
:100740005FCF19821A821B821C828A81807F8A83F2
:1007500049815A816B817C8180E090E0DC01E9CEA7
:100760008F929F92AF92BF92CF92DF92FF920F93A0
:100770001F93CF93DF93EC018A819B810E94B3F298
:10078000082F10E00430110554F40E9483F7BC01D7
:100790008A819B810E9490F70F5F1F4FF3CFEA8100
:1007A000FB81068117810115110531F0D8011296E0
:1007B0008D919C919D838C83EC81FD81309721F0FC
:1007C000828193819F838E83EE81FF81309749F0F0
:1007D0000280F381E02D309721F082819381998707
:1007E00088870115110541F0F80180858F708430EC
:1007F00059F128F4823071F0FF24FA940CC085304E
:1008000001F18630C9F76FEA75E0C8010E9470F106
:100810008C01E7CFF184FA86CE010E9456B2811195
:1008200038C010E000E01C870B87DF91CF911F914B
:100830000F91FF90DF90CF90BF90AF909F908F90DF
:10084000089506811781CDCFC184D284C114D1040B
:1008500099F2F6018081882379F291E7892E94E15B
:10086000992EB12CA12CFA2CC4010F944955AC013E
:10087000B401C6010F946255892BB9F1FFEFAF1A8D
:10088000BF0A89E0880E911CA7E1AA16B10459F7A6
:10089000B3CFCE010E9498F68C010097B1F0FC0115
:1008A00082819381892B39F08F2D0E94AEF78C01C4
:1008B000892B09F4B6CFD801ED91FC910684F78518
:1008C000E02DBE01C8011995AECF8F2D0E94AEF765
:1008D0008C01892B09F4A5CFEA85F0E0EE0FFF1F0C
:1008E000E959FF4E11830083E6CFC6010F940F3004
:1008F0008A2D90E0B0E0A0E0F80181879287A3877D
:10090000B4878085807F8260808785CF8F929F9219
:10091000AF92BF92CF92DF92EF92FF920F931F930D
:10092000CF93DF93CDB7DEB760970FB6F894DEBFF5
:100930000FBECDBF8C017B0140E050E860E070E06D
:100940000E94A4B4672B682B692B09F0B5C062E044
:1009500070E0C8010E9473B36C0119861A861B8669
:100960001C861D861E861F86188A8A85807F8A8738
:10097000D7FCA2C040E050E2B801CE0109960E9427
:10098000847863E070E0C8010E9473B3AC0118166C
:10099000190614F04FE350E081E0C816D10429F4A1
:1009A000EF2CFF0CFF08FF2404C082E0C816D1041E
:1009B000D4F32FEF30E0D7010F94065D9A01550F65
:1009C000440B550B0F949A5C49016901C8010E94C0
:1009D000E6BAE82EF12C60E0CE0109960E94477934
:1009E00088169906F9F4CD2841F082E0E816F10462
:1009F00019F185E0E816F104F9F081E090E06096E5
:100A00000FB6F894DEBF0FBECDBFDF91CF911F911F
:100A10000F91FF90EF90DF90CF90BF90AF909F909D
:100A20008F900895CD2899F186E0E816F10441F001
:100A300081E0E816F10421F061E0C8010E94C7BA24
:100A4000B401CE0109960E94137940E050E2B8014A
:100A5000CE0109960E94717782E0E816F10421F038
:100A600085E0E816F10449F430E020E040E050E190
:100A700060E070E0C8010E942BB830E020E040E068
:100A800050E260E070E0C8010E942BB8B6CF85E06C
:100A9000E816F10409F4B1CF82E0E816F10409F494
:100AA000ACCF62E0C8010E94C7BA30E020E040E06D
:100AB00050E160E070E0E7CF90E080E0A0CF3F92AF
:100AC0004F925F926F927F928F929F92AF92BF925E
:100AD000CF92DF92EF92FF920F931F93CF93DF930A
:100AE000CDB7DEB72C970FB6F894DEBF0FBECDBFE3
:100AF0005C01362E972E3A01690167E674E188E2BF
:100B000090E10F942A284AE050E0632D792D88E285
:100B100090E10F94CB276FE574E188E290E10F94A8
:100B20002A28C301B0E0A0E08F839887A987BA87FD
:100B300030E1432E512C5C864B86BE01695F7F4FAE
:100B400088E290E10E941ABC4C016BE574E10F94BD
:100B50002A284AE050E0B601C4010F94CB2763E590
:100B600074E1C4010F942A28C701B0E0A0E0898392
:100B70009A83AB83BC835E824D82BE016F5F7F4FE1
:100B8000C4010E941ABC0F94BE2680916F0A9091F6
:100B9000700A70E060E0892B09F047C081E090E0C6
:100BA0009093700A80936F0A26E040E855E260E077
:100BB00070E089EC9CE00F9477293092C90D89ECA4
:100BC0009CE09093C80D8093C70D1092D70E1092A1
:100BD000D90E1092D80E0130110509F44EC00CF058
:100BE00041C0012B09F44EC0C114D10409F457C00F
:100BF00082E0C816D10409F062C07092520E609271
:100C0000510E1092540E1092530EF092560EE09226
:100C1000550E86E00F943C081092700A10926F0AED
:100C2000882309F456C0682F70E0C5010E942ABCD1
:100C300090E080E02C960FB6F894DEBF0FBECDBFDB
:100C4000DF91CF911F910F91FF90EF90DF90CF90A8
:100C5000BF90AF909F908F907F906F905F904F90DC
:100C60003F9008950330110581F00430110509F01B
:100C7000BBCFFE24EF24FE24B7CFFE2CEE24EE24BF
:100C8000EA94B2CFFF24FA94AFCFEF2821F492E098
:100C9000E92EF12CEECFEE24E394F12CEACF709202
:100CA000520E6092510E90E080E0EE2011F080E054
:100CB0009FEF9093540E8093530E85E0ABCF67E384
:100CC00074E188E290E10F942A281092700A109241
:100CD0006F0A81E090E0AECFFF920F931F93CF9306
:100CE000DF9300D000D0CDB7DEB78C01BC01CE01C0
:100CF00001960F944B24BE016F5F7F4F88E290E115
:100D00000F941C2888E290E10F94BE26CE01019634
:100D10000F9443241A8219821C821B821E821D8218
:100D20006FED73E2CE0101960F94E623F801248162
:100D300035818D819E81F12C2817390738F0BE014D
:100D40006F5F7F4FC8010F94EC00F82ECE01019623
:100D50000F944324FF2069F0B801CE0101960F944F
:100D60004B24CE0101960F94530FCE0101960F94A0
:100D7000432426960FB6F894DEBF0FBECDBFDF9199
:100D8000CF911F910F91FF9008950F931F93CF93D1
:100D9000DF9300D000D0CDB7DEB7A091530FB09154
:100DA000540F109709F478C052961C921E925197D6
:100DB00054961C921E92539784E890E01D969C9343
:100DC0008E931C971E961C921E9787E755968C93C0
:100DD0005597ED91FC9111970088F189E02D70E015
:100DE00060E0CD01199510E000E08091530F9091E3
:100DF000540FDC01ED91FC9111971C962D913C91C3
:100E00000217130740F40190F081E02D60E019957E
:100E10000F5F1F4FEACF0088F189E02D70E060E09E
:100E200019950FE814E08091530F9091540FF80139
:100E300061918F01DC01ED91FC910190F081E02D39
:100E40001995B4E003391B0771F78091530F909106
:100E5000540FDC01ED91FC910488F589E02D199582
:100E60006BE17AE0CE0101960F945424CE010196F5
:100E70000F94530FCE0101960F94432487E090E026
:100E80000E946FF687E090E00E9479F664EB73E2CF
:100E900087E79FE00F942A281092730F1092720F29
:100EA00080E090E190936E0F80936D0F84E890E066
:100EB0009093750F8093740F81E080936F0F82E79A
:100EC0008093760F81E69FE00E9487AD81E69FE0E8
:100ED0000E94EDAD88EC90E026960FB6F894DEBF48
:100EE0000FBECDBFDF91CF911F910F9108956F92EB
:100EF0007F928F929F92AF92BF92CF92DF92EF92AA
:100F0000FF920F931F93CF93DF93CDB7DEB7AE97CA
:100F10000FB6F894DEBF0FBECDBF8091DD0A909171
:100F2000DE0A892B09F47FC680918D1181117BC661
:100F300080918D118F5F80938D116EE871E287E74C
:100F40009FE00F942A2887E79FE00F94BE26009128
:100F5000DD0A1091DE0A6EE378E0C8010E9470F1AC
:100F6000909392118093911164E478E0C8010E94FB
:100F700070F19093750A8093740A68ED79E0C80166
:100F80000E9470F19093901180938F116BE478E040
:100F9000C8010E9470F19093540B8093530B0097FB
:100FA00049F1DC011696ED91FC91309719F12085FD
:100FB0002F702530F9F46AE771E287E79FE00F941C
:100FC0002A288091530B9091540B0E94B3F2809386
:100FD000520B4AE050E0682F87E79FE00F94E1262C
:100FE00087E79FE00F94BE26E091530BF091540BDE
:100FF000868197819093510B8093500B0E94B5711D
:1010000060E578E08091DD0A9091DE0A0E9470F13F
:101010009093DC0A8093DB0A009709F4B2C00E9427
:10102000B3F2082F10E00115110509F4AAC0000F52
:10103000111F000F111F8091D90A9091DA0A892B94
:1010400009F08EC07801013811051CF040E8E42E4B
:10105000F12CC7010F9400539093DA0A8093D90AB8
:10106000E092D80A109282111092811110924F0BC7
:1010700010924E0B109280111092841110928311D5
:10108000C70101960F9400539093861180938511A8
:1010900090937F1180937E118E0D9F1D90937911F7
:1010A000809378110F94AD0660937A1170937B1141
:1010B00080937C1190937D1190E080E0E091851108
:1010C000F0918611E80FF91F10820196E816F906D3
:1010D000ACF782E090E0909382118093811180912F
:1010E0004E0B90914F0B009741F061E00F94760208
:1010F00060E080914E0B0F94480280E98093C90014
:101100001092C8001092CD0083E08093CC008EE056
:101110008093CA00F0924302E0924202209185112E
:10112000309186118091420290914302820F931F69
:101130009093791180937811232B09F45FC06AE0B2
:1011400071E288E290E10F942A28B70188E290E1E9
:101150000E9484F687E491EB909377118093761147
:1011600060E671E287E79FE00F942A284AE050E0AA
:10117000B80187E79FE00F94CB2787E79FE00F94A4
:10118000BE2666E578E08091DD0A9091DE0A0E9435
:1011900070F18C01009709F471C00E94B3F28823AA
:1011A00009F46CC06FEF680FC8010E9422F2FC01C5
:1011B000E184F28490917411992359F08091700028
:1011C0008E7F809370001092741110923E021092E4
:1011D0003D0282E180933C0291110F94CE40C70101
:1011E0000F94F64001E010E0E016F10674F060E0C4
:1011F000C8010F942A410F5F1F4FF6CF63EF70E2D3
:1012000088E290E10F944E28A5CF65EE70E288E267
:1012100090E10F942A280E948F3AAB01BC012AE08A
:1012200030E088E290E10F94D92688E290E10F94B3
:10123000BE2664E471E287E79FE00F942A284AE023
:1012400050E0B70187E79FE00F94CB2787E79FE047
:101250000F94BE266EE371E288E290E10F942A2893
:101260000E948F3AAB01BC012AE030E088E290E1B5
:101270000F94D92688E290E10F94BE260091DD0AF2
:101280001091DE0A6AE578E0C8010E9470F190933F
:101290006E0A80936D0A61E678E0C8010E9470F1E1
:1012A0009093941180939311892B09F448C08091F5
:1012B0009511811144C08091891190918A11892BD7
:1012C00009F0DFC16FEB70E288E290E10F942A2809
:1012D00088E290E10F94BE268FE090E00F940053D7
:1012E0008C0188E1D80111968C93119712961C926B
:1012F00012971C921E961C921E921D970E9414FE1D
:1013000010938A1100938911012B09F08CC060EBB6
:1013100070E281E89FE00F942A2881E89FE00F9413
:10132000BE2680E08170809395118091951188236D
:1013300031F06EE271E287E79FE00F942A28109265
:101340008C1110928B11E0919111F09192113097C4
:1013500009F4CCC2C680D7800091911110919211EE
:101360000115110509F4BBC2C114D10409F4B7C2B7
:10137000F60180858F70853099F7C6010E94B3F21F
:10138000823070F3A801B601CE0101960E9402BC22
:10139000CE0101960E9456B28823E1F18C859D858D
:1013A000009709F40DC2DC01ED91FC910284F385F4
:1013B000E02D1995892B49F08C859D85DC01ED91F7
:1013C000FC910084F185E02D19958C859D85DC01CB
:1013D000ED91FC910680F781E02D1995892BD1F0D4
:1013E000CE0101960E94E6BA882341F040E050E128
:1013F00060E070E0CE0101960E947BB48F819885F9
:10140000892B41F040E050E260E070E0CE010196AF
:101410000E947BB4D6011296CD90DC90CE0101964D
:101420000E94CFBB99CF0E9414FE809189119091A8
:101430008A110F9458418AE79DE00F94FD42811173
:1014400089C061E970E287E79FE00F944E288091A0
:10145000891190918A110F949C44E0918911F09127
:101460008A1181E080838091891190918A110F9473
:10147000AA446DE770E2811102C068E670E288E27A
:1014800090E10F944E288091931190919411892BA3
:1014900009F447CF8091871190918811892B09F029
:1014A000E2C083E190E00F9400538C018091891198
:1014B00090918A1129EC31E0F801328B218B9683CF
:1014C00085831482108289E0818381E08283838313
:1014D00010938811009387110F94AD066B017C0166
:1014E000F0E1CF0EF7E2DF1EE11CF11CD8011596EA
:1014F000ED91FC9116978FEF8387148613821482E7
:1015000015821682178210861186128614961C92F6
:10151000BB24B394BE01605E7F4FF8018581968144
:101520000F94844518160CF099C00F94AD066C15F5
:101530007D058E059F0508F091C0DE01909698E02C
:1015400080E0915039F1ED91E827F0E0EA5EFC4C43
:101550008491F7CF0F94ED468091891190918A1173
:101560000F9458418AE79DE00F94FD4281110BC012
:101570006BE470E287E79FE00F942A2887E79FE0FB
:101580000F94BE2680CF6FE270E281E89FE00F9457
:101590004E28C7CE9FA19813BDCFD8018C91811141
:1015A00038C015968D919C910F94AA44BE01605E3F
:1015B0007F4FF801858196810F947D4440E064EB74
:1015C000D80115968D919C910F945744F801858010
:1015D0009680C4010F94DB43C4010F94584167E81F
:1015E0008AE79DE00F94CB2160E88AE79DE00F94A5
:1015F000CB210E9480FEC4010F94DB43A82ED801AA
:1016000015968D919C910F94AA44A5FC02C0F801F7
:10161000B082AE014F5F5F4FBE01605E7F4FC80179
:101620000F94EB44D8011196AC9088A1803109F455
:10163000FCC2BE01605E7F4FC8010F945A458A15F7
:1016400010F5F8018181D80111968C9311971496A9
:101650008C9114978F5F14968C935CCFE0918711D7
:10166000F09188111282E0919311F0919411E6802B
:10167000F7803FE7D32E8091931190919411892B9D
:1016800071F481E04FCE88A1803111F48CE0DBCF82
:10169000BE01605E7F4FC8010F945A45D4CFE1145C
:1016A000F10479F3BE01605E7F4FF7018081918183
:1016B0000E94243C882329F368E170E288E290E1EB
:1016C0000F942A28D7016D917C9188E290E10F94C4
:1016D000142888E290E10F94BE26009187111091A2
:1016E0008811AE014F5F5F4FBE01605E7F4FC80142
:1016F0000F944045882309F45EC088A1803109F425
:101700005AC0DD82F801858196810F94AA44BE01FA
:10171000605E7F4FD80115968D919C910F947D440A
:1017200040E06EE4F801858196810F94574440E0D3
:101730006B81D80115968D919C910F94574440E090
:101740006C81F801858196810F94574488A180317E
:1017500041F040E06D81D80115968D919C910F94D8
:101760005744F801858196810F94AA44BE01605EBA
:101770007F4FD80115968D919C910F947D44F8016F
:10178000408168E4858196810F94574464E170E05C
:1017900080E090E00F94BB04D8018C91882331F055
:1017A0006AE070E080E090E00F94BB04F80185816E
:1017B00096810F94AA44D7011296ED90FC905BCFCE
:1017C00070E060E0CE0101960E9473B38C01912C11
:1017D000812C97FF06C011950195110988248394E7
:1017E000912CCE0101960E94E6BAE82EF12C8B8551
:1017F000853091F0863009F00DCEB02E61E0802F5B
:101800000F94760261E0892809F443C0EA94EF2836
:1018100009F043C060E041C0EF2829F462E0CE0146
:1018200001960E94C7BA40E050E160E070E0CE014E
:1018300001960E947BB48F819885892B41F040E00E
:1018400050E260E070E0CE0101960E947BB461E05E
:10185000802F0F94760260E0802F0F94480266E29A
:1018600071E288E290E10F942A284AE050E0B80142
:1018700088E290E10F94CB2761E271E288E290E187
:101880000F942A286FE171E288E290E10F942A28F0
:10189000C1CDEA94EF2809F0BDCFE62EF12C8B2DB7
:1018A0000F9448026AE171E288E290E10F942A28DD
:1018B0004AE050E0B80188E290E10F94CB2768E15C
:1018C00071E288E290E10F942A284AE050E0B701E3
:1018D00088E290E10F94CB2766E171E2D5CFF80161
:1018E0008681978190938C1180938B1188E290E18F
:1018F0000F94BE2664E070E287E79FE00F942A28E9
:1019000087E79FE00F94BE26E0918F11F091901130
:10191000309709F4CFC080918D118F5F80938D1126
:10192000068117815E01F8E2AF0EB11C8EEE682EC3
:1019300082E0782E9CED892E92E0992E01151105FA
:1019400009F4B3C0D80118968C918F70863009F0D5
:101950007CC019A708A770E060E0C5010E94CDDB3C
:101960008DA59EA5892B09F470C08091DD0A909108
:10197000DE0A892B09F469C0E8A4F9A4E114F10492
:10198000B9F1F70180858F70863091F5F9A2E8A250
:1019900070E060E0CE0180960E94CDDBEDA1FEA15B
:1019A000108211821282138261EA76E0C7010E94DE
:1019B00070F1FC01892BE1F090859F709550923079
:1019C000B8F4C680D780C114D10491F0DA82C982FC
:1019D000B701CE0101960E94CDDBEE81FF8110821E
:1019E000118212821382D6011296CD90DC90EBCF39
:1019F0006FEF7FE188E290E10F942A284AE050E0FF
:101A00006BA588E290E10F94E1266DEF7FE188E21B
:101A100090E10F942A284AE050E06AA588E290E11C
:101A20000F94E12688E290E10F94BE26EDA5FEA575
:101A300010821182128213828AA5853069F148F4DE
:101A40008230F0F060E08430E0F0F8010281138130
:101A500075CF8032A9F058F48630B9F7BC82AB82DA
:101A60009A828982CE0101960E94576DEECF803412
:101A700089F060E0823449F78BA50F947602E5CFB8
:101A800062E08BA50F947602EDA5FEA58181807F93
:101A90008183DBCF62E0F0CFBC82AB827A82698245
:101AA000CE0101960E94066ED0CF80918D1181509B
:101AB00080938D1160EF7FE187E79FE00F942A28E4
:101AC00068EE7FE187E79FE00F942A2881E020916C
:101AD000911130919211232B09F480E00E94CF697B
:101AE0006FED7FE187E79FE00F942A2881E0209146
:101AF0008F1130919011232B09F480E00E94CF695F
:101B000060ED7FE187E79FE00F942A2865EC7FE195
:101B100087E79FE00F942A2881E020916D0A309199
:101B20006E0A232B09F480E00E94CF696EEB7FE1FF
:101B300087E79FE00F942A2881E02091500B309195
:101B4000510B232B09F480E00E94CF6965EB7FE104
:101B500087E79FE00F942A2881E02091931130912C
:101B60009411232B09F480E00E94CF696CEA7FE195
:101B700087E79FE00F942A288091710A0E94CF691D
:101B800087E79FE00F94BE2667EA7FE187E79FE043
:101B90000F942A280E948F3AAB01BC012AE030E062
:101BA00087E79FE00F94D92687E79FE00F94BE2632
:101BB00081E08093550B86E49FE00F9427388823BB
:101BC00051F086E49FE00F94DF3E84E090E0909334
:101BD0002A0C8093290C8091290C90912A0C07974C
:101BE00031F484E090E090932A0C8093290C80914A
:101BF0008D11815080938D118091550BAE960FB64B
:101C0000F894DEBF0FBECDBFDF91CF911F910F9132
